:0200000460009A
:100400004643464200040156000000000103030079
:1004100001010000010400000200000000000000D3
:1004200000000000000000000000000000000000CC
:1004300000000000000000000000000000000000BC
:1004400000000000010403000000000000000000A4
:10045000000000010000000000000000000000009B
:10046000000000000000000000000000000000008C
:10047000000000000000000000000000000000007C
:10048000EB04180A063204260000000000000000F9
:10049000050402240000000000000000000000002D
:1004A000000000000000000000000000000000004C
:1004B0000604000000000000000000000000000032
:1004C00031040120000000000000000000000000D6
:1004D00020041808000000000000000000000000D8
:1004E000000000000000000000000000000000000C
:1004F00000000000000000000000000000000000FC
:10050000D8041808000000000000000000000000EF
:100510000204180804200000000000000000000091
:1005200000000000000000000000000000000000CB
:100530006004000000000000000000000000000057
:1005400000000000000000000000000000000000AB
:10055000000000000000000000000000000000009B
:10056000000000000000000000000000000000008B
:10057000000000000000000000000000000000007B
:10058000000000000000000000000000000000006B
:10059000000000000000000000000000000000005B
:1005A000000000000000000000000000000000004B
:1005B000000000000000000000000000000000003B
:1005C0000001000000100000010000000000000019
:1005D000000001000000000000000000000000001A
:1005E000000000000000000000000000000000000B
:1005F00000000000000000000000000000000000FB
:10100000D100204100C0006000000000000000008E
:1010100020100060001000600000000000000000D0
:10102000000000600000000100000000FFFFFFFF63
:10C0000000800020B97502609D380560D97A026011
:10C01000C17A0260C97A0260D17A02600000000031
:10C02000000000000000000000000000A5380560CE
:10C030009938056000000000A9380560AD3805603A
:10C04000B1380560B5380560B9380560BD380560A0
:10C05000C1380560C5380560C9380560CD38056050
:10C06000D1380560D5380560D9380560DD38056000
:10C07000E1380560E5380560E9380560ED380560B0
:10C08000F138056099380560993805609938056080
:10C09000F5380560F9380560FD380560013905603F
:10C0A0009938056009AF0260053905609938056067
:10C0B000093905600D3905609938056099380560C2
:10C0C00011390560153905609938056099380560A2
:10C0D0009938056099380560993805609938056088
:10C0E0009938056099380560993805609938056078
:10C0F0009938056099380560D579026099380560EE
:10C100009938056099380560993805609938056057
:10C110009938056099380560993805609938056047
:10C1200019390560993805601D39056021390560A8
:10C13000253905609938056099380560993805609A
:10C140009938056099380560993805609938056017
:10C150002939056099380560993805609938056076
:10C1600099380560993805609938056099380560F7
:10C1700099380560993805609938056099380560E7
:10C1800099380560993805609938056099380560D7
:10C1900099380560993805609938056099380560C7
:10C3F000993805609938056099380560FFFFFFFF9F
:10C40000044A03460020116A196011691362996495
:10C41000704700BF00040020024B1A6A12681A62BB
:10C42000704700BF00040020C46005614661876159
:10C43000C0F81C80C0F82090C0F824A0C0F828B034
:10C44000C0F82CD080ED0C8B80ED0E9B80ED10ABF6
:10C45000C0F808E0FFF7D4BF114A08B5136A0BB95A
:10C460001BF0A6F8996C58601161196811621846A2
:10C47000C468056946698769D0F81C80D0F82090A7
:10C48000D0F824A0D0F828B0D0F82CD090ED0C8BA8
:10C4900090ED0E9B90ED10ABD0F808E001207047B6
:10C4A0000004002010B50A460021044600F042FBBB
:10C4B00000B904B910BD204609F0C6FB0A460021A8
:10C4C00000F038BB10B50A460121044600F032FBEB
:10C4D00000B904B910BD204609F0B6FBFFF7E2BF72
:10C4E00010B501220C4600F093FC00B904B910BD50
:10C4F000204609F0A9FB00BF00F08ABC00F04CBC4C
:10C500002DE9F0434FF0030C00252B4CD4F8986133
:10C510000021013143189A0803F00303B25C5B0069
:10C5200042FA03F303F00303022BF2D0D4F8A43150
:10C53000090103EB00108B0819B300EB83010368BA
:10C540001A071BD1D4F8A4219A4217D8B2B19A1A6B
:10C55000D4F8A861C2F3011E9E424FEA92174FEA37
:10C560004E0E4FEA121209D9D4F8986116F80780D6
:10C5700048FA0EF303F00303012B09D0043088427C
:10C58000DDD1B5B1013D04EB8503D3F8B401BDE7BE
:10C590000CFA0EFE3F2D04EB85094EEA080E06F854
:10C5A00007E003D80135C9F8B421E7E7C4F8B03192
:10C5B000E4E7BDE8F08300BF00040020144A10B493
:10C5C000D2F8A431ABB1834213D8D2F8A811884273
:10C5D0000FD2C01AD2F898418109C0F301130009A3
:10C5E00014F801C05B004CFA03F202F00302012AC6
:10C5F00002D05DF8044B7047032202FA03F343EACA
:10C600000C0C04F801C05DF8044BFFF779BF00BFC4
:10C6100000040020F8B5244DD5F8A461002E40D0C8
:10C62000861B0123D5F8A0014FF0030EF109C6F3D4
:10C630000212370903FA02F2435CB60923EA020345
:10C6400007F00302B44643543846D5F89841A15D3B
:10C65000520001300EFA02F300F0030221EA030156
:10C66000530004F80C104FEA900CD5F8984114F8D8
:10C670000C1041FA03F303F00303022BE8D0C01BB4
:10C68000082828BF0820AD3055F820309E42D5F844
:10C69000D83238BF45F820609E4288BFC5F8D862BE
:10C6A000F8BD03201BF098FF00040020164A10B4C8
:10C6B000D2F8A431834204D81BB1D2F8A811884221
:10C6C00003D300205DF8044B7047C01AD2F898419C
:10C6D0008309C0F301120009E35C5200134103F027
:10C6E0000303012BEDD100230133C218910802F09E
:10C6F0000302615C520041FA02F202F00302022AD4
:10C70000F2D01801DEE700BF000400200F49D1F885
:10C71000A421131E18BF0123824288BF00230BB936
:10C7200018467047D1F8A831984202D30023184622
:10C730007047801AD1F8A021C309C0F30210D35C5E
:10C7400043FA00F000F0010318467047000400208F
:10C7500021F00F01194A38B50B1A194C013BC4F8E6
:10C76000A811C4F89801DB00A2FB03235B0AA1EB2C
:10C770008311C4F89C3101330A1AC4F8A41103448C
:10C780000021C4F8A03141F011FA2022002104F563
:10C790002E7041F00BFAD4F89C11D4F8A431002289
:10C7A000481E03EB81130121C4F8D802A282C4F809
:10C7B000AC3184F8B412C4F8DC2238BDF32C23FA6F
:10C7C00000040020024B988A003818BF01207047EF
:10C7D00000040020030701D1FFF7F0BE704700BF3F
:10C7E00070B50E4651B1051F002455F8040F0134F1
:10C7F000030701D1FFF7E2FEA642F6D170BD00BFEC
:10C8000070B5104E0022B38A06F1140406F5827545
:10C81000C6F8B0210133B38254F8040F020701D1E6
:10C82000FFF7CCFEA542F7D1D6F8DC02030701D111
:10C83000FFF7C4FEB0683169091ABDE87040890885
:10C84000FFF7CEBF000400202DE9F04F5F4C85B00C
:10C85000D4F8B031D4F89C61002B00F0B3800025EF
:10C860004FEA860CC4F8B051BCF1000F47D0002746
:10C8700007F00303B808D4F898115A000B5C134171
:10C8800003F00303032B48D001376745F0D3D4F8F6
:10C89000B031002BE6D1BCF1000F30D04FF0000ECC
:10C8A0004FF003094FF0010B4FF0020A774604E006
:10C8B000012B51D00137674521D2D4F898214FEA96
:10C8C000970807F0030512F8081002EB97006D00B7
:10C8D00041FA05F303F00303022B2ED0032BE7D11B
:10C8E0000AFA05F501374FF0000E21EA050102F8BA
:10C8F0000810D4F89C614FEA860C6745DDD32022EE
:10C9000000213348013E41F051F9A38AC4F8D862AE
:10C91000013BA38205B0BDE8F08F38460137FFF731
:10C92000EFFDD4F89C61B7EB860F4FEA860C9FD3DE
:10C93000D4F8B031002B95D1ADE7BEF1000FB9D0DE
:10C9400009FA05F54FF0010E21EA05010170D4F84E
:10C950009C614FEA860CADE7FB08D4F8A02107F0F4
:10C96000070612F803C002EBD70201934CFA06FE49
:10C970001EF0010FE4D0D4F8A411380151F800E002
:10C9800001EB0710BEF1000F0FD002AAB52109F08C
:10C9900033FBDDE9013018B103990AF0D1F8019BAE
:10C9A000D4F8A011CA1811F803C00BFA06F62CEA45
:10C9B000060C82F800C0D4F8983103EB080013F895
:10C9C0000810BDE74FEA860C65E700BF00040020B1
:10C9D000B806002038B5064C0025A38AC4F8B0512B
:10C9E0000133A382FFF730FFC4F8A45138BD00BF64
:10C9F000000400202DE9F04F484C0023D4E96912CF
:10CA00009C46521AE646654602606746664661469F
:10CA10006246C0E90133C0E90333C0E90533D4F805
:10CA2000983193F800B063464FEA42084BFA08F891
:10CA300008F00308B8F1010F64D0B8F1020F5DD01F
:10CA4000B8F1000F55D0D4F89C21013392009A42DE
:10CA50000CBF4FF001094FF000093ED04FEA930898
:10CA6000D4F8982112F808B003F003024FEA420A02
:10CA70004BFA0AFA1AF0030A14BFC84649F0010833
:10CA8000B8F1000F42D1BAF1010FCDD1C146D34662
:10CA900001292AD0022902D142690132426171453D
:10CAA00001D98E468161BBF1000F0DD0664501D9D9
:10CAB000B446C660B9F1000F05D02D013F01C0E9B1
:10CAC0000157BDE8F08F4E46D4F898214FEA9308FD
:10CAD00012F808B003F00302A6E7B8F1010F14BF83
:10CAE000CB4649F0010B0129D4D102690132026120
:10CAF000D5E70137013641468760A4E701350131AA
:10CB00004560A0E70135414645609CE7BAF1010F59
:10CB100014BFCB4649F0010BBAE700BF0004002068
:10CB2000034BD3F8A401003818BF0120704700BFA1
:10CB3000000400200F302DE9F04F050987B0059162
:10CB4000039257D0934A938A002B53D1D2F8A42151
:10CB5000002A00F01B81039B4FF0FF388D49002B0A
:10CB6000D1F8AC3114BF4FF0FF340124A3EB020322
:10CB700014BF4FF0030B4FF0000B082D4FEA1319B1
:10CB800091F8B43283F0010300932B4628BF0823A9
:10CB9000AD3304937F4B049A039953F822200292F9
:10CBA00069BBD3F8D8A294467A4B00220327D3F866
:10CBB00098310193D44514D8019B4FEA8C0E13F899
:10CBC0000C00009B002B40D10BEB0E065B4659007E
:10CBD00007FA01F101421AD04E452AD3012C28D17F
:10CBE0000022954249D9009B23B91AF0BDFC0123CC
:10CBF0000093CFE70023184607B0BDE8F08F654BE0
:10CC0000D3F8D8C2029B6345EDD8E246CCE70132A7
:10CC100095420BD901211B1928D439B3042B264482
:10CC2000D5D1A444029B6345C4D9DAE703EB0E08CF
:10CC3000D7E74E452CBF00210121621C4FF00002B6
:10CC400018BF002181F00101E5E75B4606E00132F3
:10CC50009542EBD91B1908D4042BE2D0590007FAEE
:10CC600001F10142F3D00022F4E70099A444029BB1
:10CC70006345B6D800299DD1B3E7039BABBB08F150
:10CC80000104072DA4EB02043AD805EB080305F1D3
:10CC9000AD0140484FEA930340F8213005F1AE0161
:10CCA00040F821302CD005F1AF01062D40F821309D
:10CCB00026D005F1B001052D40F8213020D005F136
:10CCC000B101042D40F821301AD005F1B201032D35
:10CCD00040F8213005F1050112D0B335062940F89E
:10CCE00025300DD1C0F8D4320AE008F1FF332949CC
:10CCF00044469B08C1F8D83202EB080303F1FF3821
:10CD000004F00303A108019D580001238340685CDF
:10CD100003436B54611C884510D3022601F00303C2
:10CD20001C4D88080131D5F898515B0088452F5C6F
:10CD300006FA03F343EA07032B54EFD2154B2601FF
:10CD40000399D3F8A45105EB041331B11148D0F87D
:10CD5000AC11994288BFC0F8AC31120118460021CD
:10CD600040F024FF059A0346D2077FF544AF002226
:10CD7000E10804F00704AA51064AD2F8A0010122F2
:10CD800002FA04F4425C2243425434E703201BF0CD
:10CD900023FC00BF00040020034B9A8A12B908B19B
:10CDA000FFF738BC704700BF00040020030701D123
:10CDB000FFF77CBC00207047F8B5144E0446D6F847
:10CDC000AC31834201D9030702D025462846F8BD7D
:10CDD000FFF76CFC07460028F7D02046FFF796FCCB
:10CDE000012201463846FFF7A5FE05460028ECD093
:10CDF000844206D9B38A002BE7D12546FFF70AFC07
:10CE0000E4E73A46214640F08DFEDFE700040020CB
:10CE10002DE9F84F88460546002800F0B580002926
:10CE200052D05E4CA38A002B52D1D4F8A41108F141
:10CE30000F0ED4F89C719C46411A4FEA1E1E4FEA11
:10CE4000870A0809461CB6EB870F80F0A480D4F847
:10CE500098910127B30806F0030B19F803304FEA45
:10CE60004B0B43FA0BF303F00303022B34D02BB923
:10CE70000CF1010C0CEB070373452ED3BE451FD0FC
:10CE80002FD3BC44F4455DD212B3D4F8A021C90914
:10CE900000F007034046515C0022194101F00101F6
:10CEA000FFF748FE064698B13A01294640F03AFE9F
:10CEB000A38A33B92846FFF7ADFB3046BDE8F88FAB
:10CEC0002E463046BDE8F88F344B9E8A002EF2D0B5
:10CED00000263046BDE8F88F01370136B245B9D19A
:10CEE000CCE700EB0E090322A7EB0E0E38444E46AA
:10CEF00006F003034FEA9608D4F8981101365B0058
:10CF000011F808C0864202FA03F32CEA030301F881
:10CF10000830EDD1BEF1080F4FEA990328BF4FF05A
:10CF2000080E0EF1AD0E54F82E20B2EB990FD4F886
:10CF3000D82288BF44F82E309A42C1D22E46C4F877
:10CF4000D832BEE7C2197044904211D94FF002089E
:10CF500002F003039608D4F8981101325B0011F82F
:10CF600006C0904208FA03F343EA0C038B55EFD155
:10CF7000AEEB07022E46002105EB0710120140F030
:10CF800015FE3046BDE8F88F024601464046BDE832
:10CF9000F84FFFF7CFBD012770E700BF0004002066
:10CFA00038B50307044614D1FFF780FB88B1154D4F
:10CFB000D5F8DC3233B90EE09A68D2B1DA68D2B172
:10CFC0001B6843B15A68002AF6D1043301201C6063
:10CFD00038BD002038BD012200211020FFF7AAFD36
:10CFE00003460028F5D0D5F8DC2232B100221060CB
:10CFF000FFDE0833EAE70C33E8E7C5F8DC0201207E
:10D000005C6038BD0004002010B50446C068FFF71E
:10D01000D3FE03462046E360BDE81040FFF7CCBED8
:10D02000034610B410B3040720D1194CD4F8A4213E
:10D03000E2B182421AD8D4F8A821824216D98207D6
:10D040000FD10268134CA24219D0134CA2421AD03D
:10D0500012498A420ED012498A420BD011498A42A3
:10D0600004D018465DF8044BFFF7A6BE18465DF8DD
:10D07000044B704718465DF8044BFFF7C5BF5DF8D9
:10D08000044B00F069B85DF8044B00F00DB800BF28
:10D0900000040020CCD00660CCD80660A0DF06607B
:10D0A0003CDD066074E3066010B5044682B009B941
:10D0B00002B010BD01394068C9B20191FFF7B0FF5D
:10D0C00003460199A0686360FFF7AAFF0346019930
:10D0D000A360E068FFF7A4FF03462046E36002B0C8
:10D0E000BDE81040FFF768BEF8B504460E4638B1FB
:10D0F00031B1184B984203D0037913F00A0501D0DF
:10D100002046F8BD43F00803C0682371FFF754FEC2
:10D11000A268E0609AB1711ECFB200E0E06850F8FA
:10D12000353000EBC50601353BB1042B394604D040
:10D130007068FFF775FF7060A2689542EED32046D5
:10D14000FFF73AFE037904466FF3C30303712046E9
:10D15000F8BD00BF940400200E2818BF00282DE958
:10D16000F84305460E4603D0B1FA81F4640911B9BB
:10D170002846BDE8F883013E8068FFF71DFE0346A0
:10D18000F6B26868AB603146FFF7AEFF686007E053
:10D1900031463846FFF744FFEB6843F80800013496
:10D1A000E8684FEA8408FFF701FEB4EB900F18D24D
:10D1B000EB6853F82400FFF7F9FD0028EFD0EB6887
:10D1C00053F824703B78022BE2D17868FFF7F4FD26
:10D1D0007860B868FFF7F0FDB860EB6853F8087046
:10D1E000D6E7E868FFF7E8FD03462846EB60FFF75F
:10D1F000DDFD8008B0F1040814D005F10C0700240F
:10D20000DFF8349057F8043F314618463BB19A078F
:10D2100002D11A684A450AD0FFF702FF386001348C
:10D220004445EFD12846BDE8F843FFF7C5BDFFF7F9
:10D230005BFF3860F3E700BF8CCB0660024BC3E9AD
:10D2400002011861704700BF0004002008B5084AB9
:10D25000C31DD2E9031023F0070303448B4201D816
:10D26000136108BD44F2F611024809F039FC00BF11
:10D270000004002024CF0660084BDB6A5A68824213
:10D2800003D91B685A688242FBD8801A1A6903EBDB
:10D29000800332F810200A8058697047000400208B
:10D2A000014488420ED241F2055310F8012B03EBE2
:10D2B0004313814283EA0203F7D1D8B2012838BF71
:10D2C0000120704705207047034B00220349C3F833
:10D2D0000821D962704700BF0004002070A80760D1
:10D2E0002DE9F84F88464118834688423CD20346D0
:10D2F00041F2055613F8012B06EB4616994286EAD1
:10D300000206F7D1F6B2012E38BF0126174BD3F82B
:10D310002CA0BAF1000F24D0DAE90374E7B101348C
:10D3200000250AF1140903E001350234AF4213D09D
:10D3300014F8013CB342F7D123784345F4D159F8AE
:10D3400025004246594640F059FC0028ECD1DAF855
:10D3500004002844BDE8F88FDAF800A0BAF1000F05
:10D36000DAD15046BDE8F88F0526CFE7000400204B
:10D370002DE9F84307460D46FFF7B2FF002846D1D6
:10D38000FF2D00F2AD805A4E6C1CD6F80881B8F122
:10D39000000F00F08280D6E94312A3188B425ED8BA
:10D3A00090447919C6F810318F4280F088803C464D
:10D3B00041F2055314F8012B03EB4313A14283EA16
:10D3C0000203F7D1DCB2012C38BF01243946002713
:10D3D0002A46404640F0A6FB08F80570F36AD3E9F8
:10D3E00002128A4215D21B6903F81240F36A1B69C4
:10D3F00003EB42035D70F36A03EB8203C3F814800E
:10D40000F16ACB680133CB60F36A58681044BDE819
:10D41000F8834FEA41090121B9F10A0F38BF4FF0F3
:10D420000A09B9F1400F28BF4FF0400909EB490044
:10D4300088401430FFF742F8034600284BD000F133
:10D44000140202EB89020261F16A01604A68C9684C
:10D450000A44C0E902974260F062C268C3E702462C
:10D4600021444046FFF748F8804668B1D6F80C31B1
:10D47000D6F808012344C6F80C3170B1D6F8103143
:10D4800000EB030823448CE70246D6F81011D6F8C7
:10D490000801FFF731F8C6F80881802CA1464FF04B
:10D4A000010138BF4FF080094846FFF707F8804672
:10D4B000C6F8080128B12346C6F80C9171E7052487
:10D4C00084E701212046FEF7F9FF8046C6F80801EF
:10D4D00050B1A146EFE74846C6F8083108F0B4FB62
:10D4E0000449054808F050FB204608F0ADFB00BF9A
:10D4F000000400202CF2066024CF066010B504461C
:10D5000040F08EFB01462046BDE81040FFF730BFDB
:10D5100000B583B001A9FFF7AFFE9DF8050003B089
:10D520005DF804FB00B583B001A9FFF7A5FE03B0C9
:10D530005DF804FB10B582B00C4601A9FFF79CFE14
:10D540009DF80530236002B010BD00BF38B5D0E9AA
:10D5500000320546114499420DD9037BDB070BD4F9
:10D5600001F11004806824F0070408342146FEF716
:10D57000B7FF2C60A86038BD0021014808F004FB0B
:10D5800024CF066070B504460E4611461546FFF7D7
:10D59000DDFF31462A46D4E90130184440F0F2FA62
:10D5A00062682A44626070BD70B50D4646680446E4
:10D5B0000121B54228BF3546FFF7C8FFA168681CA6
:10D5C000721B0844294440F0DDFAD4E901300133EC
:10D5D0002844636070BD00BF012938BF012138B500
:10D5E0000446002508462946C4E90005FEF75AFF0F
:10D5F000237BA06065F30003237338BD38B54B1C53
:10D600000C46054604D00131FFF7E6FF6C6038BDDB
:10D61000084608F019FB00BF037B826043F001035A
:10D6200010B400240373C0E900145DF8044B704784
:10D6300038B505461446FFF7CFFF024BC4E9005347
:10D6400038BD00BF85D5006010B5037B0446DB07FD
:10D6500002D50023A36010BD8068FEF74FFF0023B2
:10D66000A36010BD10B5044600211020FEF71AFF7C
:10D6700021460446FFF7B0FF204610BD10B5044612
:10D6800078B1037BDB0704D52046BDE81040FEF7E8
:10D6900035BF8068FEF732FF2046BDE81040FEF738
:10D6A0002DBF10BD38B5037B04460D46DB070AD4F9
:10D6B000016880682944FEF713FF2368A0601D44B9
:10D6C0001844256038BD0021014808F05DFA00BF0C
:10D6D00024CF066038B504460D46FFF737FFD4E97E
:10D6E00001301D441844656038BD00BF10B5D0E955
:10D6F000002304469A4204D0A2680021D154A068B5
:10D7000010BD0121FFF7CEFF6368A2680021D1544C
:10D71000A06810BD38B504460D460121FFF716FF7D
:10D72000D4E90132591C6160D55438BD7F29F8B560
:10D730000C4605462ED9B1F5006F19D3B1F5803FDF
:10D7400031D20321FFF702FFC4F38513210B04F04C
:10D750003F0463F07F0361F01F0164F07F04D5E9AB
:10D760000126B018D71C6F60B15443708470F8BDA7
:10D770000221FFF7EBFEA20904F03F04D5E90131D5
:10D7800062F03F0264F07F04C8189E1C6E60CA54A9
:10D790004470F8BD0121FFF7D9FED5E90132591CCB
:10D7A0006960D454F8BD0421FFF7D0FEC4F30531FD
:10D7B0004FEA944CC4F3851204F03F0461F07F01FA
:10D7C0006CF00F0C62F07F0264F07F04D5E9010673
:10D7D0003318071D6F6006F800C059709A70DC702E
:10D7E000F8BD00BF10B5044682B00846019140F074
:10D7F00017FA01990246204602B0BDE81040FFF733
:10D80000C1BE00BF10B51446FFF7CEFE047010BDB8
:10D8100010B51446FFF7C8FE047010BD43688B4274
:10D820002CBF5B1A00234360704700BF38B5154614
:10D83000426804460B468A4203D929448A4201D8E9
:10D84000436038BD8068521A0144184440F09AF988
:10D850006268521B626038BD0846114645F076BFCB
:10D8600070B5054608460E4640F0DAF9044620B188
:10D8700002466B68314628689847204670BD00BF55
:10D880002DE9F84F8A469DF8281091460B9A11F021
:10D89000DF0F0546A2EB09023DD030290AA9264E2A
:10D8A0000EBF10270E46012713F0800839D0002A3A
:10D8B0009046B8BF02F10108A2EB68044FEA68087D
:10D8C000B8F1000F32DDC3465F453A466B6831461A
:10D8D000A8BF5A462868ABEB020B9847BBF1000F74
:10D8E000F2DCB9F1000F05D04A465146C844D5E9EB
:10D8F00000039847002C0BDDA044A7423A466B6812
:10D900003146A8BF22462868A41A9847002CF4DCA8
:10D910004046BDE8F88F13F08008084E4FF010071E
:10D92000C5D113F0010404D01446DAE74FF0000823
:10D93000D7E79046C4E700BF18BD066004BD066087
:10D940002DE9F04F064689B000209C469DF85070A6
:10D95000139B159D8DF80F001AB3814249DB9A077E
:10D960005AD413F004021CD0202292468DF80F20C6
:10D97000D1B930220DF11F048DF81F2013F040089B
:10D980002DD0BAF1000F3AD1D04608AA3046214630
:10D990000195121B0097FFF773FF404409B0BDE8E3
:10D9A000F08F92460029E4D0129A08AC0DF11009CC
:10D9B000A2F10A0B8846B1FBFCFE0CFB1E1271465D
:10D9C000092A02F1300088BF0BEB0200E04504F8A1
:10D9D000010DD3D34C45EDD813F04008D1D1BAF1A5
:10D9E000000FD2D004AA9442CFD904F801AC013C74
:10D9F000CBE72D22494292468DF80F20D4E7012231
:10DA00000DF10F01304600970192013D1393FFF78E
:10DA100037FF139B8046B8E72B2292468DF80F20E4
:10DA2000A6E700BF2DE9F04F0F4691B080461C4697
:10DA3000F9071A9D9DF86CB00DD4BB0703D1A14B1B
:10DA40003968994207D03846059209F097FE059A41
:10DA5000400040F0010715F0810F03D1BBF1300FFA
:10DA600000F0CD80384605920DF068FB0028059A3D
:10DA700077DBAE0773D52B23E9060DF121060DF1F7
:10DA8000200A8DF8203071D4E3B2A6EB0A0115F01C
:10DA9000200F4FF000041D9805914FF010013470D5
:10DAA0000CAE0A910CBF21462C2101280B9409963B
:10DAB0006DDD009209A80BAA01948DF81F40CDE9F5
:10DAC00002313B460AA90DF009F9037807462D2BD0
:10DAD00072D18DF81F3001370B9B1D9A013B934289
:10DAE0000B93B8BF1346059A013313441C9A9A420C
:10DAF00070DC25F001054FF0000945F040054C466B
:10DB00004FF0300B9DF81F30002B40F0A180059B9B
:10DB1000002B40F0AE801D9B012B4ADD1D9B39463A
:10DB20000B9A4046CDE900B32B46FFF7A9FE04440B
:10DB3000B9F1000F0AD0002320224046624900922A
:10DB40001A46CDF80490FFF79BFE04440998B042B2
:10DB500001D0FEF7D3FC204611B0BDE8F08F680776
:10DB600056D40DF1200A5646E9068DD5022A3DD03D
:10DB7000082A00F08C80102AE3B286D1314630208A
:10DB800001F8020B03F1170070700E467DE715F0E7
:10DB900040098DF81F40CDE9023140F085803B46B9
:10DBA0000AA909A84C46CDE9002A0BAA0DF096F85F
:10DBB00007461C9B1D93B1E71D9A0B9B9342B8BF70
:10DBC00013469DF81F20002A8DD1059A13441C9AF4
:10DBD0009A428EDD15F0010922D025F001051C9A2C
:10DBE0000024A2EB030945F0400589E731463020C7
:10DBF000E3B201F8020B581C70700E4645E7DDE9F0
:10DC00001C318B42B8BF0B461C9300231D9329E7A0
:10DC100020230DF121060DEB030A8DF82030A3E738
:10DC20001C9A25F0010528494046D31A4A4645F07A
:10DC300040050193202300934B46FFF721FE044645
:10DC40005EE78DF81F3001370B9BA146013B0B931C
:10DC50001C9B01220DF11F014046013B1C93002338
:10DC6000CDE90032FFF70CFE059B0444002B3FF486
:10DC700052AF1C9B0120059A51469B1A1C9300230E
:10DC8000CDE900304046FFF7FBFD044443E7302375
:10DC90003370AB0501D40136F6E6E3B2023603F188
:10DCA0000E0106F8011CF0E63B4600920AA90BAAF9
:10DCB00009A801940DF012F8037807462D2BC0D067
:10DCC000A1461FE7F4D30660843008602DE9F043D5
:10DCD00014468BB00A460746A1079846129E1BD4ED
:10DCE00014F0040F0CBF0023202300932021139B6A
:10DCF00002A806F099FEE305054602D5431C1F2B3A
:10DD000018D914F0400909D09DF8083002A92F2B2A
:10DD10001CD94FF0000902E02B23E6E702A92346B5
:10DD20002A463846CDE90086FFF7AAFD48440BB0E5
:10DD3000BDE8F0830AAA1544252205F8202C0AAA7A
:10DD40001D461A44002302F8203CDAE70023012292
:10DD50003846013E013DCDE90032FFF791FD0DF15E
:10DD600009018146DBE700BF2DE9F04F8BB00023AE
:10DD70008346914604AFFB600B78252B14D0002B13
:10DD800000F0A9800C46254614F8013F0BB1252B65
:10DD9000F9D1A1420BD2621AFE681644DBE90003F6
:10DDA000FE6098476B782146002B00F094804B78FA
:10DDB0004C1C002B00F06D814FF0200A00260DE076
:10DDC0002B2B15D0202B16D0212B17D0302B18D170
:10DDD00046F040069A4614F8013F3BB12D2BEFD197
:10DDE00014F8013F46F00106002BF7D100251CE096
:10DDF00046F00206EFE746F00406ECE746F00806B8
:10DE0000E9E723780025A3F13002092A0AD805EBB7
:10DE1000850503EB450514F8013FA3F13002303DC1
:10DE2000092AF4D92E2B00F00D8194F800804FF0D0
:10DE3000FF33B8F16C0F48D0B8F1000F4BD0A8F108
:10DE40004502332A35D8DFE812F04B004B004B0077
:10DE50003400340034003400340034003400340022
:10DE60007B0034003400910034003400340034006E
:10DE700063003400340034003400340034003400D3
:10DE800034003400F400EA00E0004B004B004B008B
:10DE900034003400340034003400340034003400E2
:10DEA0007B00D0003400B90034006300340034003B
:10DEB0006300FB6801222146DBF800000133FB60B0
:10DEC000DBF804309847611C56E794F80180013470
:10DED000B8F1000FB3D1F8681C37BD46BDE8F08F2C
:10DEE00009F10709BB6029F00709F9E8020157F0B9
:10DEF000CBFFBB6800EE100A324641465846CDE9DA
:10DF000000535346FFF7E2FEFB680344FB60DAE789
:10DF100028F00F0208F1010359F8041B0F3A03F02F
:10DF20000603D2B2C3F11003CDE900260022CDE9E9
:10DF300002A55846FFF704FDFB680344FB60C2E7F7
:10DF4000DBE90003022255499847612359F8041B75
:10DF500000220093584610230196CDE902A5FFF751
:10DF6000EFFCFB6802300344FB60ACE759F8041B8C
:10DF7000E8463B600846B9601AF01CFEB9680246E4
:10DF80000846D11D531E21F00702BB60ADEB020D08
:10DF900004A979601AF012FE3B6879681A1E76DBD4
:10DFA000BB68934273D933465846CDE900A5FFF7C5
:10DFB00067FCFB680344FB60C54684E759F8041B13
:10DFC0007B600846B9603FF02BFE7B68B9681A1E7B
:10DFD00019DB824217D23346CDE900A55846FFF738
:10DFE0004FFCFB680344FB606DE707F1140159F82F
:10DFF000040BBB60FFF79EFABB68014678691A1EE6
:10E0000001DB9042E7D80246E5E7612059F8041B9E
:10E010000A230122CDE902A5CDE9000689E759F8D6
:10E02000040B3346012207F114013875CDE900A530
:10E03000D4E759F8043BCDE900A523B333460422C5
:10E040001749CBE794F80180B8F12A0F07D159F8A6
:10E05000043B023494F8008023EAE373E9E6A8F174
:10E0600030030134092B4FF000033FF6E2AE03EB1F
:10E07000830308EB430314F8018FA8F13002303B0F
:10E08000092AF4D9D5E6334605220649A6E7BA6837
:10E0900089E71E464FF0200A0025C6E6F8BC066058
:10E0A000E8BC0660F0BC06600EB400B582B003AAFE
:10E0B00052F8041B0192FFF757FE02B05DF804EB23
:10E0C00003B07047B0B582B0054608460C4600AFB5
:10E0D0007A601AF06FFD03462046073323F00703EA
:10E0E000ADEB030D69461AF069FD7A68694628466A
:10E0F000FFF73AFE0837BD46B0BD00BF0EB400B50D
:10E1000082B003AA52F8041B0192FFF7DBFF02B0B2
:10E110005DF804EB03B0704790F9001002460378F5
:10E1200000291ADA03F07F005B0605D5402320EAB8
:10E1300003005B081842FAD1517801F0C003802B2C
:10E140000CD1531C01F03F0C13F8011F01F0C00269
:10E150004CEA8010802AF5D070471846704700BFFF
:10E160004378013003F0C003802B05D110F8013F44
:10E1700003F0C003802BF9D0704700BF0246002097
:10E18000914209D911F8013D03F0C003802B18BF5B
:10E1900001308A42F6D17047704700BF014488427F
:10E1A0000CD2421E0139002012F8013F03F0C003D7
:10E1B000802B18BF01308A42F6D17047002070478B
:10E1C0007F2804D8034B185CC0F340007047002040
:10E1D000704700BF2CBD06607F2804D8034B185C35
:10E1E000C0F3C00070470020704700BF2CBD066020
:10E1F0007F2804D8034B185CC0F3800070470020D0
:10E20000704700BF2CBD06607F2804D8034B185C04
:10E21000C0F3801070470020704700BF2CBD06601F
:10E220007F2803460BD8074A125C12F00C0F14BF6C
:10E23000012000205F2B08BF40F001007047002044
:10E24000704700BF2CBD06607F2804D8034B185CC4
:10E25000C0F3001070470020704700BF2CBD06605F
:10E260007F2804D8034B185CC0F34010704700208F
:10E27000704700BF2CBD06607F2804D8024B1B5C92
:10E28000DB0648BF203070472CBD06607F2804D8CD
:10E29000024B1B5C9B0648BF203870472CBD0660B4
:10E2A0003038092802D920F020000738704700BF15
:10E2B000014488421FD200224FF0E50C08E003F031
:10E2C000C003802B29D10130531E8142DAB220D9FC
:10E2D0000378002AF3D1BF2B0FD81A061DD4421C95
:10E2E000914208D9104612F8013BBF2B05D81B06F6
:10E2F00013D49142F6D101207047F72B0DD8DB08DB
:10E30000013003F0060381424CFA03F303F00302E9
:10E31000DED8B2FA82F0400970470020704700BF93
:10E32000B2EB131F70B506464FEA131420D901EB68
:10E330004405141B03F00F0184462346AE46012B0F
:10E3400003F1FF3309D05EF8022B012B03F1FF33F9
:10E3500022FA01F22CF8022BF5D1601E35F81030AC
:10E3600023FA01F126F81010002918BF204670BDCD
:10E37000002070BD2DE9F041069FD21BAFB3A3F181
:10E38000020E8E1EBC460546002436F8023FBCF144
:10E39000010C3EF8028F434423444FEA134425F80E
:10E3A000023BF2D101EB470100EB470772B1A1F14B
:10E3B000020CBE4611463CF8023F013923444FEAA5
:10E3C00013442EF8023BF6D107EB420744B1012378
:10E3D00027F8023B3F1A47FA03F21046BDE8F081E6
:10E3E0003F1A7A101046BDE8F081002AF5D03C466D
:10E3F0000746DCE72DE9F041069FD21BEFB39C1ED8
:10E400008E1EBE4605464FF0000C36F8023FBEF1A8
:10E41000010E34F8028F6344A3EB08034FEA234C48
:10E4200025F8023BF1D101EB470100EB47050AB3A8
:10E43000A1F1020E2C4611463EF8023F0139634419
:10E440004FEA234C24F8023BF6D1531E05EB42025F
:10E4500005EB430303E01A4633F8021929B9984241
:10E46000F9D9101A4010BDE8F0810232101A40109C
:10E47000BDE8F081AB1E2A46F1E70546BC46D6E76B
:10E48000022938B538BF0221044680680D4618B10C
:10E490002368B1EB930F07D96900FEF721F82368D1
:10E4A000A06065F39F03236038BD00BF38B5054603
:10E4B00000210C20FDF7F6FF2B780446002103F025
:10E4C0000102037823F003031343037028682368D1
:10E4D000C0F39D0060F39F03400023606B6863609E
:10E4E000FDF7E0FFA0602A68A968C2F39D02520010
:10E4F0003FF018FB204638BD00EB410302EB410220
:10E5000019B910E00CD101390CD033F8020D32F8F2
:10E5100002CDA0EB0C000028F4DA4FF0FF3070477A
:10E520000120704770470846704700BF10B5044689
:10E530008068FDF7E3FF2046BDE81040FDF7DEBF31
:10E5400038B50C4602210546FFF79AFF002C10DB78
:10E55000214600202A78002360F300022A7000E0A0
:10E560006B68581CAA68686022F81310090CF7D170
:10E5700038BD61420120EDE70023C0E9003383602C
:10E58000704700BF0022C0E90022826001B97047D5
:10E59000FFF7D6BF9200816042F0020202600022C3
:10E5A000426003B970471946FFF7CABF10B103783C
:10E5B0009B0700D570478068FDF7A0BF38B50446BB
:10E5C0000D464968FFF75CFF2A782378A06862F35C
:10E5D000000323706A6862605200A968BDE8384091
:10E5E0003FF0A0BAF8B51D46042106469DF8187004
:10E5F0001446FFF745FF002D317816DAAFB16242BD
:10E6000041F0010165EB45033170002100E07168C4
:10E610004D1CB468100C756024F8112040EA0342C8
:10E620001B0C52EA0301F2D1F8BD6FF30001002088
:10E6300022462B46317054EA05017060E5D1F8BDE1
:10E640002DE9F04182B0027805468DED010A019C6A
:10E65000E30F63F30002C4F30F4313F4FF430270AC
:10E660002BD0B3F5FF4F28D0C4F3C752A2F17F03DC
:10E67000002B22DB4BD0B2F16F01C4F3160448BF6C
:10E68000A2F16001162B44F400044FEA21171DDCAF
:10E69000C3F117033946DC40FFF7F2FE00236F6039
:10E6A0009F4210D05B007900AA68D4520233240C38
:10E6B0009942F9D102B0BDE8F0812B7800226FF3C6
:10E6C00000036A602B7002B0BDE8F081093339465F
:10E6D00003F00F08B2F1960348BFA2F187031E11A1
:10E6E000FFF7CEFE6F6026B172000021A8683FF0F0
:10E6F0005DFAB8F1000F10D004FA08F2AB68C8F167
:10E70000100823F81620731C24FA08F4C8E7012126
:10E7100002B0BDE8F041FFF713BF3346C0E700BFCA
:10E720002DE9F8438846C2F35B0105461C460131DA
:10E7300008EB0206089FFFF7A3FE2B780020B045E8
:10E7400064F3000368602B702ED2C646B9B27246DD
:10E750000EF1010E1378A3F13000092805D9A3F1B9
:10E760004100192822D8A3F13700B84226D2D5E9B2
:10E7700001493CB3A4464A461388BCF1010C01FB95
:10E7800003034FEA134022F8023BF5D109EB44049E
:10E7900008B124F8020BA4EB090476454FEA64049F
:10E7A0006C60D4D1A6EB0800BDE8F883A3F161004A
:10E7B000192803D8A3F15700B842D8D3A2EB080018
:10E7C000BDE8F8834C46E3E72DE9F04107461446DF
:10E7D0001D4600294DD0531E4FF0FF361D44E10069
:10E7E00038460F310909FFF74BFE3B7800206FF3E5
:10E7F000000378603B70002C3DD0014680460F2915
:10E800001CDC4FF0000C95F800E0013C0B46354451
:10E810000EFA01FE01F108014EEA0C0C1FFA8CFC05
:10E8200001D00F29EFDD421CA3F10801BB687A601B
:10E8300023F810C04CB10F297868E2DDBB68421C98
:10E8400010397A6023F81080F5E77B685B00023BA3
:10E85000B868C31802D311E0984205D81A4633F8B5
:10E8600002190029F8D00232131A5B107B60BDE850
:10E87000F0810126B3E76FF00103E9E79A1CF3E7A3
:10E8800010B5047884460B7804F0010003F001030E
:10E89000181A0ED1DCF804304A6893420AD30CD817
:10E8A0008A681946DCF80800FFF726FEE30748BF30
:10E8B000404210BD4FF0FF30F8E70120F6E700BFFF
:10E8C000884210B5044601D0FFF778FE23786FF335
:10E8D0000003237010BD00BF884210B5044601D06C
:10E8E000FFF76CFE63683BB12378C3F30002C2F10B
:10E8F000010262F30003237010BD00BF884210B50F
:10E90000044684B001D0FFF759FE62684AB3237809
:10E91000D90715D4511C2046FFF7B2FDA16801208C
:10E920000DF10E036268ADF80E0000900846FFF787
:10E9300021FD2378606043F00103237004B010BD13
:10E9400018460123A1686FF300000093ADF80E3064
:10E950000DF10E0320700846FFF74CFD606004B017
:10E9600010BD01212046FFF78BFD0122A3681A800C
:10E97000237862601343237004B010BD2DE9F04783
:10E980000E4607464968144602B129B93146384651
:10E99000BDE8F047FFF712BE02F10F096FF0004823
:10E9A00001EB1911FFF76CFDBA684FEA191914F061
:10E9B0000F04D6E901C018BFC4F1100409EB0C051F
:10E9C000A84402EB48024FEA4808BCF1000F36D0D9
:10E9D00000EB4C0061469646002330F802AD013949
:10E9E0004AEA030323FA04FA4FEA03432EF802A982
:10E9F000F3D1E340CCEBCC7C9BB202EB4C02138016
:10EA0000C9F10103002102EB430309F1FF3218466B
:10EA100052003FF0CBF803464DB108F102084344E1
:10EA200001E0013D03D033F8022D002AF9D03B78F4
:10EA30007D60327862F300033B70BDE8F087634687
:10EA4000DDE700BF2DE9F0410C4684B00646496879
:10EA500017461AB1B1FA81F56D0931B92146304630
:10EA600004B0BDE8F041FFF7A9BDFFF709FD3B4643
:10EA7000B068D4E90121FFF753FC33787060227845
:10EA800062F300033370DB0717D55FEA171E626875
:10EA9000ADF80E500FD072B1D4F808809645F44608
:10EAA000294628BF9446A8F1020333F8025F0131DA
:10EAB000CDB96145F9D3964502D304B0BDE8F081E4
:10EAC000A36807F00F0733F81E100123BB40013B7A
:10EAD0001942F2D00123ADF80E3098B90123B26883
:10EAE00013807360E9E701239645ADF80E30F4D248
:10EAF00007F00F0738F81E2003FA07F7013F3A42E4
:10EB0000EBD0E7E7B168012402460DF10E03084699
:10EB10000094FFF72FFC7060CFE700BF2DE9F041B4
:10EB20004F6882B0D2F804800C4615460646474529
:10EB300028D306D892683946A068FFF7DDFC002884
:10EB400020DB23782A785340DB0720D4791C304619
:10EB5000FFF796FC6868AB686268A1680090B068CF
:10EB6000FFF708FC706023783278C3F300030028B5
:10EB70000CBF002303F0010363F30002327002B004
:10EB8000BDE8F081234647462C461D46D9E7394665
:10EB90003046FFF775FC6868AB686268A168009052
:10EBA000B068FFF727FC7060DDE700BF2DE9F0419A
:10EBB000D1F8048082B057680C4615460646B84521
:10EBC00009D306D892684146A068FFF795FC002853
:10EBD00001DB002704E02346B8462C4601271D46EA
:10EBE00023782A785340DB0715D508F10101304618
:10EBF000FFF746FCD5E90103D4E901210090B06894
:10EC0000FFF7B8FB7060A8B9337860F30003337086
:10EC100002B0BDE8F08141463046FFF731FCD5E94E
:10EC20000103D4E901210090B068FFF7E3FB7060B5
:10EC30000028E9D05FB123783278C3F30003C3F131
:10EC4000010363F30002327002B0BDE8F081227864
:10EC5000337862F30003337002B0BDE8F08100BF87
:10EC60002DE9F04F87B00B460391114602920490B4
:10EC700018465A684B689A4202D31346CDE90201FE
:10EC8000029A1278D20700F18B80039A117801F072
:10EC90000101049C19442046FFF7F2FB029B039AF2
:10ECA00093F800C011789D6858685368D2F808A09E
:10ECB0001A468CEA0103D4F80890DB075FD50CF004
:10ECC000010C01F00101CCF1000BC1F100081FFAA9
:10ECD0008BFB1FFA88F800284DD0002601964F467E
:10ECE000CDF81490023D0446914635F8023F013CB0
:10ECF000D646424683EA0B03634409EB040CACEBB3
:10ED0000000C644504D33EF8022B82EA0802F24666
:10ED100011444FEA134C019A0B40090C534016FA68
:10ED200083F31E0C27F8023B002CDED1DDF8149093
:10ED300009EB400006B30346012223F8022B03E04F
:10ED4000034630F802296ABB8145F9D9A3EB0903D0
:10ED50000498039A5B1001784360029B12781B7839
:10ED6000C2F30002C3F30003134063F30001017018
:10ED700007B0BDE8F08F484603460238E4E71CF0D0
:10ED8000010C01F001019ED0C1F100081FFA88F8C2
:10ED900050B14FF6FF7B0126CDF804B0B4469EE794
:10EDA000012176E70233D1E74846C4E72DE9F04F69
:10EDB00087B00B46039111460292049018465A6898
:10EDC0004B689A4202D31346CDE90201029A1278A7
:10EDD000D2077FD4039A117801F00101049C1944F1
:10EDE0002046FFF74DFB029BD4F8089093F800C033
:10EDF0009D685C681CF0010F039B0CF0010CD3E9CB
:10EE0000012A01925ED1197841F3000301F0010655
:10EE10009BB23146CCF1000BC1F100081FFA8BFB0D
:10EE20001FFA88F8002C59D0023D4F46CDF81490B7
:10EE3000204699460095009A0138019DD64632F841
:10EE4000023F83EA0B0300924246634405EB000C49
:10EE5000ACEB040C604504D33EF8022B82EA0802B6
:10EE6000F24611444FEA134C0B43090C83EA0903A1
:10EE700016FA83F31E0C27F8023B0028DBD1DDF8DD
:10EE80001490631E09EB440409EB430303E01C46A2
:10EE900033F8022902BB9945F9D9A4EB0904049877
:10EEA000029B6410039A017844601B781278C3F3C4
:10EEB0000003C2F30002134363F30001017007B0C3
:10EEC000BDE8F08F039B012619784FF6FF7301F020
:10EED00001019FE7012181E70234DEE7A9F1020386
:10EEE0004C46D8E72DE9F04F85B00B46019111460D
:10EEF0000092029018465A684B689A4202D3134611
:10EF0000CDE90001009A1278D2076AD4019A1178EB
:10EF100001F00101029C19442046FFF7B1FA009B61
:10EF2000019A1D781178EE43D4F808904D405C6842
:10EF3000C9439F6806F0010605F0010501F00101D3
:10EF4000D2F808A05368002C4FD0C846CDF80C90DA
:10EF5000023F20464FF6FF7B9946013837F8023FC3
:10EF6000D6464FF6FF7209EB000C5B44ACEB040C89
:10EF70003344604503D33EF8022B5A44F246114411
:10EF80001E0C4B40090C15FA83F31D0C28F8023BAC
:10EF90000028E2D1DDF80C9009EB4404E5B9A31E8A
:10EFA00003E01C4633F80229EAB99945F9D9A4EBE4
:10EFB00009040298009B6410019A017844601B7850
:10EFC0001278C3F30003C2F30002534063F300015D
:10EFD000017005B0BDE8F08F0122234624F8022B12
:10EFE000E3E7012196E70234E1E74C46D6E700BFAC
:10EFF0002DE9F04F87B04B680F4606460192002B73
:10F0000066D05168002963D087426FD0019A82424E
:10F0100077D00022029219443046FFF731FA336864
:10F020000021B068C3F39D035A003EF0BFFD019A72
:10F03000B368D2F80490D2F808800393D7E901B1FD
:10F04000B9F1000F32D003EB4B00CA46C1468846E7
:10F05000CDE904675F469B46002F44D0ABF1020424
:10F0600039464546002335F8026B0139B9F800C02E
:10F0700034F8022F0CFB0622134423804FEA13437B
:10F08000F1D104466BB3851C03802C4657F0ECF994
:10F09000BAF1010A0BF1020B09F102092846DBD192
:10F0A000039BE41ADDE904674FEA6409019AC6F894
:10F0B000049011783B7832784B4063F30002029B56
:10F0C00032705BB1184607B0BDE8F04FFFF72EBABB
:10F0D000337800226FF300037260337007B0BDE82D
:10F0E000F08F851CD2E7851C5C46CFE7FFF7DEF981
:10F0F000019B0746B34243680AD0019A02905168C7
:10F1000089E7FFF7D3F97B6841680190029082E7B5
:10F110001946CDE901007EE770B54B6806461446F6
:10F1200073B31378DA072BD46368002B38D0084602
:10F13000FFF7BCF905462046FFF7B8F90446012160
:10F140003046FFF7FDF9626872B920E001230846F6
:10F15000FFF7E6F803462A46294628466360B3B11E
:10F16000FFF746FF626892B1A1680B88DB07EDD517
:10F170002A4631463046FFF73BFFD4E90121E5E757
:10F18000337800226FF300037260337070BD15B1E5
:10F190002846FFF7CBF92046BDE87040FFF7C6B917
:10F1A0000121BDE87040FFF7CBB900BF2DE9F04F5A
:10F1B0000D4651688DB01646013104461F46069231
:10F1C00004930390FFF75CF973680021A068013392
:10F1D0005A003EF0EBFC237828466FF300032370BF
:10F1E0000023636071680131FFF74AF93146284610
:10F1F000FFF7E4F97B68D5F804800193434500F2FA
:10F200002281A368AE68BF6805930AD33A46414697
:10F210003046FFF771F9002800F01A81013000F044
:10F220001281019B6FF0004E00219E4437F91E3081
:10F230004FEA4E0437F81E20002B05DB5300013146
:10F24000180489B29AB2F9D5002326F818306A68F2
:10F25000013206EB42006A60864211D2C1F1100809
:10F260003046028802FA01FC22FA08F24CEA030353
:10F2700020F8023B93B26A6806EB420C6045F0D37B
:10F2800037F81E308B400293019B012B08D93B19A4
:10F29000C1F1100033F8023CC340029818430290B9
:10F2A000019B6FF0004C0398D31A6244436063449F
:10F2B000059806EB420C019A00EB43006B689A42FA
:10F2C0005AD2ACEB040483460CF1020C0796A4F16D
:10F2D000020A3CF8028D029B3CF802ECE2454EEA41
:10F2E000084EBEFBF3FE4FF000031CD2A7F102094B
:10F2F0005446984639F8022F20888A4010FA83F045
:10F3000042EA18481FFA88F20EFB02F296B2120C7B
:10F31000801BC2EB234224F8020B644502EB20431E
:10F32000E8D3BCF8008018EB03081AD0E2454FF090
:10F33000000311D2BE1E50461C4636F8022F8A40EA
:10F3400042EA1444028812FA84F2134420F8023B81
:10F3500060454FEA1343F0D318EB03080EF1FF3E6C
:10F36000E4D12BF802E9AAF1020A6B68019A013B89
:10F370009A426B60ADD3079E6FF000421A4406EBD1
:10F38000420296420CD8C1F110070024138843FAB8
:10F3900001F0BB4020439CB222F802099642F5D905
:10F3A0000398436853B1059A02EB430201E04360BE
:10F3B00023B132F8021D013B0029F8D06B6853B12C
:10F3C00006EB430601E06B602BB136F8022D013BE2
:10F3D000002AF8D06B682A78C2F30001002B0CBF1A
:10F3E000002101F001011346049A61F300032B7020
:10F3F000069B12781B785340DB070BD5039A5368A2
:10F4000011461278003B18BF012363F300020A7013
:10F410006B6813B90DB0BDE8F08F002309A84FF059
:10F42000FF310B93CDE90933FFF78AF8039909AA55
:10F430000846FFF773FB049A29462846FFF76EFB40
:10F440000DB0BDE8F08F0023039A53606B68C2E7EC
:10F450000123059A68601380039A53606B68BAE7CA
:10F460002DE9F04398464B6885B00C460646154694
:10F47000002B49D01378DA0746D4D8F80430012B92
:10F4800004D1D8F808301B88012B3DD0012130462B
:10F49000FFF756F86B68002B3CD020460DF10409AD
:10F4A000FFF704F804462846FFF700F80023074654
:10F4B0000193CDE902334268A2B92EE00846012348
:10F4C000FEF72EFF05462246214620467D6025B3E5
:10F4D000FFF78EFD2246434621464846FFF766FE6B
:10F4E0007A68D2B1B9680B88DB07E7D52246314686
:10F4F0003046FFF77DFD3246314643464846FFF72A
:10F5000055FED7E90121D9E7337800226FF30003D4
:10F510007260337005B0BDE8F0834846FFF746F8E7
:10F5200014B12046FFF702F83846FEF7FFFF05B09A
:10F53000BDE8F083D0E901318446002001EB4303AC
:10F54000994205D233F8022D994242EA0040F9D39C
:10F550009CF80030DB0748BF4042704710B4D0E948
:10F560000134002204EB43039C4203D308E0B2F5CC
:10F57000004F0ED233F802CD9C424CEA0242F6D341
:10F58000037801205DF8044BDB0748BF52420A6054
:10F59000704700205DF8044B704700BF2DE9F04F25
:10F5A00083B00192002948D09D18D0E901ABBAF18F
:10F5B000000F2CD00022019E012403EB0609944683
:10F5C0003BF8026B0CF1100C46EA024290F800E0A6
:10F5D00096B22F4605F1FF381EF0010F6FEA060EB6
:10F5E00005D054FA8EFE1FFA8EF6CEF30724E1B151
:10F5F000434505F8016C45461CD0ACF1080C120AD5
:10F60000BCF1070FE2DCBAF1010AD9D1D9B1EA1A8B
:10F610001D460378284613F0010F14BFFF21002177
:10F6200003B0BDE8F04F3EF0C1BA07F8016B4F459B
:10F630003D46E2D103B0BDE8F08FD0E901AB1D46F5
:10F64000BAF1000FB6D1019A13445A1BE1E700BF8B
:10F65000D0E901329FED0C0A02EB43039A420DD22E
:10F660009FED0A7A33F8021D07EE901A9A42F8EEDF
:10F67000E77AE0EE077AB0EE670AF3D30378DB07A8
:10F6800048BFB1EE400A704700000000000080470C
:10F690002DE9F84F1646426880460C469A469DF87A
:10F6A0002890AAB9002E00F09E8033780B992BB1D8
:10F6B00001F8013B16F8013F002BF9D10846302232
:10F6C00000230A7000F8013F0B9BC01ABDE8F88FB9
:10F6D0004FEA420B00215846FCF7E4FE05465A4625
:10F6E000D8F808103EF01EFA05EB0B01DDF82CC02F
:10F6F000AAF13A0E881E6246A84225D3824600230C
:10F70000BAF800B04BEA0343B3FBF4FB2AF802B9A2
:10F71000554504FB1B33F3D930339246392B88BF50
:10F720007344A942DBB20AF8013B13D92B4601E02E
:10F7300099420FD933F8027B002FF9D0B9F1000FAD
:10F7400041D15246A842D9D230239246A9420AF862
:10F75000013BEBD8B9F1000F08D0AAEB0C0CBCF1BF
:10F76000030F03D102F1020A82F801902846FCF748
:10F77000C5FE76B130463EF053FA33189E4208D2A9
:10F780000AF1FF3213F8011D9E4202F8011FF9D160
:10F79000824498F80030DB0720D40AF1FF330B9A3B
:10F7A0009A4208D20B9A1178187802F8010B03F8E4
:10F7B00001199A42F7D300230B9A8AF80030AAEB7A
:10F7C0000200BDE8F88FAAEB0C03032BB9D102F1BC
:10F7D000020A82F80190D4465246B3E72D225346DE
:10F7E0000AF8012BDBE70B9968E700BFD0E902328A
:10F7F000934203D25A1C8260187870474FF0FF3052
:10F80000704700BF10B50368044623B92046BDE821
:10F810001040FCF773BE4068FCF770FE2046BDE860
:10F820001040FCF76BBE00BFF8B50E461546044607
:10F83000002110201F463544FCF734FE044A054BD6
:10F840000760C560C0E90166C4E90002A360F8BDB5
:10F85000EDF7006005F8006010B40369272B18BFAE
:10F86000222B0CBF0122002203D110465DF8044B6D
:10F870007047A3F162011329F7D8124C24FA01F161
:10F88000C907F2D54169272918BF22290CBF0122D7
:10F890000022EAD0722B10D0662B01D0622BE4D16B
:10F8A0007229E2D182695DF8044B272A18BF222A07
:10F8B0000CBF01220022104670476629F2D062294F
:10F8C000D3D1EFE71100090038B5036904460A2BCC
:10F8D0003CD0092BC36A04BF073323F0070301336D
:10F8E000C362216FD4E90523C4E9042381B1606EAA
:10F8F00081421ED24D1CA06E2567415CA161E2B120
:10F900000D2BA0690BD10A239842636124D038BD26
:10F91000D4E9010398476369A0610D2BF3D001304E
:10F92000F5D163690A2BF2D00133F0D00A23A36129
:10F9300038BD0021A161002AE2D1606A6266A0613F
:10F940002267D4E90713C4E90413E6E7836A0122B6
:10F950001344C0E90A32C4E7D4E901039847A0611F
:10F96000DDE700BF70B504460D4600690026431C64
:10F970000BD00A280BD10DB1636B33B120460126A1
:10F98000FFF7A2FF2069431CF3D1304670BDFEF79C
:10F9900017FC50B92369232B0CD05C2BF5D163697C
:10F9A0000A2BF2D12046FFF78FFF2046FFF78CFF8E
:10F9B0002069DCE72046FFF787FF20690A28D6D0B8
:10F9C0000130F7D1304670BD2DE9F04F436E87B05E
:10F9D00004461BB1036F002B00F027810021204655
:10F9E0006165FFF7BFFF226BD4E90A35002A049254
:10F9F000C4E911351346C0F2108108D0049B0722D8
:10FA0000013B84F84C20236307B0BDE8F08F08B3B6
:10FA1000636BFBB9E26B6FF00043206C062113446B
:10FA2000013D84F84C1030F8131000EB43038D4275
:10FA3000EAD000F2DB8309D2511E881AE163013952
:10FA4000206333F8020D8542F7D3DDD0022384F81A
:10FA50004C30D9E7D4F810B0BBF1FF3F00F0F9808B
:10FA60002046FFF7F9FE0390002800F06F82002384
:10FA7000BBF1750F04F1600584F84C3000F0B380E1
:10FA8000BBF1620F00F0FE81BBF1720F00F0048247
:10FA9000BBF1660F00F01A824FF00009049E0C23A0
:10FAA000CDF8089094F84C20002A40F0A78084F804
:10FAB0004C30002E40F0A880BBF1220F204618BF2A
:10FAC0004FF0270BFFF700FFD4F810A0DA4500F045
:10FAD000C6814FF00108B9F1000F40F0BB81D4F8A6
:10FAE00010A0BAF1FF3F534600F0FB81B8F10102CC
:10FAF0004FF0000704F1500618BF012201920A2BB3
:10FB000002D1019A002A54D0B84557D95B4500F07C
:10FB1000BA80B9F1000F3AD057467B2F36D1204634
:10FB2000FFF7D2FE21697B2900F09C804A1C676E9A
:10FB300000F08C814FF0000ABAF1000F03D17D294B
:10FB400012D03A2910D021F020035B2B40F08580A1
:10FB50000AF1010AC9B22846FDF7DCFD2046FFF78D
:10FB6000B3FE21694B1CE7D1626EA16E8B1813F8AE
:10FB7000013C3D2B7ED02C212846FDF7CBFD7B217F
:10FB80003046FDF7C7FD27697B2FC8D0BA46BAF1CA
:10FB90005C0F7ED05FFA8AF130460027FDF7BAFD90
:10FBA0002046FFF791FED4F810A0BAF1FF3F53466C
:10FBB000A5D1B84502D9032384F84C30394604F165
:10FBC0005000FDF72BFE01212046FFF7CBFE20461B
:10FBD000FFF742FE00283FF417AFD4F810B0BBF196
:10FBE000750F7FF44DAF4FF0000994F84C200126BB
:10FBF0000C23CDF80890002A3FF459AF9A427FF4C5
:10FC000003AF002E3FF458AF2046FFF75DFE022EF3
:10FC100000F09381D4F810B04EE70822013384F845
:10FC20004C20236307B0BDE8F08F29216030FDF739
:10FC300071FDA36EA269D4E9040162620322C4E9E2
:10FC4000070119782161597861619B782267A36166
:10FC5000C4E6002384F84C30D6E65D2B08BF0AF1D9
:10FC6000FF3A77E730463946FDF754FD2046FFF767
:10FC70002BFE84E7D21B39443046FDF783FC636ECC
:10FC8000013B636677E7594630460137FDF74EFD85
:10FC900086E72046FFF718FE029A2369002A79D1E9
:10FCA000A3F10A026E2A70D8DFE812F085006F0017
:10FCB0006F006F006F006F006F006F006F006F00CC
:10FCC0006F006F006F006F006F006F006F006F00BC
:10FCD0006F006F006F006F006F006F003E016F00DC
:10FCE0006F006F006F003E016F006F006F006F00CC
:10FCF0006F006F006F006F006F006F006F006F008C
:10FD00006F006F006F006F006F006F006F006F007B
:10FD10006F006F006F006F006F006F006F006F006B
:10FD20006F006F006F006F006F006F006F006F005B
:10FD30006F006F004D016F006F006F006F006F006C
:10FD40006F0087006F006F006F006F006F006F0023
:10FD50003E016F006F006F006F004B01CC006F0021
:10FD60006F006F00AE006F006F006F006F006F00DC
:10FD70006F006F00C8006F006F006F00C6006F005B
:10FD8000CA008700BB006F00CE00A3F13007072F29
:10FD900040F2A9805C2130460593FDF7C7FC059B26
:10FDA0005F1C08D0B3F5881FC0F0BE800123002778
:10FDB00084F84C30F4E60027F2E694F84C200D2A43
:10FDC00000F0AC80752B0CBF032707270023CDF86C
:10FDD00014B0C346A0469A4607E020464FEA0A1AE6
:10FDE000FEF75EFA013F824463D34046FFF76CFDA5
:10FDF000D8F810402046FEF707FA0028EDD1444617
:10FE0000D846DDF814B0D1E70C2394F84C200C2A26
:10FE10000CD00D2ACAD1D9B230460027FDF77AFCA2
:10FE2000BEE694F84C200B230C2AF2D1194630463A
:10FE30000027FDF77BFCB3E60D23E6E70A23E4E7A2
:10FE40000923E2E70823E0E70127BFE73A468CE60B
:10FE50004FF00108AE492846FDF7C4FC3FE6636950
:10FE60005B4506D0B9F1000FF2D15B464FF00108B7
:10FE70003CE620464FF00308FFF726FD2046FFF73B
:10FE800023FD28E66369722B19D04FF00009012683
:10FE90000D23CDF8089005E66369622B0FD0662B21
:10FEA00000F02B81039B01264FF0000902930C23E5
:10FEB000F8E544465346D846DDF814B070E7039B96
:10FEC00002264FF0000902930D23EBE56369722BC4
:10FED00000F013810022DDF80C9001260C23029221
:10FEE000E0E5002767E66369303B072B00F2FE8000
:10FEF0002046FFF7E9FC62692369303A303B072A64
:10FF000003EBC7033FF64CAF20460593FFF7DCFC3D
:10FF10002269059B303A02EBC30341E75C2130467E
:10FF20000593FDF703FC059B94F84C200C2A3FF445
:10FF30007DAFFF2B7FF66DAF38E72046FFF7C4FC9F
:10FF400068E6072361E7734806F0AAFD5846FEF706
:10FF500043F9002850D12069A0F15F05B5FA85F575
:10FF60006D097F2888BF45F00105002D46D004F1BA
:10FF700050050923C1B2284684F84C30FDF7CAFB6E
:10FF80002046FFF7A1FC2069431C0AD0FEF724F9A4
:10FF900070BB20697F282CD85F282AD0FEF728F96B
:10FFA00030BB28465C4FFDF7A1FB00255B490646A8
:10FFB00007E0FFF629AD0135242D3FF425AD57F8B4
:10FFC000041F30463DF03AFE0028F2D105F10F0340
:10FFD000DBB2122B84F84C307FF416AD504BD3F8C3
:10FFE0001431002B0CBF11230F2384F84C300BE588
:10FFF0002069C1B22846C1E72069B8E7FEF7F8F8E2
:02000004600199
:1000000000285FD021692E2958D00A23302984F88E
:100010004C3047D004F150063046FDF787FB2046B0
:10002000FFF752FC2169481C3FF4EEAC0B27A5B941
:1000300021F02003452B10D16521304684F84C7007
:10004000FDF774FB2046FFF73FFC21692D2911D0F5
:100050002B290FD04A1CEAD1D6E40846FEF7BCF89B
:1000600080B1216921F020034A2B01D02E2901D132
:1000700084F84C703046FDF759FB2046FFF724FC0E
:100080002169E7E72069FEF7B3F80028E9D1216983
:100090002E29EDD05F297FF4B7AC2046FFF714FC82
:1000A0002169D7E7636943F02003623B162BB1D87F
:1000B0001C4D25FA03F303F00105ABE70B2384F88D
:1000C0004C30A7E723692E2B5FD00027164D28263A
:1000D00006E0632E08D06E7801376A1C8EB1154693
:1000E0009E4223D0652EF4D10135F4E794F84C20DC
:1000F0003B460C2A7FF48DAE98E6052384F84C30FD
:1001000082E42046FFF7E0FB012384F84C307BE4D7
:10011000FCBD0660E00A076008BF0660ACBD066073
:100120000004002001204000B4BD06602046FFF717
:10013000CBFB212E3CD02E2E33D06E780135632E92
:1001400001D0652E0ED1B8466B7808F101082269FE
:100150009A4237D0632E05D015F8026F632EF3D084
:10016000652EF1D02C4BDB5D592B03F0FD0284F89A
:100170004C3012D0552A10D0562B02D0582A7FF47A
:1001800043AC636B013B63633EE46069FEF730F8A8
:1001900000287FF437AF236997E7636B013363630C
:1001A00032E423692E2B14D05D2384F84C302BE4E9
:1001B00023693D2BA8D12046FFF786FB3A2384F81C
:1001C0004C3021E420464746FFF77EFB652EC3D125
:1001D000C8E763692E2BE7D12046FFF775FB204661
:1001E000FFF772FB0E2384F84C300DE4A36B9A42A8
:1001F00007D2531CE36320F81250236B01332363AF
:1002000002E408335900FCF76BF92064D4E90E329C
:100210000833A363EDE700BFDCBE066070B584B0B1
:100220000646742001AD85E80E000021FCF73AF97E
:100230000446034695E8070043F8046B002583E86D
:1002400007000A2201236FF001011420E3632563F4
:10025000C4E90D52C4E90A312946FCF723F90346E3
:10026000202104F150002364FDF7B6F9294604F17A
:100270006000FDF7B1F9236C20461D802561C4E9BB
:100280000555FFF721FB2046FFF71EFB2046FFF731
:100290001BFB2046FFF798FBA36C012B02D0072322
:1002A00084F84C30204604B070BD00BF30B585B036
:1002B000054601AC2046FFF7B7FA284694E80E0041
:1002C000FFF7ACFF05B030BD30B585B0054601ACD9
:1002D0002946204615F04CFF2846FDF70FF994E813
:1002E0000E00FFF79BFF05B030BD00BF10B5044600
:1002F00090B1E3684068984704F15000FDF7A4F915
:1003000004F16000FDF7A0F9206CFCF7F7F8204637
:10031000BDE81040FCF7F2B810BD00BFD0E90432D0
:10032000013B036152F82300704700BF38B50D460A
:100330000446D0E903138B4205D240695A1C22615E
:1003400040F8235038BD103140698900FCF7C8F8E7
:100350006061D4E903231032E2605A1C226140F844
:10036000235038BD2DE9F0418846044617461E4605
:10037000D0E900158D420ED280686B1C636050F886
:10038000353068F3170340F8353000EBC500C7700F
:100390004660BDE8F08110318068C900FCF7A0F824
:1003A000236865681033A0602360E6E710B48469B1
:1003B000CAB20023616C5DF8044BFFF7D3BF00BFE6
:1003C000F8B5446A06460D4634B363685A18216886
:1003D0008A4204D804F1080062601844F8BD05F1AF
:1003E0000803204600221944FCF786F848B104F1BE
:1003F0000800D4E900235119EA181844216062600A
:10040000F8BD6168024620460831FCF775F863685C
:100410002360336A63603462102D2F464FF0000171
:1004200038BF102707F10800FCF73CF8002304460A
:10043000C0E900737062436804F10800EA181844C8
:100440006260F8BDF0B5866983B005460F4696F840
:100450004C30092B25D00A2B55D00B2B64D0A3F19F
:100460000C02012A08D91901284641F00E0103B0F7
:10047000BDE8F040FFF75ABFD6E915100A2920D889
:10048000FCF776FF08B396F84C300C2B0CBF062215
:100490000A2242EA0011284603B0BDE8F040FFF707
:1004A00045BFD6E91510FCF763FF902F4FEA001403
:1004B00043D044F00201284603B0BDE8F040FFF706
:1004C00035BFFCF70DFF0028DDD196F84C00214A1E
:1004D000214B0C280CBF10461846D6E915210CF00C
:1004E0008BFF04460C212846766CFFF769FF4FF41A
:1004F0009D7301468460C0E90063284603B0BDE8EF
:10050000F040FFF713BF33460022D6E9151004F080
:10051000FDFDC3070446E5D544F00101284603B0BC
:10052000BDE8F040FFF702BFD6E915100023012215
:10053000009604F085FE0446D4E7002244F006014C
:1005400005F1280055F088FF0028B2D04468E20782
:10055000C8D5E1E7A0DF06603CDD0660FE2809D0D3
:1005600010F0010304D043080CBF012000207047A5
:100570001846704701207047B0F58F7F09D010F002
:10058000010304D0430814BF01200020704718461F
:1005900070470120704700BF10F0010308D130B14F
:1005A00010F0030217D103793A2B06D0104670479A
:1005B00040F0010301200B607047836813F00100D5
:1005C0000B60F4D19A07F2D11868044BC01AB0FA44
:1005D00080F0400970471846704700BFF4D30660AA
:1005E0002D2A2DE9F04F1746044688461E462DED6C
:1005F000028B87B045D0922A2DD0962A00F05C81DC
:10060000A2F11E03012B00F2E3800369002E00F02B
:100610003E8242699B1B701E52F8233016D01E2F5B
:10062000314600F0C880FE2B05D0DA0740F1B180DA
:100630005B0840F0B280013900F08781761A2369A7
:10064000012EA3EB0101216140F07F8107B0BDECD9
:10065000028BBDE8F08F03694269013B52F8232009
:10066000BAB1910715D11179952900F0E881962941
:100670000FD10361536823F0FF0343F092035360EB
:10068000E4E703694269013B52F82330002B40F054
:10069000B980A7F12603022B40F2BC80292F00F07D
:1006A000D381052F40F07181D4E90432013B52F827
:1006B00023509B00002D47D0A90745D1696801F060
:1006C000FE00562840D0134453F8049C09F00F0351
:1006D000022B39D1C9B22C2936D1AB6803F00F02F5
:1006E000022A31D11B09482B2ED1EA6862B312F0DD
:1006F000030308EE103A27D11379302B24D1D2F816
:1007000008A004A94FEA191B5046FFF745FF00282F
:1007100000F0D08129F00F01012204F1280041F0FE
:10072000060155F099FE049A014658464A60FCF7C6
:10073000F9FE02785F2A00F0B18123695146204614
:10074000013B2361FFF7F2FDB51C2046AD002946B1
:10075000FFF736FE014647EA0623C0F800804360F3
:100760007EB12A1F0A44013ED4E9043003F1FF336D
:10077000236150F8233042F80439F4D1962F00F069
:100780005481204607B0BDEC028BBDE8F04FFFF767
:10079000CDBDB3F58F7F00D00139D4E904522B1AB7
:1007A0006D1A013852F8233042F825303FF443AF38
:1007B0001E2F7FF438AFB3F58F7F3FF43CAFDD07DA
:1007C00003D55B087FF437AFE7E7FE2BE4D1E4E71E
:1007D000202A78D103694269013B52F82320FE2A7E
:1007E00067D0D50740F1AE80520814BFFE214FF408
:1007F0008F712046236107B0BDEC028BBDE8F04F3E
:10080000FFF794BD98077FF421AF1B79922B3FF43B
:1008100040AF1BE7236903A962699B1B52F82300C1
:10082000FFF7BAFE00288FD0B51E002D40F33281AD
:10083000A6F1030A0DF110092AF00103A6F1040A3A
:10084000AAEB030A0DE00028FFF67EAF023D5846F2
:10085000DDE9031255F020FE55450346039000F0F4
:1008600084802369494662695B1B52F82300FFF7C5
:1008700093FE00283FF468AF23696269013B5B1B6C
:1008800052F82300C0F3071043283FF45DAF45281A
:100890003FF45AAF25385FFA80FB04980AF04EFC0B
:1008A000BBF11A0FCFD90028D0D1BBF11E0FCDD983
:1008B0004AE74FF48F719CE7A7F126030136022B1C
:1008C0003FF6ECAEA6E7A2F12303022B02D92A2AB7
:1008D0007FF4DFAE236903A962699B1B52F82300F2
:1008E000FFF75AFE88B3232F00F0CC80242F00F0AE
:1008F000A380252F0CBF4FF0180A4FF0220AB51E17
:1009000000F1C8800DF1100909E0013D5046DDE914
:10091000031255F0C1FD03460390681C25D02369DE
:1009200049466269013B5B1B52F82300FFF734FE26
:1009300058B1BAF1220FE8D104980AF0FFFB002861
:10094000E3DA02E0B2F58F7F7CD0B51C2046AD0023
:100950002946FFF735FD014647EA0623C0F8008027
:100960004360002E7FF4FDAE08E703F0010116B1ED
:100970002269921B226101F0FF05002945D043F056
:1009800001012046FFF7D2FC60E62C2FDDD1D4E92F
:100990000423023A53F8221003EB820301F00F0202
:1009A0005B68022A7FF4D0AE002B3FF4CDAE13F08B
:1009B00003027FF4C9AE187932287FF4C5AE21F066
:1009C0000F0144489D6841F0060155F045FD00289F
:1009D0003FF4BAAE2909406804AA05F00DFB049B58
:1009E000002B3FF4B1AED80703F0010107D49A07FA
:1009F0007FF4AAAE384A186890427FF4A5AE059AF3
:100A0000002A7FF4A1AE0393B1E70C2120460193A5
:100A1000FFF7D6FC4FF49D720146019B2046C1E9C9
:100A200000528B60FFF782FC10E620460191FFF731
:100A30007DFC01992046A5E64FF0170A5FE7013ECD
:100A4000036126E6FE21D4E6236903A96269013B1E
:100A500052F82300FFF7A0FD00283FF475AED4E95B
:100A60000432023B52F82330C3F30713342B0CD06B
:100A7000403BD8B2039905F047F9034600F0010165
:100A8000039074E74FF0160A39E70220F2E70133CA
:100A90000361DBE5039B03F0010168E7206918EEC1
:100AA000103A082218EE101A023820612046FFF78B
:100AB00097FDCBE509490190094809F0E3F9A169DF
:100AC0000446019B2A68096809F02AFA2046FBF7C8
:100AD000C3FC00BF98BF0660F4D3066018FD066033
:100AE00078CF06600346006848B110F0030F03D1C9
:100AF00090F804C08C4504D001201360704710604A
:100B0000704700F1080313604068000A704700BF97
:100B10002DE9F04F402393B000240F460390184670
:100B200002920593CDE9064404E0059840080128A7
:100B3000059006D90021C000FBF7C0FC07900028F3
:100B4000F3D0002320200A93CDE9080305E008989C
:100B500040080128089040F2428200218000FBF703
:100B6000ADFC0A900028F2D0079B002B00F03782E2
:100B700000210FA80B97CDE90D1106F047FB029B52
:100B8000002B00F0F181022B0CBF3F22002200233A
:100B9000796C05A8FFF7E6FB069B002B4ED04FF0C3
:100BA000000BDFF80893013B079A069302EBC301A1
:100BB00052F8332091F803A0C2F317024C68BAF13F
:100BC000630F0192B44A12F80A200092B34A12F855
:100BD0000A50B34A88BF45F4807502EB4505009A78
:100BE00002F0300102F00F0610297FD0202952D0E8
:100BF000BBF1000F00F01A81022E00F01281012CCF
:100C000000F0B08014F0010B03D0032E52D14FF04E
:100C1000010B009A631ED20706D5698809EA010113
:100C2000B1F5805F08BF6308012B40F09180BBF1F4
:100C3000000F40F08D80069B002BB4D10FA806F06A
:100C400005FB0E9860B1416800220831FBF754FCA7
:100C50000E9B5A681A60DDE90D235A600E9B0D93B6
:100C600097F84C1041BB099B93B30A9B07981B68EC
:100C70000C93FBF743FC0A98FBF740FC3846FFF760
:100C800035FB0CAB93E80300039B83E80300184695
:100C900013B0BDE8F08FBBF1000F6ED06FF00041D4
:100CA000214435F8111009EA0101B1F5405F60D027
:100CB000012CC1D997F84C10072900F08A8102292C
:100CC00000F08181042900F07881052900F06F810E
:100CD0007449754809F0D6F80446204600237A6C1A
:100CE000396809F01DF92046FBF7B6FB14B1BBF1DA
:100CF000000FA1D0B44236D205EB440509E0C1F3A0
:100D00000B0197F84C208A4200F0B8800134B442BD
:100D100029D2A84635F8021B01EA0902B2F5805F24
:100D2000EDD0631CB342C0F0E68005A84FF0000B85
:100D3000FFF73CFB069B002B7FF435AF7EE7BCF151
:100D4000010F00F01381009B190600F10181234679
:100D50005246019905A84FF0000BFFF741FC6AE7E6
:100D6000002CA9D1069B4FF0010B002B7FF41BAF89
:100D700064E7002105A8FFF7D9FAA64222D905EBBE
:100D8000440B05E001343846FEF71EFEB44219D08C
:100D9000D8463BF8023B03EA0902B2F5805F40F017
:100DA0009880DBB297F84C109942D9D10929E9D142
:100DB000514605A80134FFF745FB3846FEF704FE0F
:100DC000B442E5D1029B002B00F0C980BAF1050FB7
:100DD00040F0C58009990A98013950F821308C00FB
:100DE000002B40F09680044454F8044CA30700F014
:100DF0008A8004F00F04022C00F08B8005A8019972
:100E0000FFF78CFA05A8FFF789FA0023082205A846
:100E1000FFF7E6FB069B4FF0000B002B7FF4C3AE01
:100E20000CE7012C9ED04FF0000BF2E606EA04031B
:100E300003F0010335F8138008EA0901B1F5805F7A
:100E40000FD035E001343846FEF7BEFD04EA060354
:100E500003F0010335F8138008EA0902B2F5805F58
:100E600026D1C8F30B0897F84C2042452FD1002B10
:100E7000E8D1514605A8FFF7E5FAE3E7514605A892
:100E8000FFF7E0FA3846FEF79FFD069B4FF0000B98
:100E9000002B7FF488AED1E6ACBF0660E4C30660E9
:100EA0005CC00660C802076078CF066000F0FFFFF4
:100EB000631C5246019905A8FFF754FA414605A85C
:100EC000FFF774FA069B002B7FF46DAEB6E6013493
:100ED00092E6631C5246019905A8FFF743FAB8F859
:100EE000001005A84FF0000BFFF760FA069B002BDF
:100EF0007FF459AEA2E60199524605A8FFF732FAEF
:100F0000B8F8001011E7002C4AD023793A2B3FF4AF
:100F100075AF002E47D0002405EB4606A44609E035
:100F20000B1B50F823300BB10CF1010C0134B5420E
:100F30003FF405AF36F8023D03EA0902B2F5805FDF
:100F4000EED1DBB2092BF2D101340CF1010CEEE74A
:100F50000134002105A8FFF7E9F92346F8E616B3A6
:100F600009990A980139D6E73D2210E6009B5806F8
:100F70007FF5E9AECCB100252946013505A8FFF77C
:100F8000CDF9002818BF0146AC42F6D105A84FF0B4
:100F9000000BFFF7CBF9069B002B7FF404AE4DE668
:100FA000002EB8D1CFE63446CDE62146EEE70E4915
:100FB0000E4808F067FF04468FE60D490B4808F01D
:100FC00061FF044689E60B490B4808F05BFF0446C5
:100FD00083E60A49084808F055FF04467DE60849BB
:100FE000084804F0D1FD00BF0808076078CF06600C
:100FF000A4030760EC0A0760F0CD0660CC0A076026
:101000003CF706607CCE066010B544682CB12046E3
:101010006468FBF773FA002CF9D110BD2DE9F0419B
:1010200005460E463020002190461F46FBF756FA33
:10103000072D04460570C660A0F8148013D0012D5A
:1010400011D00B4B5B5DE38204F08CFA042320612A
:101050000021238520206783FBF724FA03462046DE
:10106000E362BDE8F081B368C3F30F13EBE700BFA1
:1010700094C4066010B50446C06AFBF73FFA2046E8
:10108000BDE81040FBF73ABA2DE9F041458D07461F
:101090000E469046C06A7DB14FF0000C034601E059
:1010A000AC4509D05C6819460CF1010C0833A64226
:1010B000F6D10846BDE8F081398DA9420CD900EB84
:1010C000C50100236A1C7A8500F8358008464B70FC
:1010D0004B804E60BDE8F0810631C900FBF700FA95
:1010E0003B8D7D8D0633F8623B85E8E730B4458D56
:1010F0007DB1C36A002201E0AA4207D05C681846AD
:10110000013208338C42F7D130BC7047002030BC2C
:1011100070472846F8E700BF30B40346406800280F
:10112000FBD15C8D5CB1DB6A024603E0A24203F1B5
:10113000080304D05D680132A942F7D1184630BCDB
:10114000704700BFF8B543689BB15E688EB14D68CB
:101150005C8D7CB1DA6A002303E0A34202F108024D
:1011600008D057680133BD42F7D11378033B022BF7
:1011700006D9F8BD72683346002AFAD01646E7E76A
:1011800005260E70446801E0067064680022294656
:101190002046FFF779FF0378002BF5D0032BE8D129
:1011A00004230370F8BD00BFF0B51D4683B0B1B194
:1011B00011F0030603D14F68FBB2934204D02B46D3
:1011C00003B0BDE8F04018473F0A08D00C1D0136B7
:1011D000019054F8041FA847B7420198F7D103B013
:1011E000F0BD00BF024B9D228968FFF7DDBF00BF45
:1011F000151E0160024B6B228968FFF7D5BF00BF47
:10120000A119016010B50446084611462268FFF78F
:1012100005FF0023626AC0E90123236A2BB11A4645
:101220009B68002BFBD1906010BD206210BD00BFF9
:1012300010B504460021806A03F014FBA06A102157
:1012400003F0A6F9A06A0121BDE8104003F0D6BB67
:1012500089680022806A090903F054BA806A8968A3
:1012600003F00ABA2DE9F04F804683B00F4692464C
:1012700099461BB10B8B43F008030B83A7F820A002
:10128000D8F824201378002B38D0538D002B35D07C
:101290000025AB4603E00135538DAB422BDDD66A0A
:1012A00016F8353006EBC506043B012BF3D8788DD4
:1012B0000028F0D0002401E0A04216DDFB6A13F8FC
:1012C000342003EBC4030134052AF5D171685B684F
:1012D0009942F1D1D8F82800002372880BF1010B54
:1012E00003F03EF8788DA042E8DCD8F824200135E0
:1012F000538DAB42D3DCBBF1000F09D14B465246B4
:101300003946D8F8280003B0BDE8F04F03F028BBF9
:10131000D8F8280053465A463946CDF8009003F0D5
:101320002BFB03B0BDE8F08FF8B50D4611461A4609
:101330000023044686794769837143610F4BFFF7A9
:1013400033FFA36803B1F8BDE18AA38A01B153B1A9
:101350000A4620462946FFF785FF003E676118BF11
:101360000126A671F8BD1A46A06A03F0BBFAA06A6E
:1013700003F096F9E18AA38AEAE700BF1526016027
:1013800070B5437904460D46012B07D00969AA6858
:1013900020464C23BDE87040FFF7C6BF436A0A46AB
:1013A00002215B8BFFF72EFF01462861EFE700BFAC
:1013B00070B5437905460C46012B08D08E69284646
:1013C0004623E2683146FFF7AFFFF08A70BD13464F
:1013D0000A460721FFF716FF0646A061EFE700BFA8
:1013E00010B500220446806A03F05EF90023A06A6B
:1013F0001A46194603F0E4FA2046BDE81040FFF70C
:1014000017BF00BF10B50446806A03F005FAA38B2E
:10141000626A01339BB2A383D18C994238BFD384D3
:1014200010BD00BF2DE9F04F134687B0814600295B
:1014300065D08A076DD10A790191682A79D001F0C7
:101440000F02022A6BD08A680021120903911A60E8
:10145000019A53684FEA132808F1FF36B8F1000FDC
:1014600077D0171D0024BA465AF8040F25460134D8
:101470000009FCF74DF8A0450644F5D130464FF081
:10148000000BFBF7E3FE4FF02E0A0446029001E04A
:1014900004F801AB57F8040F05A90009FCF74AF856
:1014A000059A014620463CF03DFB059B0BF10102ED
:1014B000AB451C449346EBD1029C31462046FBF7DA
:1014C00057FF2B4B01460022D9F828001C6103F07E
:1014D00047F8039B83B1B8F1010F0DD0019D0124A2
:1014E000083555F8041F01340022D9F828000909ED
:1014F00003F008F9A045F4D107B0BDE8F08F012151
:1015000000221960D9F8280007B0BDE8F04F03F0B9
:1015100027B801F00F02022A01D0019193E70909CF
:1015200019600022D9F8280007B0BDE8F04F03F099
:1015300017B8CA6812091A6089680029DFD001F05B
:101540000F03022B03D001230191039380E70909C4
:10155000E7E73046FBF77AFE31460446FBF708FF23
:10156000034B01464246D9F828001C61CCE700BF76
:101570000004002001B9704701F00303C26813435F
:10158000F9D10B68C360704738B504460D4606486C
:10159000114608F077FC034629462046A360BDE8C3
:1015A0003840FFF7E7BF00BF78CF0660836803B11C
:1015B0007047FFF7E9BF00BF836803B17047014A76
:1015C000FFF7E2BF1006076010B50B7982B0092B58
:1015D0000FD0448B4FF6FF730D4A9C420FD0828B85
:1015E0002146C38B806AD21A02B0BDE8104003F0D6
:1015F000E1B8048B4FF6FF73064A9C42EFD1836833
:10160000002BECD10190FFF7BFFF0198E7E700BF87
:10161000B0020760F40107602DE9F04F437983B011
:1016200005460E46012B02D003B0BDE8F08F91F8BD
:101630000480B8F1100F03D0436A1B78002B4FD001
:1016400001AA6D2106F10800FFF74CFA07460028B1
:10165000EAD04FF0000BDFF8B49009E00AB3052A96
:1016600002D0AA68002A44D00BF1010B5F45DBD001
:1016700001990022686A51F82B100909FFF704FD4F
:10168000B8F1100F04460278E8D112F0FD0F1AD01D
:10169000AA68002AE8D11A4A31462846FFF774FFA3
:1016A000E2E7012201460270686AFFF74BFD2278EB
:1016B000012AD9D1AA68002AD6D1124A3146284631
:1016C000FFF762FFD0E74FF0020A416880F800A000
:1016D000686AFFF721FD0028C6D080F800A0C3E7A4
:1016E0008368002BA0D1084A03B0BDE8F04FFFF794
:1016F0004BBF4A4631462846FFF746FFB4E700BFD6
:10170000700007603405076050FB066080000760CA
:1017100070B50546406A0C46B0F818C01CF0020FC0
:1017200032D101F00F01022918D0217991421FD046
:10173000994230D0A1684CF0020C05260909A0F8A6
:1017400018C001B970BD0022686AFFF79DFC0378DC
:10175000002B37D103234670037070BDAB7921098C
:101760005BB1C38B01260133C3830029EAD0EAE7CA
:10177000A168AB790909002BF3D1838B01260133D2
:1017800083830029DED0DEE721462846134ABDE8E0
:101790007040FFF70BBFAB79002BF5D10123AB7184
:1017A000A368002BCED003F00F030326022B038B7C
:1017B00043F0040303830CD0A36899680909002946
:1017C000C0D0C0E721462846054ABDE87040FFF773
:1017D000EDBEA16809090029B4D0B4E7C8020760CA
:1017E000ACF9066049234822FFF792BF4F234E22EF
:1017F000FFF78EBF42790B46012A04D0426A0349A3
:10180000806A02F089BB406A02F076BB88C5066038
:1018100042790B46012A04D0426A0349806A02F0E9
:101820007BBB406A02F068BB98C5066010B5436A8E
:1018300004465A8BFFF7BCFD01462046BDE8104028
:10184000FFF7E6BF2DE9F0418F6884B00D460446EE
:1018500007F00F030E2B75D07FB90020EA6840F225
:101860002E439A422ED1636A1E788EB1A368002B54
:1018700000F08C8004B0BDE8F081BB07EDD13B796E
:10188000652B5FD0622BE8D1BB680293FF685BE0F9
:101890000146A06A02F09EFEA06A052102F0E6FE63
:1018A0003246A06A012103F01DF803AA39462046FA
:1018B000FFF7B8FD02223146A06A02F051FE04B0E3
:1018C000BDE8F0810146A06A02F084FE02AA6A2106
:1018D00005F10C00FFF706F9804600284BD00025E3
:1018E000029B2E46A06A53F82530013599680909F4
:1018F00002F0BCFEA845F3D100224146A06A0025B3
:1019000002F0F0FF03AA39462046FFF78BFD029B49
:101910000122A06A53F82570B9680909019102F003
:101920001FFEFB682046019903B11909FFF770FFFC
:101930006B1CB5421D46EAD1A06A02F00FFF04B04D
:10194000BDE8F0810297002703AA652102A8FFF7EE
:10195000C9F8002882D0039B40F2DE51043B03EB20
:101960008006002053F8042F8A420CBF0130033058
:101970009E42F7D172E702460146A06A02F0B2FF2A
:1019800003AA39462046FFF74DFDD5E7034A29460D
:10199000204604B0BDE8F041FFF7F6BD90000760B7
:1019A00030B5044683B00D46806A002102F012FE75
:1019B000A06A102102F0ECFD2946204601AAFFF79B
:1019C00031FD01992046FFF723FF03B030BD00BF72
:1019D00042790B46012A04D0426A0349806A02F028
:1019E0009BBA406AFFF750BB90C5066030B505460C
:1019F00083B00C4671B1CA070ED48B072AD001F010
:101A00000F030C09062B1ED00A2B0CD0022B14D06E
:101A1000062C2DD103B030BD4910806A03B0BDE85B
:101A2000304002F0D7BD4379042B28D00E21806AC4
:101A300003B0BDE8304002F01FBE214603B0BDE850
:101A40003040FFF7C5BF2146806A03B0BDE8304093
:101A500002F00CBE0968806A02F016FD22790E4B76
:101A60002146284653F8223003B0BDE830401847DD
:101A7000E1B2806A03B0BDE8304002F089BD01A93F
:101A80002046FBF757FDAC6A01990BF03BFD014680
:101A9000204602F0F1FDBDE79CC406602DE9F04F41
:101AA000074683B00C461646984611E0FEF764FDE3
:101AB00050BBD4B1A30718D16168CBB2090A1E2B61
:101AC0002BD01F2B59D0202B0DD1A46886F00106F6
:101AD0002046FEF743FD03462046002BE6D0AEB17C
:101AE00003B0BDE8F08F2D2B0BD038462146FFF711
:101AF0007DFF42463146B86A03B0BDE8F04F02F0C0
:101B000041BEA368002BEAD0002EE9D04146B86A56
:101B100003B0BDE8F04F02F02FBE86BBD7F810909F
:101B200001F1FF3A09F10103BAF1000F3B6114DD45
:101B300004EB810586F0010204F1040B01962646B0
:101B40002C4615465BF8041F4B462A463846FFF7DD
:101B5000A5FFA345F6D13446019E0AF1020A384694
:101B60004346324654F82A10FFF798FF4946B86AB0
:101B700003B0BDE8F04F02F0E3BC002ECED1002947
:101B8000AED0251D05EB810455F8041F43463246AF
:101B90003846FFF783FFAC42F6D103B0BDE8F08FC3
:101BA00070B5466A04460B463278072A04D0022AEA
:101BB00002D0836843B370BD9D6875B1AA0702D196
:101BC0002B79AF2B13D029462046FFF70FFFA06AD1
:101BD0000021BDE8704002F011BFA06A102102F0A0
:101BE000D7FC2946A06ABDE8704002F007BF338BDE
:101BF000DB060ED5A368002BDDD129462046094A15
:101C0000BDE87040FFF7C0BC074ABDE87040FFF771
:101C1000BBBC2046A968FFF7E9FE2046BDE870403E
:101C2000FFF706BBD80407606405076001F00F03E7
:101C3000022B70B50E460446154601D083689BB151
:101C400029462046FFF7D2FEA06A02F07FFD656AB2
:101C50002B78033B032B01D86B6863623109204664
:101C6000FFF7D6FD656270BD014AFFF78DFCE7E71F
:101C700018FB0660D1E90212FFF7D8BF38B50C4651
:101C80000546C968FFF7B2FEA1682846BDE838409E
:101C9000FFF7ACBE38B50B790C460546342B17D090
:101CA0001021806A02F074FCA468C4B1A30704D1B7
:101CB00023799A2B2AD09B2B16D021462846FFF752
:101CC00095FEA86A04220221BDE8384002F00ABE4F
:101CD0008968FFF78BFEE468A468002CE6D1102128
:101CE000A86A02F055FCECE7A1682846FFF77EFEE3
:101CF000E36899680029E4D02846FFF777FEA86AD0
:101D000004220321BDE8384002F0ECBD1021A86A8E
:101D100002F03EFCA1680029EED1D2E710B50446DE
:101D20008968FFF763FE0021A06ABDE8104002F059
:101D3000CBBC00BF2DE9F04706690446838B0D46F6
:101D4000B0F81E80771CC383B31CD0F818900361D1
:101D5000068347838868FEF701FC68B12046C4F813
:101D60001890A4F81E802969FFF740FE3146A06A4A
:101D7000BDE8F04702F0E4BBD4F810A00AF101037B
:101D80002361A868FEF7F8FB90B15146A06A02F003
:101D9000D7FB2046E968FFF729FE3946A06A02F022
:101DA000CFFB53460122A9682046FFF777FED5E70F
:101DB0003946A06A02F0E0FCE7E700BF10B5044630
:101DC0008968FFF713FEA06ABDE8104002F0C6BCA8
:101DD00010B5426A04461278072A02D0836893B18C
:101DE00010BD896831B1FFF701FEA06ABDE810405F
:101DF00002F0F4BD806A102102F0CAFBA06ABDE8BF
:101E0000104002F0EBBD024ABDE81040FFF7BCBB3A
:101E1000100407602DE9F84301F00F030C46054656
:101E2000022B21D019B9AB681BB3BDE8F88311F0C0
:101E30000306F8D10B792C2B22D02D2BF3D1A468DB
:101E4000002CF0D063681B0A022B33D0002BECD09F
:101E5000271D57F8041F2846FFF7DCFF013663688B
:101E6000B6EB132FF5D3E0E70909BDE8F843FFF718
:101E7000C1BC21462846244ABDE8F843FFF784BB8D
:101E80008968FFF7B3FDE768002FCCD017F0030691
:101E9000C9D17B683946DAB28E2A14D0312A28D0CB
:101EA000322AC0D189680222A86A0909BDE8F8432C
:101EB00002F028BCE368002BCAD09A07C8D11B796E
:101EC000AC2BC5D1AFE71B0A03F1FF38B8F1000F07
:101ED00009DD07F10409013659F8041F2846FFF708
:101EE00085FD4645F7D108F1020857F828100A7910
:101EF000D4E728468968FFF779FDA86A0221BDE882
:101F0000F84302F0E1BB00BF6CFB0660F8B54B681C
:101F100005461F0A09D00C1D04EB870654F8041F60
:101F20002846FFF763FDB442F8D13946A86A00227B
:101F3000BDE8F84002F0D6BC2DE9F0414F68884674
:101F400005463F0A15D00E1D002402E00134A742C9
:101F50000FD056F8041F2846FFF748FDAB68002B4A
:101F6000F4D00234284658F82410BDE8F041FFF7B9
:101F700001BBBDE8F08100BF10B50446FFF7DCFFF0
:101F80002221A06ABDE8104002F08ABC2DE9F0478A
:101F9000D0F8109082B00646884609F1010303612B
:101FA0008868FEF7DBFA18BB346902463046631CCA
:101FB00033612346D8F80810FFF770FD3046D8F893
:101FC0000C10FFF713FDD8F80800FEF7D5FA00282B
:101FD00045D1D8F8103013B9D8F8143023B1B06A0D
:101FE00002F032F9002846D02146B06A02F0A8FA81
:101FF00001AA712108F11000FEF774FD074648B3ED
:10200000002401E0A74225D0019B53F8245001345D
:10201000A868FEF7A3FA02460028F3D1D6F810A06C
:1020200030460AF1010153463161A968FFF736FDD8
:102030003046E968FFF7DAFCA868FEF79DFA70B948
:10204000B06A02F001F988B15146B06A02F078FA3C
:10205000A742D9D1D8F814103046FFF7C7FC49463B
:10206000B06A02F06DFA02B0BDE8F0874946B06A86
:1020700002F082FBE8E74946B06A02F07DFBB3E775
:1020800070B5437904461546CE68012B13D07169AB
:10209000002320461A46FFF7E5F8F1682046FFF7CF
:1020A000A5FC062D10D00023A06A01211A46BDE828
:1020B000704002F077BC436A0A4629465B8BFFF703
:1020C000A1F801467061E3E70021A06A02F0CAFBB3
:1020D000E9E700BF8968034671B14A68120A022A1B
:1020E00007D1CA682AB112F0030F02D11279AC2AC3
:1020F00006D01846FFF70ABF0A46806A02F0F2BB14
:102100000622FFF7BDBF00BF10B5896882B0044644
:1021100081B18B0703D14B68DAB2922A11D02046E5
:10212000FFF764FC0122A06A114602B0BDE810402E
:1021300002F0D8BB0122806A02B0BDE8104002F074
:10214000D1BB1B0A022B0CD1CB6853B19A0708D123
:102150001B79AC2B05D1032202B0BDE81040FFF77C
:102160008FBF20460191FFF7E7FE01990122A06A87
:102170004968090A02B0BDE8104002F0B3BB00BFD5
:102180002DE9F04F87B0144680461D46039105AAFD
:10219000A42103A80294FEF7A5FC0746002800F03E
:1021A0009F800024A346A2462646A146059B53F8DD
:1021B0002430002B3FD099073DD11A79A62A44D06C
:1021C000A72A48D0A82A36D1DA68002A49D19968C6
:1021D00001F00F02022A40F08C800909D8F828008B
:1021E000019302F043FA019B404609F10109D968C5
:1021F000FFF7FCFB0134A742D8D17EB1BAF1000F42
:1022000057D0DAF808104046FFF7F0FBBBF1000F9B
:1022100054D0DBF808104046FFF7E8FB029B002B88
:102220003DD033464A462946D8F8280002F0C8FB7C
:1022300007B0BDE8F08F16BBB9F1000F27D11946E2
:1022400040460135FFF7D2FBD4E7F20742D446F00F
:1022500001069A46CEE7B00745D446F002069B46F3
:10226000C8E79107B3D11179AA292CD0AC29AED1F6
:102270001946062240460135FFF702FFBAE7204A19
:1022800019464046FFF792F907B0BDE8F08F1D4AA6
:1022900019464046FFF78AF907B0BDE8F08F33468C
:1022A0004A462946D8F8280002F07CFB07B0BDE872
:1022B000F08FD8F8280002F0F3F9A7E7D8F8280043
:1022C00002F0EEF9AAE79268404699680135FFF7F7
:1022D000ADFC8FE70C4A19464046FFF767F9D3E794
:1022E000064681469AE7094A19464046FFF75EF9D5
:1022F000CAE7074A19464046FFF758F9C4E700BF46
:102300009C050760AC0507609CFB066090FB0660BF
:1023100098F1066070B50D464179044601291CD03C
:10232000A06A02F0CDF96E690023204631461A46B4
:10233000FEF798FFF18AA06A02F098F9E96829B1DE
:102340008B0703D10B79A32B08BF00212046022362
:102350000022FFF715FFF08A70BD13462A46FEF7EC
:1023600051FF6861DCE700BF10B5436A04465A8B31
:10237000FFF7D0FF01462046BDE81040FFF748BAFE
:10238000002389681A46FFF7FBBE00BF2DE9F04F16
:102390008A4685B00646422102AA0AF10800CDF815
:1023A00004A0FEF79FFB736A0746B3F81AB058B350
:1023B00000258246A946029B03AA6C2153F825708A
:1023C00007F10800FEF78EFB039B804619680A0997
:1023D000732A37D03046FFF709FBB8F1010F0BD94C
:1023E0000124039B0022B06A53F824100134090928
:1023F00002F088F9A045F4D1F968002938D10135F7
:10240000AA45D8D1AAEB0907019BD9680B79032B00
:102410003FD0442B30D05A463046FFF77BFF05466D
:102420004FB10024002301340121B06A1A4602F0A2
:10243000B9FABC42F6D129463046FFF7E9F905B0B2
:10244000BDE8F08F022806D159680B09412B07D04F
:10245000B3F5737F01D0B3682BB109F10109CEE761
:102460004FF0010BF9E70E4A3046FFF78DF8F4E71D
:102470003046FFF7BBFAC2E78C685A463046214621
:10248000FEF796FFA2690546138B43F011031383F1
:10249000C6E75A463046FEF78BFF0546C0E700BF49
:1024A000A00207602DE9F0418E6882B0044615460F
:1024B0001EB922BB02B0BDE8F08116F0030712D1AD
:1024C0003379372B2BD09F2B0DD1F3681A79A12AA2
:1024D00036D0B368DBB19A0719D11B79372B16D1E7
:1024E0000422314616E031462046FFF77FFA0322E8
:1024F0000121A06A02B0BDE8F04102F0F3B9022266
:102500003146A06A02B0BDE8F04102F0EBB9052205
:102510003146204602B0BDE8F041FFF7B1BD4AB9EF
:1025200020463146FFF762FAA06A02B0BDE8F041EA
:1025300002F0E4B902220121806A02F0D3F9EFE748
:10254000A22103F1080001AAFEF7CCFAB168804687
:1025500021B1880702D10B79372B3DD02046FFF7F8
:1025600045FAB8F1000F26D0002502E00137B84542
:102570001ED9019B204653F82730194623B19A07EC
:1025800002D11A79372A0CD0FFF730FA002DEDD09E
:10259000A368002B8ED11B4A31462046FEF7F4FF7C
:1025A00088E7FFF723FA6DB1A06A02F0A7F9DDE72B
:1025B000002D7FF47FAF032208F10101A06A02F031
:1025C00091F977E7A368002B7FF474AF0E4A314688
:1025D0002046FEF7D9FF6DE75DB92046FFF706FA02
:1025E000A06A02F08BF9B8F1000F3FF463AF012548
:1025F000BFE708F101010222A06A02F073F9B16895
:10260000EBE700BF74FE066068FE06600122FFF77C
:1026100049BF00BF01F00F03022B70B5044626D05E
:102620000B79492B01D04F2B02D10123A37170BD2F
:102630004A2BFCD0502BFAD0482B8E680CBF0D696A
:10264000CD68A5B183796BB3838A01339BB2012B2B
:1026500083821BD029462046FFF7C8F9A06A3109BA
:1026600002F004F8A06ABDE8704002F047B9A3790F
:10267000002BDCD1E38A002BD9D0A368002BD6D164
:1026800020460E4ABDE87040FEF77EBFC18A89B180
:102690000022806A02F026F902220021A06A02F0DC
:1026A00021F9D7E7C38A29460133C382BDE87040C8
:1026B000FFF79CB9806A01F0F3FFEDE78005076042
:1026C000F8B50C460646D1E90171FFF78FF93F0ACC
:1026D000022F0FD9022521693046FFF787F9E168FB
:1026E0000235B06A090908342539C9B202F0D8F8B0
:1026F000AF42F0DCF8BD00BF2DE9F0414F680D4658
:1027000089680646A7F10D083F0AFFF76FF9012F08
:102710005FFA88F80DD908350124304655F8041FB2
:102720000134FFF763F94146B06A02F0B9F8A742F5
:10273000F3D1BDE8F08100BF38B50C46C968054645
:10274000FFF754F9A168C1F30711342906D04039C5
:10275000A86AC9B2BDE8384002F09CB8A86A022154
:10276000BDE8384002F096B810B504468968FFF716
:102770003DF90321A06ABDE8104002F08BB800BF0C
:102780002DE9F8430769064691F804907B1CA9F1EE
:102790001E0903614B68B9FA89F95FEA13284FEA09
:1027A00059190BD00D1D0024013455F8041F304673
:1027B000FFF71CF944453A46494605D13946B06A07
:1027C000BDE8F84301F0BCBEB06A01F0E7FFEBE7FB
:1027D0002DE9F8430D460646D1E90171FFF706F9E8
:1027E0003F0A032F4BD9D6F8109009F1010333614A
:1027F000022F42D9A7F10308012428F0010808F1AB
:10280000030813E00B79852B2ED08B6853BB07216F
:10281000B06A02F045F8BC4204DA4A460021B06AC8
:1028200001F0BCFF444505F1080524D002342969B4
:102830003046FFF7DBF8BC4205DAB06A01F086FFEC
:10284000B06A01F095FFE96801F00F030E2BD9D1B2
:10285000C1F3071126290CD03539C9B2B06A02F08C
:102860001FF8D8E73321F9E73221B06A02F018F8EF
:10287000D1E70621F2E7032F04D8BDE8F8834FF033
:102880000009B5E73469B06A631C2146336101F081
:1028900073FF4946B06A01F053FE0121B06A01F0AE
:1028A000D9FCB06A01F060FFB06A01F057FF214621
:1028B000B06ABDE8F84301F043BE00BFF8B5056952
:1028C0000E46CF680446AB1C002203612B46B96854
:1028D000FFF7E4F8B1686E1C2046FFF787F8A06A9E
:1028E000314601F049FF2946A06A01F029FEA06A9D
:1028F0004FF0FF3101F0AEFC2046F968FFF776F8A3
:102900003146A06ABDE8F84001F01ABE2DE9F04F4B
:1029100085B005691F4692460E9B012204460E466D
:102920000393AB1C29460361AB180293FEF76AFDC3
:1029300031462046FFF75AF80022A06A691C01F0D0
:10294000A3FF2946A06A01F0FBFDA06A02F064F82B
:10295000D4F810B0BAF1000F0BF10106266140F374
:102960008F8001251CE05545A94640F0A180A06A52
:1029700001F0F4FED8F80C102046FFF737F80122DA
:10298000A06A5946154401F07FFF3146A06A01F064
:10299000D7FD0121A06A01F05DFCD14570DA2669FE
:1029A0003946731C0437D1F800802361D8F80890A9
:1029B000B9F1000FD7D019F0030303D199F804201F
:1029C000762A14D0A06A01F0C1FE49462046FFF7DE
:1029D0000DF8A06A082101F063FF32460021A06AC9
:1029E00001F0D0FEA06AA94601F0B8FEC2E7D9E91D
:1029F0000212A06A4FEA12190193009101F0A6FE9B
:102A000000992046FEF7F2FFA06A082101F048FF76
:102A1000019B3246A06A194601F0B4FEB9F1000FDD
:102A2000E0D049462046FEF7F3FE23690222204605
:102A3000591C009321611946FEF7E4FCD8F80C10EC
:102A40002046FEF7D3FFA06A102101F0A1FD009BF4
:102A5000A06A194601F074FDA06A102101F098FDEA
:102A600049462046FEF7D4FE49462046A946FEF7D1
:102A7000C1FEA38BA06A013BA38301F0EDFE7EE7BC
:102A8000A38BA06A013BA38301F0E6FEA06A01F0DC
:102A9000C7FF0299A06A01F053FD03992046FEF793
:102AA000A5FF5946A06A05B0BDE8F04F01F048BD4A
:102AB000A36843B1A38BA06A013BA38305B0BDE823
:102AC000F04F01F0C9BE034A20460968FEF75CFDDD
:102AD000F0E700BFB0FD06602DE9F04706699846B3
:102AE00082B01546731C0F4602223146036104462C
:102AF000DDE90AA9FEF786FC0DBB0321A06A01F0FF
:102B0000A9FB39462046FEF771FF6FF00201A06A6B
:102B100001F0A0FBA06A102101F03AFD3146A06A45
:102B200001F00EFD20464946FEF760FFA38BA06A28
:102B3000013BA38302B0BDE8F04701F08DBE4346E0
:102B40002A4639462046CDF800A0FFF7DFFEE1E730
:102B500070B5CD6884B00C4606462B79782B1BD017
:102B6000742B03AA4FF077010DD004F10C0000255F
:102B7000FDF7B8FF0246A1683046039B0095FFF7BA
:102B8000C5FE04B070BD05F10800FDF7ABFF2B6971
:102B900002465BB9ED68EEE70023AA688968CDE9D3
:102BA00000321A46FFF798FF04B070BD9B683046AC
:102BB000A1680193EC68039B0094FFF78DFF04B0BC
:102BC00070BD00BFF8B5154B04460D46D3F814612F
:102BD00006B1F8BD07690122BB1803613B4689684D
:102BE000FEF75CFF1F210122A06A01F0F9FBE968F2
:102BF00049B9A06A012101F0FBFE3946A06ABDE88F
:102C0000F84001F09DBC2046FEF7F0FE3346324608
:102C10000121A06A01F0C6FEEBE700BF000400201E
:102C200038B58D68044675B1AB0702D12B795E2BA0
:102C30000FD029462046FEF7D9FEA06A0121BDE843
:102C4000384001F0D5BE2946806ABDE8384001F021
:102C5000CFBEA968FEF7CAFEE9682046FEF7C6FEA9
:102C6000A06A0221BDE8384001F0C2BE2DE9F0475C
:102C70008F070C460646154610D001F00F03022BB5
:102C800004D0B368002B58D0BDE8F087D6074FEAD0
:102C900011114ED5BDE8F047FEF79ABE4968CBB298
:102CA0002D2B51D023D8062B39D02C2BE9D1022A39
:102CB00060D1E768002FE4D017F00308E1D17B680A
:102CC000B946DAB28E2A59D0312A72D0322AD8D1F6
:102CD000012D00F08F80022D00F09880D9F80810A7
:102CE0000122B06A0909BDE8F04701F00BBD2E2BA7
:102CF00013D1002AC5D1A168002937D08D0704D18E
:102D00000A464968CBB2922B24D004F1080230461F
:102D10000121BDE8F04700F07FB89D2BB1D1002D17
:102D2000AFD104F108023046090ABDE8F04700F0CF
:102D300073B8BDE8F047FEF76BBD21463046354A13
:102D4000BDE8F047FEF720BCA268002A99D0002D0C
:102D500097D15168090A022906D1D36823B198078F
:102D600002D11B79AC2B8CD008323046BDE8F0473D
:102D700000F052B8A168FEF739FE9AE74FEA13292E
:102D8000022D09F1FF390DD0B9F1000F0ADD07F16D
:102D9000040A08F101085AF8041F3046FEF726FE1F
:102DA000C845F6D109F1020957F8299099F804208D
:102DB0008AE7022D0CD0D9F808103046FEF716FE2F
:102DC000012D0ED0B06A0121BDE8F04701F07CBCB6
:102DD000B06A01F0CDFCB06A0121BDE8F04701F016
:102DE00073BCB06A01F0B6FCB06A0021BDE8F047E0
:102DF00001F06ABCB06A01F0A9FCD9F80810B06A09
:102E000000220909BDE8F04701F07CBCB06A01F07E
:102E1000ABFC63E718FB06602DE9F04781460E46E0
:102E2000174600294CD04FF0FF38151F002401EB46
:102E3000080A02E00134A64216D055F8043F002BE0
:102E4000F8D09A07F6D11A79222AF3D1B8F1FF3FC8
:102E5000AAEB0402214628D1A0460134D9F8280063
:102E600001F076FDA642E8D1B8F1FF3F17D000246B
:102E700006E001343968FFF7F9FE0437A6420CD9A1
:102E8000A0454FF000024846F3D13B6801340437B7
:102E90009968FFF7EBFEA642F2D8BDE8F08731460D
:102EA000D9F8280001F04EFDE1E7D9F80820002A02
:102EB000F3D14846054A1946BDE8F047FEF764BB22
:102EC000806ABDE8F04701F03DBD00BFA404076083
:102ED0002DE9F843066905461F460C46B31C06F16A
:102EE0000109806A31462B61904601F029FB494671
:102EF000A86A01F0BFFCA16800222846FFF7B6FED1
:102F000024692CB926E0A168FEF7C8FDE4680CB37B
:102F100094F804C0334600222846BCF1AD0FF2D02D
:102F2000E168FEF763FD0121A86A01F09BFC7B1CB0
:102F3000424621462846FFF7CBFFA86A314601F0FA
:102F40001BFCA86A494601F0FBFAA86ABDE8F843F1
:102F500001F096BC41462846FEF748FD6B6A197899
:102F6000062905D0BA00A86A053201F0CDFCE4E7D5
:102F7000A86A002101F042FDA86A01F0EFFBDCE73E
:102F80002DE9F04F2DED028B8B6887B00F4604467C
:102F900003F00F03022B02D1CB68002B46D1256929
:102FA0002046A84BD4F818A06E1C2B43B4F81E90F2
:102FB000668305F102082383A38BE383EB1C236163
:102FC000F968FEF713FDA06A012101F04BFC3146C0
:102FD000A06A01F0B5FA4146A06A01F04BFC00225C
:102FE000B9682046FFF742FE20463969FEF7FEFC2D
:102FF000A06A01F029F9002800F0C6804146A06AC5
:1030000001F09EFAA06A01F03BFCC4F818A0A4F8F5
:103010001E9020467969FEF7E9FC2946A06A07B0B0
:10302000BDEC028BBDE8F04F01F08ABA9807B6D12B
:103030001A792C2AB3D19A6802F00F010229AED175
:1030400012097C2AABD1DB681A79302AA7D19B6898
:1030500005AAA42104A80493FDF744FD431E0246DB
:10306000022B9CD8012800F09480022800F0968062
:1030700005998E68D1E9002BF10790D573088ED0A1
:103080002AB1930703D11179A639022987D9BBF157
:10309000000F08D01BF0030F05D19BF80410A639D0
:1030A00002297FF67CAFBB68256908EE103A3B69C0
:1030B000A18B05F1010808EE903AA369281D7F69EC
:1030C000029305F10209E38B05F1030A20610193E4
:1030D0001BF001032583A4F81A80E183009300F01C
:1030E000888011462046FEF781FC5146A06A01F017
:1030F00043FB4946A06A01F023FAA06A01F026FBCF
:10310000002218EE101A2046FFF7B0FD18EE901AB4
:103110002046FEF76BFC4146A06A01F011FA3146E9
:103120002046FEF763FCA06A0E2101F0B9FBA06AFD
:10313000514601F005FA009BA06A002B52D101F024
:1031400009FBA06A01F010FB002EA06AACBF0021B1
:10315000012101F0A5FBA06A4A46012101F012FB02
:10316000029BA06AA361019BE383E7B9294601F0B2
:10317000E7F9A06A01F0F2FA009B002B40D007B0FB
:10318000BDEC028BBDE8F08F3146A06A01F0F4FA85
:1031900034E7059B0326D3F800B078E7059B0326A8
:1031A000D3E9002B6CE701F0D9FA009B63B33946F1
:1031B0002046FEF71BFC2669A06A731C314623617A
:1031C00001F0DAFAA06A012101F044F8A06A294668
:1031D00001F0B6F9A06A01F0C1FA3146A06A01F027
:1031E000AFF9CCE701F0B2FA59462046FEF7FEFBF4
:1031F000AAE7594620460392FEF7F8FB039A70E7C8
:10320000A06A01F0ABFABAE7A06A01F0A7FA394662
:103210002046FEF7EBFB2669A06A731C314623614A
:1032200001F0AAFAA06A022101F014F82946A06A66
:1032300001F086F9A06A01F091FAA06A01F08EFA15
:10324000CBE700BF0080FFFF2DE9F043044683B0C9
:1032500090460D4661B307697A1C0261D8F8006098
:103260002EB116F0030902D132797B2A26D03146DD
:1032700020460193FEF7BAFB204600223946FEF7AE
:10328000C1F8A06A01F06AFA019B08F10402691E04
:103290002046FFF7D9FFA06A394601F0C7FAA38B91
:1032A000A06A013BA38303B0BDE8F04301F0D4BAA8
:1032B000194603B0BDE8F043FEF798BBB16801932F
:1032C000FEF794FB4A4639462046FEF79BF84A46ED
:1032D000F1682046FFF7CAFC019BD6E730B50C46E3
:1032E00083B005467A2101AA04F10800FDF7FAFB34
:1032F000E3680146019A2846FFF7A6FF03B030BDF8
:103300002DE9F04F044683B017460E46002900F021
:10331000D68005692A1D05F1010905F1020A05F1AA
:1033200003080261D7F800B0BBF1000F07D01BF013
:10333000030204D19BF804107B2900F0C680594693
:1033400020460093FEF752FBA06A01F0FFF92046E9
:10335000A821FEF745F8A06A01F000FA009B0222BE
:10336000294620460093FEF74DF8A06A032100F09D
:1033700071FF009B3A1D711E2046FFF7C1FFA06A36
:103380006FF0020100F066FF1021A06A01F000F961
:10339000A06A01F0E9F94946A06A01F0EDF9294671
:1033A000A06A01F0CDF8A06A01F0D0F90122A06A6C
:1033B000212101F015F8A06A082101F071FA5246A6
:1033C0000021A06A01F0DEF9A06A01F0BFF9A06A4D
:1033D00001F0CEF9A06A01F0C7F90022A921A06A84
:1033E00001F062F9A06A01F0C3F9A06A01F0C0F926
:1033F000A06A01F0ABF900220A21A06A01F082F96B
:10340000A06A01F0B1F9A06A102101F0C1F800230F
:103410000321A06A1A4601F0D3FA2046FDF708FFFF
:1034200042460021A06A01F0ADF9A06A01F096F9C8
:10343000A06A102101F0ACF84146A06A01F09CF9A5
:10344000A06A022100F006FF5146A06A01F078F858
:10345000A06A01F08DF9A06A01F08AF94946A06AD4
:1034600001F06EF80022A06AA92101F01DF91021D7
:10347000A06A01F08DF8A06A01F068F9A06A01F075
:1034800065F900230321A06A1A4601F099FA204643
:10349000FDF7CEFEA06A01F061F9A06A4FF0FF319E
:1034A00000F0D8FEA06A414601F04AF8A38BA06A5A
:1034B000013BA38303B0BDE8F04F01F0CDB919463D
:1034C00003B0BDE8F04FFEF791BADBF80810CDE984
:1034D0000032FEF78BFAA06A01F038F92046A821E5
:1034E000FDF77EFF019ADBF80C102046FFF7BEFBCC
:1034F000009B34E72DE9F0410D46002611460446B5
:1035000006612A4645624171806A00F069FD63796F
:10351000012B08BF6E62EE680EB1B20737D02B7870
:10352000002B5BD0072B41D0022B00F08980033B9E
:10353000032B58D86779D6F80C80012F00F0B4809F
:103540003168A06A00F0A0FF2B78032B00F0A58063
:10355000042B00F0B680052B00F0BA80062B00F09B
:10356000858001212046FEF733FA0121A06A01F08F
:1035700079F90023B26841462046FFF7A9FC2B7871
:10358000062B55D11021A06A01F002F850E03379E2
:103590003F2BC4D12046B168FEF728FAA06A01F09B
:1035A0001DFAA06ABDE8F04100F0FABD6379012B75
:1035B0006AD020467169FEF719FAA06A00F044FE4D
:1035C0000028EED1A06A102100F0E2FFA06A01F00D
:1035D00005FAA06ABDE8F04100F0E2BD31462046A0
:1035E000FEF704FAEEE76379012B64D01721204639
:1035F000FEF7EEF916212046FEF70AF9B168A06A37
:10360000090901F033F81A212046FEF701F9316962
:103610002046FEF7EBF90A212846FDF767FD0378FF
:10362000032BAFD0428800230A21A06A00F098FE45
:10363000A06A01F0D3F9A06ABDE8F04100F0B0BD86
:103640003168A06A00F020FF6379012B47D0F16850
:103650002046FEF7CBF92B8BDB07E9D5A06A01F0FA
:103660007DF81021A06A00F093FFE1E7A06A01F065
:1036700017F801212046FEF7ABF9A06A01F010F817
:10368000A06A01F00DF874E70021194B462220468C
:10369000A171F168FDF788FD8BE701220021A06A86
:1036A00001F020F92B7859E703223946606AFDF7CB
:1036B000EBFCAF8344E703220A212846FDF7E4FC34
:1036C00094E702220021A06A01F00CF92B7845E76B
:1036D00003220021A06A01F005F92B783EE70022C1
:1036E000044B2046A2714C22B168FDF75DFDAEE7A8
:1036F000E5170160ED1701602DE9F0410C4682B03D
:1037000089680746FEF772F9E668002E39D07568B9
:10371000EBB28E2B38D004F10C0601257B6A1B78A6
:10372000072BA36803F00F0231D0022A52D00024E5
:1037300002E01C46FEF75AF9A54222D9631CA200FA
:10374000384656F82410AB42F3D291F804C0BCF1CD
:10375000320FEED13244D2F8048098F80420302A97
:10376000E7D189680022B86A0234090900F09CFF99
:10377000D8F80810002301223846FEF701FDA542C3
:10378000DCD802B0BDE8F0812D0A0836C6E7022A6F
:10379000CDD11B099A2B1FD0B3F5D97FC7D1336880
:1037A0001A79302AC3D19C68002CC5D014F00302CA
:1037B000BDD123792F2BBAD113461146B86A012403
:1037C000019201F0EFF833683846019A9968FEF7E4
:1037D00069FEB1E71B09DFE733681A79302AA6D101
:1037E0009B68002BA3D10A213846FEF7F1F87A6ACC
:1037F000D36A528D22B918E0013A03F1080314D0BC
:103800005978C907F8D559683846FEF7E1F8022D0E
:1038100003D973681A79322A12D000230221B86AB8
:1038200001241A4601F0BEF886E7BB68002BA8D138
:103830000C4A3846316802B0BDE8F041FDF7A4BE3D
:10384000B4682279302AE8D199680122B86A090956
:1038500000F02AFFA1680023012238460324FEF766
:103860008FFC69E7B009076010B5426A04460B4651
:103870001278072A04D0022A02D08368CBB110BD87
:1038800019462046FFF738FFA06A0022AD2100F05C
:103890000BFF0023A06A19461A4601F091F8A06AAE
:1038A000102100F075FEA06A0121BDE8104001F072
:1038B000A5B8024ABDE81040FDF766BEA00007604B
:1038C0002DE9F843CE680D4604464EBB037943B953
:1038D000A9688D071BD001F00F03022B18D0BDE89B
:1038E000F883436A1E78002EF2D1D221FEF770F8D9
:1038F000A9682046FEF77AF8A06A334632460121CD
:1039000001F050F8A06ABDE8F84300F027BFF9B90C
:103910002046FEF76BF8A06ABDE8F84300F01EBF32
:1039200016F0030709D17168CBB25B2B14D0562B6C
:1039300025D0572B6ED0062B37D031462046FEF7C8
:1039400055F8A96820460022BDE8F843FFF78EB974
:103950000B793A2BDCD1C2E7F668002E40F0858067
:10396000406A0378072BBAD1A96801F00F03022B34
:10397000B5D103220909BDE8F843FDF785BB012253
:10398000A968FFF773F9F1682046FEF72FF8B168D0
:10399000A06A09093F39C9B200F082FFA968204630
:1039A0000222BDE8F843FFF761B9AF68002FC4D029
:1039B000B807C2D17B68DAB2062ABED1090A1A0A50
:1039C000B1EB132FB9D1022AB7D1BB6823B1990744
:1039D00002D11B79222BB0D0FB6823B19A0702D108
:1039E0001B79222BA9D0B1682046FDF7FFFFF168B3
:1039F0002046FDF7FBFFA06A00F0B6FEB96820463E
:103A00000022FFF733F9F96820460022BDE8F843A9
:103A1000FFF72CB94FEA112808F1010308F1FF392B
:103A200056F82310FDF7E2FFB9F1000F89DDA06A17
:103A300000F08CFEA9683A462046351DFFF716F9BE
:103A400001374F4507D156F8281020460022BDE81F
:103A5000F843FFF70BB9A06A00F078FE002255F892
:103A6000041F2046FFF702F9EAE7B3077FF465AFCA
:103A70007168CBB25FE700BF2DE9F04F8D6885B06C
:103A800004462B79032B1ED0426A128BD20710D525
:103A9000162B23D003AA7A2105F10800FDF722F89E
:103AA000EB680146039A2046FFF72AFC05B0BDE803
:103AB000F08F8368002BF9D1544A294605B0BDE840
:103AC000F04FFDF761BD2946FDF7B0FEAA69138BE3
:103AD00043F01103138305B0BDE8F08F0669EB686E
:103AE00006F1010A4FEA1318331D0361E968FDF777
:103AF0007DFFA06A0022AA2100F0D6FD0023A06A63
:103B00001A46194600F05CFF41462046FDF780FE4C
:103B10002769A28B07F10109B91CA369B4F81EB08B
:103B2000A06A21614946E2832783A4F81A90019391
:103B300000F006FD012251462046FDF763FC414698
:103B4000204606F10208FDF743FF2046AC21FDF7B1
:103B500047FCA96820460022FFF788F80022A06AE7
:103B6000414600F091FE5146A06A06F1030A00F0BA
:103B7000E7FCA06A00F050FFA06A00F0E7FD012218
:103B8000A06A40F2F71100F02BFCA06A082100F0B7
:103B900087FE52460021A06A00F0F4FDA06A00F002
:103BA000DDFD0122A06A314600F06EFE5146A06A9A
:103BB00000F0C6FC0121A06A00F04CFBA28BA06AB9
:103BC000013AA28300F048FEA06A00F029FF4146B6
:103BD000A06A00F0B5FC20462969FDF707FF4946B9
:103BE000A06A00F0C9FD019B3146A06AA361A4F858
:103BF0001EB000F0A5FC20466969FDF7F7FE3946C6
:103C0000A06A05B0BDE8F04F00F09ABC4C01076017
:103C10002DE9F04F8DB014460D4628220021824632
:103C200002A839F0C3FF00234FF0FF3201A8194664
:103C30008DF808400792DAF800200195FDF7E2FAC6
:103C4000044600F0B5F9DDF8248006460B90B8F183
:103C5000000F00F04D812346002544469846039FFF
:103C6000FFB90122214601A8FFF744FC628D1AB971
:103C700010E0013797420DD2E16A11F8373001EBBD
:103C8000C701012BF5D120460137FDF75BFA628DA4
:103C90009742F1D3059BA4689D4238BF1D46002C76
:103CA000DDD1099B4446002B00F0C6804FF0020E88
:103CB000C346039C002C40F0BE801A8B598D5207DE
:103CC00017D5481E002900F01181DF6A07EBC107F4
:103CD00001E001380DD317F8072C083F12F0020F4E
:103CE00040F0E780002CF4D1012A08BF3C4601389F
:103CF000F1D24FF000025A84002940D00022A84699
:103D00000DE0C15D02D9012900F0C380032915D05F
:103D10006178CD0712D4598D01328A4216DA93F8B0
:103D200000C0D700D86ABCF1010F00EBC204E8D193
:103D300065680A2DF0D0C15D0329E9D1598C0132A3
:103D4000481C58846180598D8A42E8DB4546B1B1F0
:103D5000002202E001328A4211DAD86A10F83240B9
:103D600000EBC200042CF5D14478E407F2D4598C5E
:103D700001324180481C598D58848A42EDDB5F68CE
:103D8000002F54D07A8D002A51D00024A44604E09C
:103D90000CF1010C7A8D944528DAF86A10F83C2071
:103DA00000EBCC08043A012AF2D80029F0D0002216
:103DB000A94602E001328A4211DAD86A10F832705C
:103DC00000EBC200052FF5D14768D8F80450BD427A
:103DD000F0D144800132598D01348A42EDDB5F68B5
:103DE0000CF1010C4D467A8D9445D6DBFCB11FFADF
:103DF00084F9A9B1002206E061880132494461805A
:103E0000598D8A420CDAD86A00EBC20410F83200ED
:103E10000528F1D16078C007EED401328A42F2DB86
:103E20009A8B598C4A4489449A83A3F822909B68C0
:103E3000002B7FF43EAF5C462946304600F0BCF8CC
:103E4000099D039B65B13BBB0222294601A80B9645
:103E5000FFF750FB039B002B38D0AD68002DF2D14B
:103E6000D3B9304600F0B2F85046FDF7CDF82569D9
:103E70002046A468FDF7FEF8002CF9D1039800282D
:103E800038D12246214628460DB0BDE8F04F01F05A
:103E900079BB00F807E03BE70A9B01A8D968FDF76A
:103EA00069FB0A9B049ADB8A0199039806F038F8AB
:103EB000D7E7002C3FF41DAF97E80300D4E9008258
:103EC00084E80300C7E90082598D12E703222946DE
:103ED00001A8FFF70FFB039B002BBED1042229464C
:103EE0000DEB0200FFF706FB039BB6E75C8446E799
:103EF0004546A1E7F8F7B0FA10B504460122FDF7F0
:103F0000C3F82378012B02D90378012B00D010BD10
:103F10000323037010BD00BF70B506460D46104662
:103F200019461C46FDF7E2F80378012B14D0022B4A
:103F30000BD02D68032B428821463046AC460CBF7F
:103F400000230123BDE8704060476B68214630467E
:103F50000122BDE8704018476B68214630460022B8
:103F6000BDE87040184700BF42790346032A026A41
:103F700002D8114419627047006B11441044196251
:103F8000704700BF10B442790346032A05D8826AFD
:103F9000114499625DF8044B7047D0E90924006B25
:103FA00021442244996210445DF8044B704700BFDD
:103FB00000214820F8F792BA0B46002110B50446BC
:103FC0009800A361F8F76EFAE06110BD10B50446E1
:103FD000C069F8F793FA2046BDE81040F8F78EBAAA
:103FE0002DE9F04F0023914683B00122417105462F
:103FF000836083714261836203620191C0E903932C
:10400000B9F82430B9F82210B9F826601944B9F883
:104010001870B400B9F81E309142B9F820A004F02D
:10402000040407F01F0738BF1146B9F81C2043EA03
:104030000A0001394FEA920802F0030238434FEABE
:10404000111B1443CA0002F07802144348EA5602D6
:104050007608104350EA111235D00121284600930A
:10406000FFF782FFB90164F07F044FEA0B1C009B4D
:1040700001F0400104700CF0300CD800740041EAEB
:104080000C010AF0010C4FEA9B0B00F0080041EA1A
:104090000C0176087F0804F0020408434BEA06018D
:1040A0004FEA880C39434FEA58085B080CF0040CBF
:1040B00041EA08014FEA5A0A40EA0C001943044356
:1040C00051EA0A02C9D101212846FFF74DFF019BA1
:1040D0000470022B1AD9D5E90D230121284602FAD2
:1040E00001F403EA01069209CB4004F07E04C5E91D
:1040F0000D233443134318BF44F08004FFF734FF0B
:104100000470D5E90D2353EA0201E6D12B6A02219E
:1041100028466B63B9F81640FFF726FF02210470AA
:10412000240A44702846B9F81440FFF71DFF019B8C
:104130000470240A042B44704FF00004AC87A5F8E7
:10414000404002D003B0BDE8F08FB9F81C30B9F898
:104150001E20D342F6D0B9F82A0068B1D9F82C3025
:1041600000215A780131D20702D55A88A24212D0D2
:10417000814203F10803F4D156236A6C42F82430DB
:104180000134B9F81C30B9F81E201344A342E2DC14
:1041900003B0BDE8F08F5B681B0143F00603ECE75A
:1041A00070B543790546012B2CD000240121FFF77F
:1041B000DBFE04706A6B2B6AE8689B1AAC636B6366
:1041C000438D1BB917E0438DA34214D9C36A13F87A
:1041D000342003EBC4030134042AF4D19E78012176
:1041E0002846FFF7C1FE0670AB6BE8680133AB638E
:1041F000438DA342EAD86B79AA8F032BEA870AD0B2
:10420000042B00D070BD038B6A6C296B0069BDE87C
:10421000704001F0AFB92A6A0021AB6A6A62D01817
:10422000EB62F8F75BF9EB682863D98B988BAA8F60
:104230000844B5F840300021104418448000F8F7D5
:104240004DF9686470BD00BF8079003818BF012047
:10425000704700BF4379012B09D0D0E902231144F4
:1042600081609A8C9142C8BF998400238371704702
:1042700010B51446FFF7EEFF0121FFF783FE04702F
:1042800010BD00BF2DE9F04182B080461D46FFF70A
:10429000EFFF0DF105010F4605F07F04ED093E46E5
:1042A00007F8014DF8D1C91B4046FFF76BFE01A985
:1042B0008F420CD03346024601E013F8014B64F004
:1042C0007F048B4202F8014BF7D1DB1B18449DF8A9
:1042D0000430037002B0BDE8F08100BFF0B5C468DF
:1042E0001F46C68FB4F81CC0E48BB0F840E0A4446D
:1042F0004579B444042D0EEB0C030EF1010EA0F829
:1043000040E002D1446C44F82370BDE8F040FFF770
:10431000B9BF00BF9C46002113460CF1280C5FFA80
:104320008CF2FFF7AFBF00BF30B4DDE9024565B1E5
:1043300003EB440C013243EA04230CF1020CD2B229
:10434000A1EB0C0130BCFFF79DBF03EB440CD2B2D4
:1043500043EA0423A1EB0C0130BCFFF793BF00BF7D
:1043600000B5864643B90F2A06D8503A01215DF8B8
:1043700004EBD2B2FFF77CBF03F1240C7046134666
:1043800001215FFA8CF25DF804EBFFF77BBF00BF01
:1043900000B586464BB90F2A07D8403A4FF0FF3197
:1043A0005DF804EBD2B2FFF763BF03F1260C704651
:1043B00013464FF0FF315FFA8CF25DF804EBFFF724
:1043C00061BF00BF38B51C461546FFF743FF032108
:1043D000FFF7D8FD0570230A4470837038BD00BF15
:1043E00011320B460121D2B2FFF7ECBF16320B4659
:1043F0004FF0FF31D2B2FFF7E5BF00BF19320B46D5
:104400000021D2B2FFF7DEBFF8B51C461646FFF713
:1044100021FF43790546032B12D9C369826A53F8F9
:10442000243047F6FD74A41A1C44E7B2C4F30724F1
:1044300003212846FFF7A6FD067047708470F8BD7B
:1044400000242746F4E700BFF8B51C461646FFF7E0
:1044500001FF43790546032B12D9C369826A53F8D9
:1044600024306FF00204A41A1C44E7B2C4F30724FA
:1044700003212846FFF786FD067047708470F8BD5B
:1044800000242746F4E700BF2C4B2DE9F047D3F872
:10449000143181460F46022B02D844698C4201D365
:1044A000BDE8F087856A0C1B036940F2FF78ED1ABE
:1044B000062C24D9444526464FF00201484628BF21
:1044C00046460F2D94BF4FF0000A4FF0010ABAF193
:1044D000000F14D1FFF748FDA41B46703609234690
:1044E00006F070062E43554666F07F060670002BD8
:1044F000DED1D9F82830C9E90437BDE8F0871F2D8F
:10450000AA464FF0000628BF4FF01F0AAA4506D35F
:10451000032C264628BF0326A41B7601F6B2A5EB82
:104520000A050121484646EA0A06FFF71DFD44EA4E
:1045300005030670002BBBD1DBE700BF00040020A1
:1045400038B50D460021FFF785FE4379032B05D8CA
:10455000012B03D0826AC36943F8252038BD00BF10
:10456000012A84460B460DD0022A04D169224FF05D
:10457000FF31FFF77DBE1B324FF0FF316046D2B2F4
:10458000FFF720BF11461B326046D2B2FFF71ABFB9
:104590000E29844605D001F141020121D2B2FFF774
:1045A00067BEC168838F8A8B4079C98B04280A440F
:1045B00003F101011344ACF83C1004D1DCF84420B1
:1045C000034942F82310232201216046FFF75ABE17
:1045D00064DC066001F110033F2B70B50C4682B01D
:1045E000064608D8A1F180020121D2B202B0BDE88E
:1045F0007040FFF73DBE01212222FFF739FE0DF189
:1046000005010D4604F07F03E2B2E411AC4605F863
:10461000013D631C012BF5D8013419D053061FD47A
:1046200001AC491B3046FFF7ADFCA5420BD001465B
:104630002A4612F8013B63F07F03A24201F8013BD6
:10464000F7D1521B10449DF80430037002B070BDC6
:104650005206E5D47F2305F8013CACF10205DFE703
:10466000002305F8013CACF10205D9E70B46102206
:104670000121FFF7A7BE00BFC268938BD28B1A44FB
:10468000838F03F1010C13444279A0F83CC0042A43
:1046900002D1426C42F8231023220121FFF7F2BD20
:1046A00053220121FFF7E4BD002A0B464FEA4201E5
:1046B00014BF15221422C1F10101FFF783BE00BF10
:1046C00054220121FFF7D4BD10B5044649B1022997
:1046D0000ED0204656226FF00201BDE81040FFF7D1
:1046E000C7BD55224FF0FF31BDE81040FFF7C0BDF8
:1046F00053220121FFF7BCFD5B2200212046FFF77A
:10470000B7FDE6E710B50B4682B00446114652B13C
:10471000022A0ED018226FF00101204602B0BDE837
:104720001040FFF74FBE132202B0BDE81040FFF764
:1047300049BE532201210193FFF79AFD5A2200211D
:104740002046FFF795FD019BE4E700BF57220121BA
:10475000FFF78EBD58220221FFF78ABD59224FF084
:10476000FF31FFF785BD00BF5A220021FFF780BD52
:104770005B220021FFF77CBD0B4642220021FFF7A0
:1047800043BE00BF134621B143224FF0FF31FFF774
:104790003BBE44224FF0FF31FFF736BE134621B136
:1047A00045224FF0FF31FFF72FBE46224FF0FF3179
:1047B000FFF72ABE2DE9F04105460C461646C2B960
:1047C0000B0408D424F40043284642220021BDE80B
:1047D000F041FFF719BE592703260121FFF7D2FB4D
:1047E000077001212846FFF7CDFB013E0770F8D185
:1047F000E8E721F4004340220021FFF705FE0121F4
:10480000230A284623F07F0343EA0604FFF7BAFB96
:10481000E4B20470BDE8F081002A0B4602F14702C1
:104820000CBF02210021D2B2FFF70EBE38B50446FC
:104830000D4651220121FFF71BFD20462946FFF7B7
:104840007FFE02215C22FFF713FD20466FF003017B
:10485000BDE83840FFF7FEBC5D224FF0FF31FFF7A7
:1048600007BD00BF002915BF5F225E220321002182
:10487000FFF7FEBC0B464B220121FFF7E5BD00BF51
:104880006FF00301FFF7E6BC0B464A220021FFF759
:10489000DBBD00BF0A460021303AD2B2FFF7E8BCC8
:1048A000322910B5044616D0332908D0A1F12902C7
:1048B0004FF0FF31D2B2BDE81040FFF7D9BCDE2285
:1048C0004FF0FF31FFF7D4FC2046D3220021BDE892
:1048D0001040FFF7CDBCDD224FF0FF31FFF7C8FCE1
:1048E000F2E700BF022A02F12A020B46D2B214BF3D
:1048F000C1F101010121FFF7C5BC00BF62226FF0C9
:104900000101FFF7B5BC00BF032912D0042907D06D
:1049100002234FF0FF3143EA82032F22FFF7B2BC9C
:10492000013201236FF0010143EA82032F22FFF7D6
:10493000A9BC00234FF0FF3143EA82032F22FFF787
:10494000A1BC00BF0B4630220139FFF79BBC00BF62
:104950009446312241EA0C236144FFF793BC00BF27
:1049600013430B6903D132220121FFF7B7BC332275
:104970004FF0FF31FFF7B2BC38B51446049A054634
:1049800013430B690AD12022C4F10101FFF7A6FCF1
:1049900001212846FFF7F6FA047038BD2122E143D1
:1049A000F4E700BF30B5154683B01C4634220B46F1
:1049B0000021CDE90054FFF7B7FC03B030BD00BFC4
:1049C00030B5154683B01C4636220B464FF0FF31FA
:1049D000CDE90054FFF7A8FC03B030BD10B5632249
:1049E0004FF0FF310446FFF743FC0123A37110BDD4
:1049F00001F164024942D2B2FFF73ABC01F1670209
:104A0000494210B50446D2B2FFF732FCE268138B7C
:104A100043F00103138310BD0421FFF71BBC00BF4B
:104A20006FF00201FFF716BC2DE9F04F062983B0A5
:104A300006469DF8300040F2DC80B4EE400AF1EE0C
:104A400010FA80F1D08010EE104A002C80F2CB805A
:104A5000B1EE400A34462D204D1E04F8010BF0EE55
:104A6000C07A9FEDC47A02F02007F4EE477AF1EEA7
:104A700010FA00F31082B4EE400AF1EE10FA80F161
:104A8000BB82002B05F1FF3C42F02009C0F2C3803D
:104A900047F045020192A9F16702B2FA82F2520987
:104AA000002B14BF4FF0000802F00108B8F1000F0E
:104AB00000F06F8210EE103A1A1E40F03881BCF1FF
:104AC000060F00F32682EB1F4FF067094FF0000C32
:104AD00023EAE37E6746CDF800C0B9F1670F40F0E6
:104AE0003A82002B40F31982BEF1000F4FF000050F
:104AF0004FF06709D4BF4FF0000A4FF0010A0AEAED
:104B00000808BCF1000F12DA9B4BF7EE007A202266
:104B100003F1180017424FEA620203D093ED007AC6
:104B200067EE877A04338342F4D120EE270ABEF180
:104B3000000FC0F27481BCF1000FB2EE046AF7EE10
:104B4000007A05F1FF350EF1FF3EDFED8C6A4FF084
:104B50002E0B504631DCB0EE667A0023B4EEC07AFC
:104B6000F1EE10FA04D8013330EE670A092BF5D1C3
:104B7000BEF1FF3F00F0298103F1300222706A1C70
:104B800040F02181002800F01E8184F801B0023439
:104B9000BCF1000F05F1FF350CF1FF3C0EF1FF32C7
:104BA000D8BF20EE060ABEF1FF3F00F00E81BCF137
:104BB000000FF7EE007A9646CDDD6F4B202203F111
:104BC000180A1CEA020F4FEA620203D093ED007A42
:104BD00067EE877A04335345F3D117EE903A023BE0
:104BE00007EE103AB9E798B134464D1E04F8010BB0
:104BF00035E7012940F24B813F2306F8013B0023B2
:104C00003370012994BF0020012003B0BDE8F08F6C
:104C10000D46344623E7A9F1670847F04503B8FA83
:104C200088F8019306234FEA581810EE102A002A3C
:104C300000F08680B2F17E5F31D2514AF0EE407AC8
:104C40009FED507A2020DFF830E1002702F1140AAE
:104C500001E0B2EC017AB4EEE77AF1EE10FA04DD8D
:104C60009EED007A074467EE877A92454FEA60002E
:104C70000EF1040EEDD117EE902AB2F17E5F80F0B6
:104C800022819FED417AF4EEC77AF1EE10FAC0F27C
:104C90004B81002F14BF2D222B22009215E13B4A9D
:104CA000B7EE007ADFED3A7A4FF0200E002702F1DE
:104CB000140001E0F2EC017A67EE877A17EE90AA11
:104CC000AAF1020A06EE90AAB4EEE60AF1EE10FA94
:104CD00002DBB0EE677A774482424FEA6E0EE9D18A
:104CE000B9F1660F00F05781B9F1650F52D0B9F1F3
:104CF000670F40F093811A1D624500DBAB1F9F4296
:104D000080F2A7817A1C9B1A002B07EB030ED4BFFD
:104D10004FF0000A4FF0010A08EA0A0800230EF1DA
:104D2000010EBC463D464FF066090093E9E6B2F13C
:104D30007E5F4FF067094FF00103FFF47EAFAEE7EF
:104D4000B9F1660F40F03D8103F1010EE64502DB4B
:104D5000EB1EA5F1020E002B4FF00003D4BF4FF065
:104D6000000A4FF0010A1D461F4608EA0A089C4641
:104D70000093DCE6FFFF7F7FB8C50660FEFF7F3F44
:104D8000A4C506601FB14F0AF8FF7F3FBCC506608F
:104D9000AEC59D74AA1F9A4240F3CA8023EAE37EFF
:104DA000BC462B230093BEF1000F4FF000050EF11F
:104DB000010E4FF06509D4BF4FF0000A4FF0010A11
:104DC0000AEA08089DE60134E2E6042B27DD621EAC
:104DD0004FF0300C104612F801392E2BA3F130059C
:104DE000F8D0092D67D8392B6AD1B04282F801C0BA
:104DF000F0D135466B782E2B03D1B9F1660F40F018
:104E0000B780631C9A1B8A4238BF1C46AC4204D947
:104E1000621B2946681C38F0B5FE31232B70B8F1AF
:104E2000000F0DD014F8012C302A05D1631E1C464A
:104E300013F8012D302AFAD02E2A08BF04F1FF34CE
:104E4000009BF3B1019A043404F8033CFB1704F807
:104E5000042C834A82FB0701C3EBA10382FB0321DD
:104E6000DA17C2EBA10202EB8202A3EB420203EBD0
:104E700083033032A7EB430304F8022C303304F8E9
:104E8000013C0023A01B237003B0BDE8F08F002974
:104E90003FF4B7AEB3E687F0490387F04E0287F0E0
:104EA00046002370E31CA07062700022981B1A70E9
:104EB00003B0BDE8F08F4378302BB0D1451C99E7A3
:104EC00001330370ABE72D220092B9F1660F09D0D0
:104ED000042F2FDCB8F1000F2CD0B9F1670F01D1EE
:104EE0007A1E134403F1010EE64502DBEB1EA5F129
:104EF000020E002B4FF000034FF06609D4BF4FF0B5
:104F0000000A4FF0010A1D469C4608EA0A08009371
:104F10000DE64FF067090123D8E54FF0010A00259F
:104F20004FF06709D646ECE52D2201370092CCE719
:104F3000EB1F33E7AA1F9A4222DCB9F1670F00F09A
:104F40008280A5F1070EB9F1650FC7F1000C2EEABA
:104F5000EE7E3FF428AFBEF1000F4FF0000ED4BF3D
:104F60004FF0000A4FF0010A754608EA0A08C8E542
:104F70002B7030236B70009B2D2B5FD0013745E7E2
:104F8000B9F1650FC7F1000C23EAE37E3FF40BAFE4
:104F9000A3E5904649E66745BFF6FCAE07EB030E76
:104FA0000EF10102624530DBACEB070CBCF1010FE6
:104FB000ACF102037FF4A8AE4FF00008BE46C24633
:104FC000ACE65A1D9445D8BFEB1FB9F1650F7FF4CD
:104FD0007DAD002723EAE37EBB424FF02B030EF1A9
:104FE000010EBC46D4BF4FF0000A4FF0010A3D4607
:104FF00000930AEA08089EE547F04E0287F0410058
:10500000E31C22706070A2704FE7002BD4BF4FF0FA
:10501000000A4FF0010A08EA0A087FE6002B4FF069
:1050200000054FF02B03BC46D4BF4FF0000A4FF0F1
:10503000010AAE46009308EA0A0862E5013F08BF8C
:105040002B230093E2E6C7F1000C22EAE27E13462E
:1050500047E52B2223EAE37EBC46009241E500BFF0
:10506000676666660129136809D933F0100190F864
:1050700000C009D1BCF1300F15D0082B19D0C3B92D
:105080000A23002013607047082B14D0022B10D184
:10509000BCF1300F0DD1437843F02003622B14BFD5
:1050A000002002207047407840F02000782815D07A
:1050B00063B100207047BCF1300FFAD1437843F060
:1050C00020036F2B14BF0020022070476F2809D0E7
:1050D0006228D5D10223184613607047102302209E
:1050E000136070470823022013607047044608B518
:1050F00031B1054A002302604A6C096804F010FFD0
:105100002046F7F7A9F900BF78CF06602DE9F04FE8
:1051100085B00646984647180192002A6AD1BE42D9
:1051200012D2344602E0A74226460DD0264614F895
:10513000010BF9F745F80028F5D1B74204D93378C7
:105140002B2B5FD02D2B5FD0B91B304601AAFFF768
:1051500089FF0644B74266D94FF0000B344600255C
:10516000A14614F8013BA3F1300ABAF1090F09D99D
:105170005F2B14D043F02003A3F16102192A11D848
:10518000A3F1570A019951450CD928460EF0F4FBBA
:10519000019B28BB05FB03A595EA450220D4A74245
:1051A000A146DDD8BBF1000F00D06D426D0045F087
:1051B0000105B14537D0B9450CD24C4602E0BC429E
:1051C000A14607D0A146013499F80000F8F7F8FF8E
:1051D0000028F4D14F4526D1284605B0BDE8F08F10
:1051E0005A46B91B03A8039606F0AEF8DDF80C90FA
:1051F0000546DEE74FF4137310460221242201F026
:10520000FFFE8CE726469FE7013601AAB91B304610
:10521000FFF728FF0644BE4202D24FF0010B9DE784
:10522000B1460125C5E70449019A044804F01CFE73
:105230004146FFF75BFF00BFD002076004D0066065
:105240002DE9F04F04469146984667182DED028BE4
:1052500083B0BC420E98019080F03C81264603E06A
:10526000B742344600F0C080344601362078F8F763
:10527000A7FF0028F4D1A74240F2538123782B2BBB
:1052800000F0E3802D2B00F022810546237843F0C7
:105290002002692A00F0ED806E2A00F005814FF0AF
:1052A000000EF2EE046ADFEDA78A26469FEDA67A8D
:1052B0007046F446724619E0022A00F08980F4EE46
:1052C000C78AF1EE10FA40F18B8007EE90AA012A0E
:1052D000F8EEE77AE8EEA67AF0EE678A00F0A880AA
:1052E00000228F4240F228810B780E46A3F1300A4B
:1052F000711CBAF1090FDFD9002A08BF2E2B0CBF91
:105300004FF0010A4FF0000A60D0022A04D043F0A7
:10531000200BBBF1650F4ED0B9F1000F05D043F063
:10532000200BBBF16A0F00F0E0805F2BD9D0BEF1FB
:10533000000F00F00581A0EB0C0010F1250F80F2AA
:10534000F98000F125032E30DFED807A082868EE21
:10535000A78A53D85B42B2EE040A00EE903AF8EE08
:10536000E00A35F033F988EE808A002D52D1A6424A
:1053700078D0BE420AD2344601E0BC4208D026466C
:1053800001343078F8F71CFF0028F6D1BE4269D10D
:10539000BAF1000F4ED1B8F1000F3ED118EE103A1D
:1053A00023F0030040F00200A0F1FF4003B0BDEC89
:1053B000028BBDE8F08F8F4253D973782B2B00F00E
:1053C00092802D2B00F0888002228DE7012288E751
:1053D0005F4B9C4585DC0CEB8C0C0AEB4C0C80E79E
:1053E000002AF3D101307CE700253E46DFED558AE7
:1053F0002B46AA4603F109000828ABD907EE903ADC
:10540000B2EE040AF8EEE70A35F0E0F828EE808AFA
:10541000002DACD0B1EE488AA9E7B0EE480ADFED26
:10542000490A03B0BDEC028BBDE8F04F03F028BD84
:10543000013856E7F0EE480A9FED420A03B0BDEC92
:10544000028BBDE8F04F03F01BBD05463446BE425B
:10545000FFF41CAF4FF0000ADFED3A8A26465346B0
:10546000CCE765D13B493C4804F00CFD0199FFF7BE
:105470003DFEA31C9F42F5D9637843F020036E2BB9
:10548000F0D1A37843F02003662BEBD1E31DE61C9B
:105490009F4204D9E37843F02003692B28D09FED85
:1054A0002F8A4FF0000A60E7A31C9F42DAD9637885
:1054B00043F02003612BD5D1A37843F020036E2B5A
:1054C000D0D19FED278AE61C4FF0000A4DE7344605
:1054D0000125BCE70025BDE7B11C4FF0010EB94224
:1054E000C0D00222FDE6B11CF9E7CA460E461EE70F
:1054F000237943F020036E2BD1D1637943F020034D
:10550000692BCCD1A37943F02003742BC7D1E37965
:105510009FED128A43F02003792B04D04FF0000A4C
:1055200023E7054696E704F108064FF0000A1CE75A
:105530000E46FCE603465DE70E464FF0000AF6E62F
:105540006044FAE600000000EC78AD60EA1C080256
:1055500064666606E002076004D006600000807F93
:105560000000C07F08B500210C20F6F7B7FF01232B
:10557000037008BD4FF0020C437080F800C0C0E912
:105580000112704710B5044608461146D4E90123BC
:1055900005F056F86178CB0700D410BDC1F30011B7
:1055A000BDE8104005F030B938B5154611F48072E9
:1055B0000C460CBF1146D5E90012FFF7E3FF620964
:1055C000E1B202F008022A44BDE8384003F0DCBA38
:1055D00070B505460C464AB18E18D5E900039847C8
:1055E000431C04D004F8010BB442F6D170BD01484D
:1055F00000F046FBA40F076008B58847431C00D0A5
:1056000008BD014800F03CFBA40F076070B5002600
:1056100005460C46D5E900039847421C0DD024B13D
:105620002368187023680133236000F07F0343EA86
:10563000C6160306EED4304670BD014800F020FBCC
:10564000A40F076070B50D4600210646FFF7DEFF88
:10565000002839D010F001011CD144082046F6F78B
:1056600021FF0346304622461E461946FFF7B0FF8B
:1056700021463046F7F77CFE04463046F6F73EFFFB
:105680002B882046013303F01F0305EB43022B80D8
:10569000548070BD2A88A2EB500000F01F0305EB78
:1056A00043019A424E88344614D3D21A013358002B
:1056B000811C29445200284438F064FA2B88204683
:1056C00005EB43056E8070BDD6E90001BDE8704072
:1056D000FFF792BF581CC3F11F0240005200811C0B
:1056E0002844294438F04EFA6B882A880421022085
:1056F000A5F84030DDE700BF2DE9F04F88468DB0BA
:1057000000210446FFF782FF00F003039A1C039276
:1057100043B1039B052B40F03E810DB0BDE8F04F37
:10572000FFF720BF4FEA9009002108AF4846F6F77F
:10573000B9FE0546394606902E4608902046FFF7EA
:1057400065FF39462046FFF761FF16F8013B2A4600
:10575000190603F0030540F133810021D0438E4642
:1057600006EB000C16F8013BC3F3801202FA0CF2B0
:105770004EEA020E03F0040202FA0CF21543C3F3E0
:10578000C0021B0602FA0CF241EA0201E8D40D4401
:10579000CDF81CE016F8013B190603F0010EC3F327
:1057A000450C11D50620002116F8013B013103F00C
:1057B00001028A404EEA020EC3F3450282400630DF
:1057C0004CEA020C1A06EFD4DDF820A0F444069B44
:1057D0004146204666449944FFF734FF8AF80000AA
:1057E000000A41468AF801002046FFF72BFF8AF89D
:1057F0000200000A8AF80300204608990431721A50
:105800000891FFF7E5FEB1450AD832E0022826D01C
:1058100051462046FFF7DCFE089E5644B14528D984
:1058200006F1010AD4E90001FFF7E6FE002230701C
:10583000394630460DF012FE089A012802F1FF3277
:105840000892E3D141462046FFF7FCFE7070000A43
:1058500006F1030AB070089A023A0892D8E7D4E930
:105860000001FFF7C9FE03060AF8010BF7D4089AF6
:10587000CEE700212046FFF7C9FE834600212046DF
:10588000FFF7C4FE04905844002128448000F6F736
:1058900009FE0590002D00F096800746002641463F
:1058A0002046FFF7CFFE01360001AE4240F0060071
:1058B00047F8040BF3D1059B03EB8606BBF1000F01
:1058C0003ED0B146002727E0FFF7A0FE0246504633
:1058D00011460292F7F792FE029A0A992046FFF7C4
:1058E00077FE732D48D0A5F16201B1FA81F1490923
:1058F0000B46002940D1692D47D0A5F163020091E4
:10590000B2FA82F2DDE909105209FFF799FC01377A
:1059100049F8040B5F4511D00DF1200AD4E90001CC
:10592000FFF76AFE054600212046EDB2652DCBD17A
:10593000013726485F4549F8040BEDD106EB870691
:10594000049B53B10025049F013541462046FFF7D3
:10595000D3FEBD4246F8040BF6D1FFF703FE039BCE
:105960000446022B04D1079BDDE90521FFF702FE67
:1059700020460DB0BDE8F08F154B51461548732DEC
:1059800018BF184607F060FDC1E70A22DDE90910DB
:10599000FFF7BCFBBBE700212046FFF737FE0021E5
:1059A00083462046FFF732FE0021049058440D46FE
:1059B00006918000F6F776FD0795064605907DE78F
:1059C00000230793E6E6059E78E700BF64DC0660E7
:1059D0003CDD0660A0DF066010B592B004220446EC
:1059E0006946FFF7F5FD9DF80030432B25D19DF862
:1059F0000130052B21D19DF8023003F00303022B67
:105A00001BD19DF803301F2B17D800212046FFF72C
:105A1000FDFD202811D89DF802309B0810D101A966
:105A20002046ADF80430FFF767FE0346A268206801
:105A30001C469047204612B010BD034800F03CF9C8
:105A4000024800F039F900BFB0F00660AC00076012
:105A500000B585B0014601A810F08AFB01A8FFF748
:105A6000BBFF05B05DF804FBF8B51E4C0025F7F749
:105A70002BFC1D4904F1540004F19406656204F006
:105A800047FA04F16C00194904F042FA04F1840069
:105A9000032104F1A407C4F8145103F0A1FE304619
:105AA000012103F09DFE4FF4AB724FF4BB71304601
:105AB00003F02EFF29463846C4F8C450C4E90666F0
:105AC00006F07AF81621384605F0D6FD40F6167134
:105AD000384605F0D1FD294604F1B400BDE8F84090
:105AE00006F06AB80004002044CE066008CF0660C5
:105AF000704700BF08B5074BD3F8C40040B100227F
:105B000040F60631043050F0A7FC08B1406808BDEB
:105B1000014808BD0004002034E506600101034B84
:105B200041F00601986903F027BF00BF0004002080
:105B30000101034B41F00601D86903F01DBF00BF0E
:105B40000004002070B506F03BFB82680546CAB130
:105B50000024EB68E60053F8340080B104280ED02E
:105B600008F072FB03785F2B08D0EB68985907F0B8
:105B7000E7FCEB683344596850F07AFCAA680134BA
:105B8000A242E6D870BD00BF08B519B104F07AF999
:105B9000F6F762FC04F00EF9F6F75EFC08B504F0C7
:105BA00017F9F6F759FC00BF0EB400B582B003AA8E
:105BB00052F8041B0192FFF7F1FF00BF70B50546D4
:105BC000114E00222C01F06944F0060404302146F5
:105BD00050F042FC08B1406870BDD6F8C43033B113
:105BE00002462146181D50F037FC0028F3D1002250
:105BF0002146064850F030FC0028ECD12A460449E2
:105C00000448FFF7D1FF00BF0004002074E60660DF
:105C1000E804076098CE066038B50A4B0446D3E91D
:105C200006539D4209D001010022281D41F00601C2
:105C300050F012FC08B1406838BD2046BDE838403D
:105C4000FFF7BCBF0004002008B50446F6F7BAFD14
:105C500018B104490448FFF797FF22460349024858
:105C6000FFF7A2FF4C0407607CCE06603404076097
:105C70000146024808B5FFF787FF00BF10CD066058
:105C80000146024808B5FFF77FFF00BF24CF06603A
:105C90000146024808B5FFF777FF00BF0CCE06604B
:105CA0000FB400B583B0034804AA52F8041B019254
:105CB000FFF774FF0CCE06600146024808B5FFF7F7
:105CC00063FF00BF04D006600FB400B583B0034883
:105CD00004AA52F8041B0192FFF760FF04D006608B
:105CE0000146024808B5FFF74FFF00BFCCCF066062
:105CF0000FB400B583B0034804AA52F8041B019204
:105D0000FFF74CFFCCCF0660032830B5054685B0C1
:105D10000C4659D0CA071ED406282BD13D4B0B4048
:105D2000062B64D08B0756D0204601F0FFFB01F014
:105D3000B7FF034618B1214606209847C0B9364B35
:105D40002046595D019101F0F1FB0346019933486A
:105D5000DA88FFF7CDFF4810082D24D8DFE805F0DA
:105D600007282323302307050700002820DB2046CF
:105D700005B030BD084601F0D9FB01F091FF0346A4
:105D800020B12146284698470028F1D1042D18D08B
:105D9000082DD4D1204601F0C9FB03465E222048DD
:105DA000D988FFF7A5FFC043400040F00100DFE7BE
:105DB000B0F1404F1FD04042400040F00100D7E713
:105DC00038B13E2005B030BD084650F061FB0028D8
:105DD000F7D01E20CCE7086801F06AFF114B834220
:105DE000A2D1606870B1400040F00100C0E708092E
:105DF00050F042FBF6E74FF0804005B0BDE8304080
:105E000005F000BA03A9204607F0B4FB0399F7F7A1
:105E100047FAE8E70F0080FFB0E30660780B076001
:105E200030FB0660E9E901602DE9F0410D461646B8
:105E30001F46044601F07AFB01F02AFF864638B17E
:105E40003B46324629462046F446BDE8F0416047CD
:105E5000204601F06BFB03460148D988FFF748FF55
:105E600010FC066000231A461946FFF7DDBF00BF8D
:105E70002DE9F041194C9AB00E460746E16907A892
:105E8000E261A2690391A3610492F6F7CDFA054697
:105E9000E8B93946324605A8D7F80080FAF738FE47
:105EA000B6FA86F2414605A85209FDF7B1FE2B4627
:105EB0002A462946FFF7B8FF0190F6F7ADFA039A94
:105EC0000198049BC4E906321AB0BDE8F081039A38
:105ED000049B0898C4E90632F6F7BEFA00040020D5
:105EE00000B583B00022019101AB0121FFF79CFFB7
:105EF00003B05DF804FB00BF10B5144682B0002269
:105F00006B46CDE900140221FFF78EFF02B010BDF1
:105F100013460A465968003918BF0121C1F1020C25
:105F20000144186803EB8C03FFF77EBFF0B50D4604
:105F300085B012F003011C4601901CD11668B3888D
:105F400013F020070ED05B0608D5244BEE689E4266
:105F500011D0234B9D4201D0002830D0C4E900204D
:105F600005B0F0BD1F4B9E4208D01F4B9E4208D08B
:105F70001E4B9E420FD0226005B0F0BD53682360D7
:105F8000FAE720B1009201F0D1FA009A0546536871
:105F9000C4E90035F0E7E968104B9942EBD00028DE
:105FA000E9D003A9104606F0BDF900680E2811D00B
:105FB00001AB3A460121FFF737FF2060DCE70C20F8
:105FC0000092F6F76FFA0A4B009AC0E9003582603A
:105FD0002060D1E70748FFF74BFE00BF550902607C
:105FE0001CD806603CE3066020E30660CCD806605F
:105FF000D8C50660240B076000232DE9F0410D464B
:1060000014460746C2E9003301F090FA0A2D06460D
:106010002ED0192D23D0304601F052FE034650B148
:1060200022462946384698476368042B01D0BDE8CC
:10603000F08100236360B0680028F8D029010430A3
:10604000002241F0060150F007FA0028EFD0234665
:10605000426831463846BDE8F041FFF767BF01F0BE
:106060006FFE0028D7D0044BC4E90037BDE8F081AB
:106070002060BDE8F08100BF04E6066070B51446FC
:1060800005460E46FFF7B8FF236803B170BDAB07A6
:1060900003D1094B2A689A4208D0284601F07EFABB
:1060A0003346024605490648FFF77EFD3346EA8837
:1060B00004490348FFF778FD74E306609CFE066020
:1060C00010CD0660B40A076000B583B06A46FFF7DA
:1060D000D5FFDDE9000109B102F0ECFC03B05DF889
:1060E00004FB00BFF0B595B005460E46174601A863
:1060F0001C46F6F799F960B10CB115B0F0BD029BE2
:10610000084918680AF02CFE0028F6D10298F6F724
:10611000A3F93A4631462846FFF76EFFF6F77CF9B9
:1061200015B0F0BD10CD06602DE9F04105460C46D6
:1061300017461E4629B1186801F0F8F96B688342CA
:1061400007D133463A462146A868BDE8F041FFF73B
:106150006BBE0148FFF7C4FDA4F90660F0B585B039
:106160000F461446054601F0E1F9064601F0A8FD88
:10617000034650B10421284602AA039402913946ED
:106180009847029B93BB05B0F0BDB06870B339016E
:106190001A46043041F0060150F05EF930B3406811
:1061A00010F0030622D10268134B9A421ED1EDB1C2
:1061B00001A906F0B7F8019BCDE902545CB1012BAF
:1061C00014D940680E2811D002AB32460221FFF7E5
:1061D0002BFE05B0F0BD032B08D180680E2805D03A
:1061E00002AB22460121FFF71FFECCE73A460349E6
:1061F0000348FFF7D9FC00BFCCD80660E8FB066077
:1062000010CD066010B5044603F03EFE28B92046C6
:1062100003F050FE68B1204610BD002320461A4608
:106220001946FFF701FE0446204603F043FE00280E
:10623000F1D103490348BDE8104003F023BE00BF7D
:1062400044FE0660CCCF0660F0B587B01D4606461A
:106250000C46174601F06AF9454B834255D001F0D0
:106260006FFD034660B10E2C0CD10022414C30462C
:10627000A26298472860002850D0012007B0F0BDE6
:106280000E2C30D0F4B9384601F050F93A490AF0F2
:1062900067FD002849D03046472103AAFFF7ACFE2E
:1062A000039B002B5AD13549384603F00BFE0028DA
:1062B0004DD03349334803F0E5FD034602202B60FF
:1062C00007B0F0BD03AA30468A210192FFF7D6FE3F
:1062D000019A002101200594FFF71AFE03460120D0
:1062E0002B6007B0F0BD03AA192130460192FFF7D9
:1062F00083FE039B019A002BE5D000210846FFF79F
:1063000007FE034601202B60B8E72B463A4621469C
:10631000304607B0BDE8F04004F084BAA36A002B11
:10632000CDD10E2218462A60A8E730469B2103AA49
:10633000FFF762FE039B002BB5D003AA2146012084
:106340000597FFF7E5FD034601202B6096E73846E9
:10635000FFF758FF034602202B608FE703AA214670
:106360002046FFF7D5FD034620462B6086E700BF99
:10637000B0D2066000040020B8CD06605CCF066095
:106380005C00076024CF066010B50001104C86B099
:106390000E2340F00600D4F8C44002930592019009
:1063A000CDE9033134B1002240F61641201D50F0F2
:1063B00053F828B901A905200BF0F6FE06B010BD70
:1063C00001AB002205214068FFF72EFD06B010BD8D
:1063D00000040020F0B587B004460E4604AAFFF77B
:1063E0000BFE059B002B40D1049808B107B0F0BD0F
:1063F00020460CF04DF8002837D004AA204617217B
:10640000FFF7FAFD03A9049807F03AFF014630466A
:106410000191F7F77DF8039B01331D182846F6F725
:1064200015FF0199039A044637F07CFB039B2E224B
:106430003046E254039B0133E718F7F773F801463F
:1064400030460191F7F764F801990246384637F073
:1064500069FB29462046F6F78BFF064B01223E21B9
:106460001C61FFF791FF07B0F0BD324602490348B7
:10647000FFF79AFB0004002068FC0660D4CD06609C
:1064800070B582B00C46064601F050F801F050FCA1
:106490001C4B0546984223D030B19CB12146304672
:1064A000A84708B102B070BD0F2130466A46FFF719
:1064B000A3FD009BEBB1B4B12146684604F0B4FAE9
:1064C00002B070BD104B9842E8D021461020F5F77D
:1064D000E9FF044630462146A8470028E2D1E3E719
:1064E000304602B070BD21461020F5F7DBFF0446B0
:1064F000E2E7304601F01AF803460448D988FFF76E
:10650000F7FB00BF217C016005000260DCFC066037
:1065100030B583B0054601F009F801F011FC0446DE
:1065200040B10F4B002228469A62234603B0BDE8D3
:1065300030401847192128466A46FFF75DFD009B49
:1065400033B16A4621462046FFF7E2FC03B030BD76
:10655000284600F0EBFF03460248D988FFF7C8FB46
:106560000004002060FB066030B5054697B000F0DF
:1065700079FC284600F0DAFF01F0E2FB044640B166
:106580001A4B002228469A62234617B0BDE83040D5
:1065900018471921284601AAFFF72EFD019BE3B1F8
:1065A00003A8F5F741FF014668B1049B104918683C
:1065B0000AF0D6FB70B1049803F00EFB0B4B986207
:1065C000204617B030BD01AAFFF7A2FC0446F5F73C
:1065D00023FFF5E70498F5F73FFF284600F0A6FFF4
:1065E00003460448D988FFF783FB00BF000400205E
:1065F0005CCF066060FB06602DE9F04F2DED028B4D
:1066000013688BB008EE103A002860D102F1040B39
:106610008146C1F307235FFA81FA02930AEB430430
:106620005B0000930BEB8403D3F804805BF8243009
:10663000B8F1000F08D018F0030F05D1974AD8F829
:106640000010914200F0DF80009D002B00F0E680FA
:106650009A0706D11A6892498A423DD091498A42E6
:106660003AD00AF1040201931544A800F6F7EEFDB2
:10667000019B0646B9F1000F00F0C0800AF1010746
:1066800040F8049B4FEA8A090393874B59464A46D0
:10669000AA46019337F046FA039B06A91846FFF76E
:1066A000EFFE044602E046F8275001372046FFF788
:1066B0005BFF054600283AD0BA45F4D8019B4FEA63
:1066C000CA004FEA4A0A1E61F6F7C0FDEBE702F185
:1066D000080BD2F804909CE7184606AA05A901F019
:1066E0004DF9059B013353441D44A800F6F7AEFD58
:1066F0000646B9F1000F00F083800AF1010401277A
:1067000040F8049B4FEA8A09674B59464A46019371
:1067100037F008FA059A06EB84000699920037F0E4
:1067200001FA059B53441F44009BDC1902E0009BC7
:106730005546DC19029B0BEB090106EB8700DA00DA
:1067400037F0F0F9B8F1000F49D018F0030104D187
:10675000524BD8F800209A4277D06A21404606AAC8
:10676000DFF848A1FFF78AFC002106AA0846FFF7D8
:10677000CFFB0021FFF784FEDDF804B081460097CF
:1067800018E007EA0A023846062A02D008F01EF985
:10679000074606AA0F214046FFF770FC06AA002113
:1067A00001200897FFF7B4FB46F82470331F02342A
:1067B00043F824004846FFF7D7FE621C074658B14D
:1067C0009542DED86D00CBF81060042D38BF04254B
:1067D000A800F6F73BFDD4E7009FE31B0093009B66
:1067E000394618EE100A5A083346FFF71DFB019B85
:1067F0001E610BB0BDEC028BBDE8F08F574641E740
:106800004F4654467EE74046019303F07DF8029BD5
:106810001D18019B6D00002B7FF41AAF0AF10107D0
:106820003D44A800F6F712FD0646B9F1000F32D03C
:10683000009B40F8049BDC194FEA8A091A4B594621
:106840004A46019337F06EF974E7D8F80820002A19
:10685000C5D00D46DFF85490D8F80C304FEAC50A81
:1068600053F83500013500EA090388B104280FD038
:10687000062B01D008F0AAF846F82400D8F80C300E
:1068800053445A68A300023433445A60D8F80820AD
:106890009542E1D3A1E75746CEE700BF8CCB066017
:1068A00050E2066024D50660000400200F0080FF3F
:1068B000830770B50C4686B0154606D103681F4A9B
:1068C00093421DD01E4A93421AD002A9FFF7D8FD69
:1068D0000023064601936CB13046FFF745FE28B30E
:1068E000019B6FEA030C0133A444A342019345F8D2
:1068F0002C00F1D33046FFF737FED8B906B070BD93
:1069000001A902AA01F03AF80199A1420FD311D8C6
:10691000002CF3D0029A043D02EB840454F8043DA9
:10692000A24245F8043FF9D106B070BD019905486F
:10693000FFF7CAF921460448FFF7C6F950E206609E
:1069400024D50660F4040760480A07608307F0B5A1
:10695000154685B0CFB2C1F3072406D103683C4A7F
:10696000934240D03B4A93423DD00021FFF788FD3F
:106970000023064601936FB13046FFF7F5FD00286E
:1069800061D0019BFA1A01332244BB42019345F8BE
:106990002200F1D30021084605F0CCF9074602E0B9
:1069A000384604F069FE3046FFF7DEFD0146002858
:1069B000F6D1BB68A34246D305EB840245F82470A8
:1069C00054B1D7E902311B1B0344013051F8233085
:1069D000844242F8043DF4D1B9683846091B05F0F9
:1069E000D7F905B0F0BD029001A903AA029800F002
:1069F000C5FF01993B198B4226D8DDF80CC054B174
:106A00000CEB81032A1FA3EB840653F8040D9E426E
:106A100042F8040FF9D1C81B0CEB8701001B05F0ED
:106A200089F945F82400BB004FB1039905EB8404B4
:106A30000B4453F8042D8B4244F8042FF9D1002362
:106A4000029305B0F0BD01990348FFF73DF900BF7F
:106A500050E2066024D50660F4040760014602484F
:106A600008B5FFF791F800BFD0CE066043000C4692
:106A70000648022143F0010300B583B06A46009343
:106A8000019403F09DF9F5F7E7FC00BFD0CE066056
:106A90000146024808B5FFF777F800BF64CD0660ED
:106AA0000146024808B5FFF76FF800BFB4CE066094
:106AB0000FB400B583B0034804AA52F8041B019236
:106AC000FFF76CF8B4CE06600FB400B583B003488E
:106AD00004AA52F8041B0192FFF760F8ECCE06609E
:106AE00000B583B00C460022012101AB019402F0F5
:106AF000F7FFF5F7B1FC00BF0146034808B509B13F
:106B0000FFF7EEFFFFF740F85CCF06600146034851
:106B1000490008B541F00101FFF7E2FFD0CE066061
:106B2000014808B5FFF7ACF8F403076002490348D1
:106B300008B5FFF729F800BF08FE066020D0066000
:106B400030B595B004460D4601A8F5F76DFC48B97F
:106B500029462046FFF7C4F90446F5F75DFC2046B8
:106B600015B030BD00240299024800F0E9FD20462E
:106B700015B030BDFCBC0660034B044903F1540260
:106B8000D9655A62704700BF000400201CE206600D
:106B900008B5054B5A6A1AB10022596A5A6200B9FF
:106BA00008BD0846F5F758FC0004002038B5034638
:106BB0000C46154699B1D2B111462046984748B1C6
:106BC0006368B3B1A368DD6044F00103A5602046AB
:106BD000EB6038BD6B68E3606C60E3680BB128461E
:106BE00038BD45F00103AC602846E36038BD084677
:106BF00038BD6560E8E700BF2DE9F04111F0010400
:106C00000B46064621D1A046DA68C3F80C8012F084
:106C100001070AD021461A463046FFF7C7FF04464F
:106C200000232046E360BDE8F081D5681946D760AF
:106C30003046FFF7BBFF214602463046FFF7B6FF5E
:106C4000EB070446ECD42B46DEE70023DB60FFDED7
:106C500009B1FFF7D1BF0846704700BF8A4284469A
:106C6000F8B50D462BD0D668E6B1344600E0E468AE
:106C7000E107FCD524F001046368934214D01F4659
:106C8000DB689342FBD100225968DA605A6029B16F
:106C90006046FFF7B1FF08B1F8600746F307FE60F2
:106CA00048BFA7602846F8BD516891B100236046EF
:106CB0005360D360FFF7A0FF07466060EEE75568BA
:106CC00000215160002DEDD02946BDE8F840FFF7C6
:106CD00093BF16F0010F4FF0000008BF314661600E
:106CE000D060DFE738B50D46044600212846F5F7A9
:106CF00021FF00232060C01AE360236118BF012038
:106D0000C4E9015338BD00BF0023C0E90033C0E926
:106D100003338360704700BF4068704710B48268D7
:106D200003467AB1C0681C68411C205C5C68D9606D
:106D3000A14204D2013A9A605DF8044B70470021E9
:106D4000D960F7E74FF0FF30F6E700BF10B5836872
:106D50000446012B09D9FFF7E1FF034620461C46F4
:106D6000FFF7DCFF40EA042010BD4FF0FF3010BDFC
:106D70000346D0E9012090420FD21A691868815465
:106D80001A69596801328A421A6101D300221A61D4
:106D90009A68002001329A6070474FF0FF307047C8
:106DA0000023C0E903338360704700BFD0E90120AE
:106DB000101A7047806870472DE9F84306469046E0
:106DC0008AB18F184C1EC1F10105013F01E0BC42A0
:106DD00009D005EB0409304614F8011FFFF7C8FF7E
:106DE0000028F4DAC8464046BDE8F8832DE9F843A8
:106DF0000646904682B14C1EC1F1010504EB020922
:106E000003E004F8013F4C4506D030462F19FFF748
:106E100085FF031EF5DAB8464046BDE8F88300BF9B
:106E200038B5D0E9013204460D469B1A012B08D92A
:106E3000090AFFF79DFF2046E9B2FFF799FF0020FE
:106E400038BD4FF0FF3038BD82B0024B01AA1A6046
:106E500002B0704700040020014B5860704700BF2B
:106E60000004002000B583B0054A01A9D2E9003230
:106E70005B1A9A4202D903B05DF804FBFFF750FE9B
:106E80000004002008B5C2F34F0C530C09B1D2071F
:106E90000DD5634504D0834211D884450AD308BD7B
:106EA0008342FCD0024619460748FEF721FF0748F7
:106EB000FEF716FF024661460548FEF719FF191A4C
:106EC0000448FEF715FF00BF0C00076060FF066076
:106ED0006CFF0660B0FF06602DE9F04F804683B07E
:106EE0008A4693461F46002B4FD000240D9E0C9DD2
:106EF000A146019411E06B889A0549D4DBB209F1EF
:106F000001095AF82400012B1DD0022B39D0306022
:106F1000013404360835A7421FD0A045EBD8BBF199
:106F2000000F28D0298800225846090141F00601A7
:106F30004FF092FAF8B1019B4068013301936B88DE
:106F4000DBB2012BE1D101344FF0A2FA043606F88E
:106F5000040CA74205F10805DFD1C84518D8BBF1DC
:106F6000000F05D0DBF80030019AB2EB131F16D3E7
:106F700003B0BDE8F08F6B88DB050CD46B68336021
:106F8000C6E700F0FBFB3060C2E799460193E4E7F7
:106F90000448FEF7A5FE29880348FEF7A9FE03482A
:106FA000FEF79EFEA8FE066044FA066090FE0660AC
:106FB00030B589B00446154602EB800205A803935C
:106FC00000F038F90D9B20460C9C019305AA039B09
:106FD00029460094FFF780FF09B030BD014808B58D
:106FE000FFF75EFD3C030760884208B5134600DBEF
:106FF00008BD0A4601481946FEF766FE34F50660EC
:10700000884208B59E4602DB904200DC08BD13466C
:1070100002480A467146FEF757FE00BF30F306608D
:1070200010B50C4608B100F03BFCB5EEC00AF1EE1D
:1070300010FA00D910BD002221460148FEF744FE97
:1070400034F50660884208B59E4602D3904200D8C7
:1070500008BD134602480A467146FEF735FE00BFDA
:1070600014F10660884208B5134600D308BD0A46ED
:1070700001481946FEF728FEF4F10660884208B57B
:10708000134600D808BD0A4601481946FEF71CFE03
:1070900064F10660884208B5134600D108BD0A466F
:1070A00001481946FEF710FE58F00660884208B500
:1070B0009E4602DB904200DC08BD134602480A46A9
:1070C0007146FEF7EDFD00BF74F7066010B514467B
:1070D000820782B0034604D102688A4201D102B01D
:1070E00010BDCA881846019200F020FA019A214684
:1070F000C3880148FEF7FCFDD4F6066010B584078E
:1071000084B0034604D104688C4201D104B010BDA0
:107110001846CB880392029300F008FAC4887521C0
:1071200002480094DDE90232FEF7E2FDB4ED0660AC
:107130000E2830B5144685B004D0830704D1036807
:107140008B4201D105B030BDCA88039200F0EEF940
:10715000C5884FF4D573039A214602480095FEF77F
:10716000C7FD00BF24F606600B4B0340062B00B59D
:1071700083B005D0830706D1084B02689A4202D13A
:1071800003B05DF804FB019100F0D0F99722C388A9
:1071900001990348FEF7ACFD0F0080FFA0DF0660F9
:1071A000D4F6066030B583B00C46054601A900F060
:1071B00011FB10B1019803B030BD284600F0B6F9BC
:1071C0005E22C38821460148FEF792FDD4F6066090
:1071D0000146024808B5FEF777FD00BF28F10660BA
:1071E000094A0023014602F1420C03E0624505D042
:1071F00032F8023F8B42F9D31846704701EB510138
:1072000041F001031846704714C6066010B50B46DE
:10721000044641B9C0E90111236803F0080343F0B3
:107220000103236010BD0021D8006360F5F756F913
:10723000A060F1E70B01C0E90112026843F0070307
:1072400002F0080213430360704700BF10B50378D3
:1072500004469B0706D50022236862F31F13C4E986
:10726000003210BD8068F5F749F9F4E710B50378EE
:1072700004469B0709D52368002203F00C0343F062
:107280000103C4E90122236010BD8068F5F736F9D7
:10729000F1E700BF2DE9F04147680646781CFFF78B
:1072A0009FFF00210446C000D6F80880F5F716F9C4
:1072B0003368746003F00E03B06043F00103336081
:1072C0009FB108F10404002554F8041C013541B1B4
:1072D00004294FF00102304603D04FF0BDF8236877
:1072E0004360AF4204F10804EED14046BDE8F041EE
:1072F000F5F704B90B46002210B504461146980074
:10730000C4E90032F5F7EAF8A06010BD2DE9F04FAE
:1073100083B0134606468B46009202681AB9D90715
:1073200052D500F075F859460620FEF7EDFC009A9C
:1073300033684FEA600A02F001020192BAFBF3F2ED
:1073400003FB12A94C4600270BE000F05DFC00286F
:107350003FD133680134B4FBF3F103FB1144A14581
:1073600015D0B06859464FEA840850F8245000EB15
:10737000840E2846C5B1042DE7D10134002F08BF83
:107380007746B4FBF3F103FB1144A145E9D1019B1E
:10739000D3B1002F34D1304600F03AF83368BAFB4D
:1073A000F3F203FB12A9CDE7009BDA070CD5726854
:1073B000002F08BF77465D4601327260C7F800B003
:1073C000284603B0BDE8F08F0025284603B0BDE88D
:1073D000F08F009B9B07F3D573680134B268013BC3
:1073E00073603368B4FBF3F103FB114452F82430AB
:1073F00003B10423284642F8083003B0BDE8F08FFB
:1074000072685D4601327260C7F800B0D8E700BF0D
:107410002DE9F041076806460024D0F80880781C62
:10742000FFF7DEFE2146C6E900048000F5F756F8B6
:10743000B06077B1A8F1040555F8041F013431B1EB
:1074400004294FF00102304601D0FFF75FFFA74249
:10745000F2D14046BDE8F041F5F750B810B50168EB
:107460008646F9B184680023224601E08B4217D09A
:10747000944652F8040B01330028F7D00428F5D0C5
:10748000DEF80420013ACEF80420B3FBF1F201FB50
:10749000123354F8233003B10423CCF8003010BD6C
:1074A000002010BD084610BD10B504468068F5F7F1
:1074B00025F80023C4E90033A36010BD00B582683D
:1074C00053685FEA131C0FD0D268002302F1040E48
:1074D00001E09C4508D05EF833000133B0F9042088
:1074E0008A42F6D15DF804FB0E205DF804FB00BF74
:1074F00010B50C4601462046FFF7E8FDB4F904003C
:1075000010BD00BF13460246084610B582B01C6885
:10751000B3F90610E38800910249F6F7C5FD02B001
:1075200010BD00BF58C60660704700BFC20709D42F
:10753000830705D0074B0340062B05D0064870474C
:107540000068704705487047054BC0F3C10053F809
:1075500020007047070080FF7CD00660F4D30660EF
:1075600078C6066038B5044680680146FFF7DEFF3E
:10757000036A054605209847E168B1EB600F0ADA17
:107580004900AB6A0422A06841F001019847E36812
:107590000133E36038BD002038BD00BF08B5FFF7F8
:1075A000C5FFC088BDE80840F5F7BCBF2DE9F04134
:1075B00006460C461546FFF755FC4EF055FF3BF0CE
:1075C00019FE58B92046FFF7B1FF076947B12A46AF
:1075D000214630463B46BDE8F0411847BDE8F08102
:1075E000C28830460249BDE8F041F6F75DBD00BFF4
:1075F00064C6066003460A4601481946FFF7D6BF2F
:10760000C4EB06602DE9F04F044683B008460F46F0
:10761000154602F04FFC58B9394620460222FFF7C2
:10762000C5FF4049204603B0BDE8F04FF6F718B952
:1076300011F046F90028EFD0384602F0BFFAC668CC
:10764000002E66D0DFF8E89096F81580B8F1000FAC
:1076500049D001AA6946384602F0BAFC009B002BCB
:10766000DAD005EB4505A3F10308002D32DDAB426E
:107670002CBF5D1B00252C492046F6F73FFD4545F4
:10768000CADCDFF8B0A0DFF8B0B0DFF8989006E011
:107690002046F6F7E5F8A8F103084545BCDC88EA82
:1076A000E876019B51462046A6EBE87603EB860C74
:1076B00053F82620B600DCF80430F6F71FFD019BD6
:1076C000494633449A68002AE2D059462046F6F7E4
:1076D00015FDE0E7CFD06A424FF00008934238BF73
:1076E0005D420335C7E701232A46314620467375BC
:1076F000FFF788FF0B49204686F81580F6F7D4FC83
:1077000049462046F6F7FAFC08492046F6F7CCFC35
:107710009FE7037D002B9CD10669002E99D0DFF8EE
:107720001C9091E7D4BE076060F606606CC60660E8
:107730003CF506609CED06609006076098EE0660DA
:107740000022FFF75FBF00BF08B50146FFF7EEFE5E
:10775000838813F080030CD0C069074A904203D09D
:10776000003818BF012008BD0846BDE8084009F0F0
:10777000A9B9184608BD00BFB50802601E28014619
:1077800008B512D03E2812D0C2070CD4830703D10B
:10779000084B02689A4202D00820FEF7B5FABDE80D
:1077A000084003F0F1BD401008BD002008BD0120D5
:1077B00008BD00BFF4D30660C20707D4830703D116
:1077C000034B02689A4201D0FFF7D8BF03F0D4BD43
:1077D000F4D306601E2810B582B00FD03E2807D023
:1077E00010F0010210D043100B60104602B010BD23
:1077F00001231A460B60104602B010BD012200237F
:1078000010460B6002B010BD8407EED1054C036832
:10781000A342EAD1019103F0B7FD0199012208606A
:10782000E3E700BFF4D306601E28034610B582B01C
:1078300012D03E280DD010F0010210D0431000EEFF
:10784000103AB8EEC00A012281ED000A104602B0DB
:1078500010BDB7EE000AF6E79FED0E0AF3E710F051
:10786000030C08D10C4C0368A342EFD1019103F043
:10787000E1FE0199E7E7BCF1020FE7D107481840A4
:107880000628E3D003F1FF4323F0030300EE103A90
:10789000D9E700BF00000000F4D30660070080FFB6
:1078A00010B582B0044601A9FFF7BEFF18B19DEDE7
:1078B000010A02B010BD2046FFF738FE034640F231
:1078C0001D320248D988FEF713FA00BF30FB06606C
:1078D0001E28034670B50D46144618D03E280DD01C
:1078E00010F0010C1AD04310002207EE903AF8EE87
:1078F000E77AC1ED007A2260604670BD4FF07E529B
:1079000000234FF0010C0A606046236070BD002325
:107910004FF0010C0B606046136070BD10F0030E59
:107920000BD10368124EB34219D0124CA342E3D1DB
:1079300001F0BCFA4FF0010CDEE7BEF1020FDBD123
:107940000D4A0240062AD7D003F1FF4300224FF030
:10795000010C23F0030360462B60226070BD03F02E
:1079600069FE002385ED000A4FF0010C2360C3E798
:10797000F4D306609CC90660070080FF70B5164608
:107980000446FFF7D3FD83880D461A0603D5C26A65
:107990000E4B9A420CD0A30710D10D4B22689A428D
:1079A0000CD1324629462046BDE8704004F0E2B9C9
:1079B00032462046BDE8704008F020BA2046FFF766
:1079C000EDFD01460348FEF793F900BF31FA01606F
:1079D00024D506602006076070B582B005460C46C7
:1079E00001A9FFF7CBFF2846FFF7A0FD0346019E44
:1079F0002146DA883046FFF74DFB02B070BD00BF6C
:107A000070B51E46D30782B014460D4618D55010E7
:107A1000019000280BDB26B1A84218D8019802B0CB
:107A200070BD5C236A1E0021FFF740FBF6E7284487
:107A30000190002EF5D00028EEDA002002B070BDD3
:107A400001A91046FFF7C6FE20B10198E1E72846DC
:107A500002B070BD20465C21FFF768FD03465E2240
:107A60000148DB88FEF744F9D4F60660820707D1A7
:107A7000002803DB400040F00100704703F05ABCCF
:107A800003F0C0BB8307014610B503D10F4B02685A
:107A90009A420ED00846FFF749FD838813F0800311
:107AA00005D0036A1BB10520BDE8104018471846F1
:107AB00010BD074B0340062B04D08068430043F001
:107AC000010010BD0009F5F723FDF7E73CDD066076
:107AD0000F0080FF10B50446FFF7D4FF00B110BDC2
:107AE0002046FFF75BFD01460148FEF701F900BFA4
:107AF0003C06076005282DE9F84F15BF3E261E26D7
:107B00004FF01E094FF03E09914207460C461546BC
:107B100043D03B4B2340062B2BD0A10725D014F09C
:107B2000010843D0EB0745D44FF001082846FFF782
:107B3000FDFCB0F804A001461AF0800F0CD0D0F87C
:107B400024B0BBF1000F07D01AF0080F36D1204641
:107B5000FFF7ECFC814231D0B8F1000F4BD0A542C9
:107B600018BF4E463046BDE8F88F264B22689A4231
:107B7000D5D1234B2B40062B05D0AA07D4D1214BBE
:107B80002A689A42D0D12946204606F01DFB0028DB
:107B900008BF4E463046BDE8F88FCB07E2D4084612
:107BA000FFF7C4FC83885807DCD5B2E72B4625468F
:107BB0001C46BBE74E463046BDE8F88F052F0FD078
:107BC000224629460220D8470028C5D0022F01D1DD
:107BD0000646C7E74EF05CFC002808BF4E46C1E7EA
:107BE0001AF0100FECD0224629463846D847002814
:107BF000E6D00646B6E72B4625461C4694E700BF6E
:107C00000F0080FFA0DF066008B503460A46022089
:107C10001946FFF76FFFBDE808404EF039BC00BFC2
:107C2000704700BF10B4054A0023054CC1E90203A8
:107C3000C1E9004208465DF8044B70476575016074
:107C400070D8066038B504461546FFF76FFC838888
:107C500013F0800308D0436B33B12A46204698477F
:107C6000B0FA80F0400938BD184638BD08B5FFF7B6
:107C7000E9FF00B108BD0148FEF732F84806076089
:107C8000062803D1490041F00100704700207047E9
:107C9000838813F0800314BFC0691846704700BF83
:107CA000838813F0800314BF006A1846704700BF32
:107CB000838813F0800314BF406A1846704700BFE2
:107CC00040697047838813F0800314BF806A1846A8
:107CD000704700BF70B505461446FFF727FCFFF755
:107CE000F1FF034640B1224628469847064610F069
:107CF000F7FD0EB1304670BD28466CB1042C05D09E
:107D0000FFF74CFC01460748FDF7F2FFFFF746FC82
:107D100001460548FDF7ECFFFFF740FC014603482C
:107D2000FDF7E6FF94FD066034FF066018FE06606E
:107D3000838813F0800314BFC06A1846704700BFE1
:107D4000838813F0800314BF006B1846704700BF90
:107D5000838813F0800314BF806B1846704700BF00
:107D600080697047838813F0800F14BF3C201C206B
:107D7000704700BF042808D0052804D18868400057
:107D800040F001007047002070478B68002B14BF43
:107D90003E201E20704700BF00230B4A10B40B4C3E
:107DA000C1E90233C1E900400368934203D00846A9
:107DB0005DF8044B7047436808465DF8044BC3F315
:107DC00017238B60704700BF3CC80660C4C70660BD
:107DD000F8B50D4601790446164601F07F010022F0
:107DE000402009F0B3FDE7680F4A03462F60A16801
:107DF00000FB01F16960217901F07F01A960216830
:107E0000914201D00020F8BD94F90420002A03DB40
:107E1000B20701D50120F8BD62680020C2F3172225
:107E200003FB02732B60F8BD3CC806602DE9F047E8
:107E30000C4688B0054608681F469146FFF776FB5A
:107E4000012202A980462068FFF710FF012205A940
:107E50006068FFF70BFF00229DF81C10402009F01E
:107E600075FD012835D1022DDDE9026106EB010A1D
:107E700014D9A2680E2A04D003464046FFF7C0FD7D
:107E80000644032D0AD0E2680E2A07D0404601239B
:107E9000DDE90241FFF7B4FD04EB000AB24505D26B
:107EA000D7B94FF0FF3008B0BDE8F087069BAAEBCA
:107EB00006013046059ACDF8009005F07DFA0028BD
:107EC000EED0029BC01A400040F0010008B0BDE8AF
:107ED000F0870348FDF704FF0248FDF7EDFE00BF01
:107EE0006CF90660A409076000230122FFF79EBF1A
:107EF00000234FF0FF32FFF799BF00BF01231A465E
:107F0000FFF794BF01234FF0FF32FFF78FBF00BF91
:107F10007828F8B505460E461FD0002201464020BD
:107F200009F014FD002107461020F4F7BBFA0446BF
:107F30000B4B06FB07F0257100216268A6606FF30A
:107F40001F226260074A012D18BF13462360F4F711
:107F5000A9FA03462046E360F8BD0348FDF7ACFEEE
:107F600000C8066088C7066070FA0660012800B580
:107F700083B006D10A6840F6162369460220CDE98F
:107F800000230B4600220146024805F001FB03B026
:107F90005DF804FBA0DF066010B442680346C468C5
:107FA00091688C420BD21079D1689A6800F07F00FA
:107FB00022440134DC605DF8044B09F0DDBD002093
:107FC0005DF8044B704700BF70B5426882B004464C
:107FD0000B4632F0FF050ED02079D4E9022109F0DA
:107FE000B9FF0E20D4E901320132A3F58073C4E950
:107FF000013202B070BD2A4601910179402009F09A
:10800000A5FCA16862680646083100FB01F1082062
:1080100060F31F22E0686260F4F762FA6268294642
:10802000A568C2F31722E060013A06FB02F205FBE5
:108030000666304435F0BAFD019BCDE770B50D46BC
:1080400084B00446012201A92846FFF7FBFD08B3CE
:1080500000222179402009F079FC029D63680646E0
:10806000B5FBF0F5B5EB132FC3F3172224D8521B41
:10807000E06862F31F236360A36805FB06F20199C1
:1080800003FB060035F04EFDA3680E202B44A360D1
:1080900004B070BD01462846FEF7F2F9054601E03E
:1080A000FFF792FF2846FEF75FFA014620460029B7
:1080B000F6D10E2004B070BDD4E90210294406FBAD
:1080C00001F1F4F70DFA6368E0606FF31F2363605A
:1080D000D2E700BF2DE9F04104468CB00E461546AC
:1080E000242820D8DFE800F024242424241F1F1F84
:1080F0001F1F1F1F1F1F831F131F1F1F1F1F1F1F38
:108100001F1F1F571F131F1F1F1F1F1F900012F03D
:10811000010040F08A8012F0030304D1854A2968E7
:10812000914200F08280002420460CB0BDE8F0812E
:10813000012206A93046FFF74BFE012209A9284675
:10814000FFF780FD00286BD0089B012B00F0C0805A
:108150005A2B40F3A58023F002010020643918BF98
:1081600001210B9A012A00F0B6805A2A00F3B5804B
:108170002032934240F08A80002900F08780204618
:10818000DDE90935DDE90612009508F0A3FF0028B6
:1081900046D03E24C8E706A901223046FFF718FE64
:1081A00009A928460122FFF761FD00229DF8201051
:1081B000402009F0CBFB0A9B0546B1689DF82000E2
:1081C000B3FBF5F63144FFF7A3FE0446C068DDE9D2
:1081D000061235F0A7FCE068079B06FB05F209993B
:1081E000184435F09FFC20460CB0BDE8F081524B9E
:1081F0000A689A4297D0344629463046FFF71EFF58
:1082000020460CB0BDE8F081012203A92846FFF703
:1082100019FD90B3B20703D1484B32689A4246D059
:108220001E2420460CB0BDE8F0812846FFF7A6FAD0
:10823000012209A907463046FFF7CAFD102CDDF8D8
:10824000288055D0B1689DF82C0007FB01F1FFF79D
:108250005FFE0446C568B8F1000F3FF465AF7E1EAF
:10826000002F3FF461AF013E28460999424635F0A0
:1082700059FC711C4544F6D156E7EB0706D415F0BE
:10828000030306D12B4B2A689A42C9D10020FEF77E
:1082900007FC022BC4D12A4B2B40062BF6D1BFE79B
:1082A000203323F00201643918BF012159E701246A
:1082B000012209A93046FFF78BFD0094DDE9032375
:1082C000DDE9090105F078F800287FF462AFA7E73F
:1082D0000146622345E762224BE79A42D6D1002944
:1082E000D4D0022C3FF44BAF00287FF448AFCDE749
:1082F00000223179402009F029FBB36807FB03F322
:1083000000FB03F1F068F4F7EBF8B368054607FBF0
:1083100003F3C6E9023073686FF31F2373603FB144
:10832000013F45443446B8F1000F3FF4FDAE96E7F7
:108330003446F9E6F4D306603CC8066000C806601F
:10834000070080FFF8B50D790C460646012D32D0A6
:108350002A462049F5F7A8FEA3682BB930461E49E6
:10836000BDE8F840F5F77CBA1C493046F5F778FAD5
:10837000A368B3B100251A4F2A46E1682079013578
:1083800009F0FAFB012201463046FFF70FF9A36816
:10839000AB4206D9002DEFD039463046F5F760FAEA
:1083A000EAE710493046F5F75BFA30460A49BDE87E
:1083B000F840F5F755BA0C49F5F752FA30462B4616
:1083C000D4E9022104F014FF30460349BDE8F84027
:1083D000F5F746BA94C6066050DA0660A0C6066095
:1083E000A8C60660A4C6066088C6066001282DE9F6
:1083F000F041804684B00D4635D08B072CD02846FE
:10840000FFF740FB00284ED0441021464046FFF7BE
:108410007FFD002106462846FEF732F80025074674
:108420003846FEF7A1F848B164B901463046FFF777
:10843000CBFD3846FEF798F80028F5D1304604B059
:10844000BDE8F08105F1010C2A460346F16840467B
:10845000654609F07FFDE3E70B68154A934202D0B9
:10846000144A9342CBD1012201A92846FFF7EAFB27
:108470000028C4D041460022402009F067FA029B40
:10848000B3FBF0F100FB01F4A3420ED14046FFF72D
:108490003FFD064622460199C06835F043FB304651
:1084A00004B0BDE8F0810446AFE70348FDF704FCE3
:1084B0003CDD066000C80660E0FA066038B50C4690
:1084C0001D4611460A4A2046FEF7DCFC286805F0E6
:1084D000BBFE012C05D069680078BDE83840FFF785
:1084E00085BF00210078BDE83840FFF711BD00BF0F
:1084F0000400020030B50C4683B011460622204627
:108500001D46FEF7BFFC14B32868C20712D5012C24
:1085100024D1FFF733F90246204611460192FFF7B6
:10852000F7FC0446019A0021C06835F03FFB204665
:1085300003B030BD830703D10A4B02689A42E6D0EC
:108540000146012003B0BDE83040FFF74FBF214690
:10855000012003B0BDE83040FFF7DABC0248FDF768
:10856000BFFB00BFF4D306601C0C07602DE9F0438D
:108570008C4687B004461546002A34D011F0030615
:1085800003D1864B0A689A4232D000236246A16822
:108590002068FFF735FA824B2168024699420ED0D7
:1085A000042D11D094F804C02B46E1680CF07F0034
:1085B0000E2509F0CFFC284607B0BDE8F0836368BC
:1085C000042D00EB132208D12079E16800F07F0030
:1085D00007B0BDE8F04309F0CFBA94F9043094F83D
:1085E00004C0002BE0DB0025284607B0BDE8F0837F
:1085F0006A46806808F020FD002800F0C8802179D4
:10860000042D32464FF0400001F07F016CD009F09C
:108610009DF915F00307064602D06248FEF740FABE
:108620002868FFF74FFB604B834200F09A805F4B56
:108630002A689A42F1D1012E40F0AC80324603A95B
:108640002846FFF713FB564ADDE90398DDE90001F0
:1086500023680F1AE5689342A8EB070724D0002F80
:108660002DDD6368B7EB132F58D8A368404406FB91
:1086700001513B441A1A06FB005006FB02F235F08A
:1086800081FA009806FB08F2494600FB065035F0D7
:1086900079FA63680E25C7EB132262F31F23A268E1
:1086A0003A44C4E9013286E794F90430002B9ADA9F
:1086B000002F6FD16368C3F3172306FB03554946A8
:1086C00006FB08F206FB005035F05CFA0199A2683F
:1086D0000098521A06FB0151404406FB02F206FBC9
:1086E000005035F04FFAD4E709F030F92C4B2268EE
:1086F00007469A4222D02079DDE90031C91AFFF7F6
:1087000007FCE1680546C068DDE900239B1A07FB0A
:10871000021107FB03F235F005FA4CE7A168284681
:10872000394406FB01F1F3F7DBFE63680546E060C0
:1087300067F31F236360DDE9000196E731461020EF
:10874000F3F7B0FE054694E80F0085E80F00009AA5
:1087500002EB112060F31F216960019B9B1AAB6043
:1087600029E729793A46402001F07F0109F0EEF827
:10877000B0420FD10A4A2B689342D5E902897FF4AF
:1087800065AF6B68C3F3172306FB03995EE70848E0
:10879000FEF786F90748FDF78FFA00BFB0DC0660E8
:1087A0003CC80660D8F906606D8501603CDD066056
:1087B000980607607C03076070B506460D461020DA
:1087C00000211446F3F76EFE067142686FF31F2214
:1087D0004260024AC0E90254026070BD3CC80660B3
:1087E00070B51C4684B0084611464FF00212FEF7E1
:1087F00049FB012201A92068FFF738FA9DF80C50C7
:10880000029E00222946402009F0A0F8019AB6FBFA
:10881000F0F12846FFF7D0FF05462068FEF786FEF8
:108820000D4B83420CD0032201A92068FFF70AFAFE
:1088300018B12B7963F07F032B71284604B070BD0B
:10884000226869685368C3F3172363F31F216960C3
:10885000D368EB60E7E700BF3CC80660F8B50546A3
:10886000084605F0F1FC074600224020397809F05F
:108870006DF82979AC68064601F07F01002240209E
:1088800009F064F800FB04F3B3FBF6F106FB1133C7
:108890006BB9EA683878FFF78FFF95F90430002B41
:1088A00000DBF8BD037963F07F030371F8BD014875
:1088B000FDF716FA640407600246012010B50C4665
:1088C00082B011460192FFF723FB21460446019A2C
:1088D000C06835F027F9204602B010BD02460120DD
:1088E00010B582B011460192FFF712FB0446019ABF
:1088F0000021C06835F05AF9204602B010BD00BF13
:1089000038B505460C4610200021F3F7CBFD034A8D
:1089100002600122C0E90254426038BD00C806600E
:10892000136830B40BB130BC70474568AC1C50F8CC
:108930002440002DF7D0A4F1040C02E001339D4245
:10894000F1D05CF8044FA142F8D1023350F8233043
:1089500030BC1360704700BF2DE9F04790460E46CB
:1089600015490446F4F77CFFD8F80430EBB1043E17
:1089700008F104070025DFF848A0DFF8489001E07F
:10898000F4F76EFF56F8042F514620460135F5F7EF
:108990008BFB57F8041F20460122FEF707FED8F88C
:1089A000043049462046AB42EAD820460349BDE898
:1089B000F047F4F755BF00BF0C3A086050DA066084
:1089C00078C80660A8C606604B680A46023351F8AC
:1089D0002310FFF7C1BF00BF1E3918BF0121490096
:1089E00041F001014DF058BD052807D01E3918BFD0
:1089F0000121490041F00101FDF786B900207047CF
:108A0000032A04D01E2907D00649F4F729BF1E29DE
:108A100005D00549F4F724BF0449F4F721BF044900
:108A2000F4F71EBFC4780660E8BC0660ACBD066003
:108A3000F0BC066038B50C46114602221D462046A1
:108A4000FEF720FA0CB91E2038BD28684DF020FD35
:108A50000028F8D03E2038BD2DE9F04102EB430458
:108A6000884607461E4601341546A4002046F4F702
:108A7000EDFB221F0446069940F8048B35F052F8AE
:108A800023463246691C3846FDF7CEF9014B1C617E
:108A9000BDE8F0810004002010B5944682B01C4669
:108AA0000A4663460094D0E90101FFF7D5FF02B002
:108AB00010BD00BF38B505460C460C200021F3F769
:108AC000F1FC024A8460C0E9002538BDF4C80660A4
:108AD000406870474160704710B500210446082087
:108AE000F3F7E0FC014AC0E9002410BD30C906607C
:108AF0002DE9F04715468268044686B002EB010A6C
:108B00000E4699466F000AEB450005281AD84FEA31
:108B1000820804F10C0101A8424635F003F801ABCC
:108B2000BA19494603EB0800920034F0FBFF01AB91
:108B30002A4651466068FDF777F90446204606B09C
:108B4000BDE8F08700218000F3F7ACFCA26804F1D7
:108B50000C018046920034F0E5FFA068BA1949463E
:108B600008EB8000920034F0DDFFA1682A464346FE
:108B700031446068FDF758F904464046F3F7BEFCFF
:108B8000204606B0BDE8F087F8B50D460646002140
:108B90001746EC1CA4002046F3F784FCA4F10C0259
:108BA000054B044646603946A5600C30236034F01E
:108BB000B9FF2046F8BD00BF4CC9066030B591ED45
:108BC000010A87B00C460546B5EE400AF1EE10FAF0
:108BD00010D191ED020A002106236722009102A81C
:108BE0001021FBF721FF02AA1A492846F5F75CFA83
:108BF00007B030BD00220623102102A80092672290
:108C0000FBF712FF02AA14492846F5F74DFA94ED36
:108C1000020AB5EEC00AF1EE10FA13DAB4EE400A19
:108C2000F1EE10FA0ED600220623102102A80092BF
:108C30006722FBF7F9FE02AA08492846F5F734FA3D
:108C400007B030BD06492846F4F70AFE94ED020A43
:108C5000E9E700BF88C906608CC9066094C9066050
:108C600090C9066008B52DED028B072805D8DFE80E
:108C700000F05B220404370448080020BDEC028B9E
:108C800008BD91ED020AD1ED017A20EE000AA7EEAF
:108C9000A70AB5EE400AF1EE10FA4BD4F1EEC07A15
:108CA00017EE903A23F0030040F00200BDEC028B77
:108CB000A0F1FF4008BDD1ED018A0C2091ED028AA0
:108CC0000021F1EE688AF3F7EDFBB1EE488A1C4B08
:108CD0000360C0ED018A80ED028ABDEC028B08BD05
:108CE000D1ED017AF5EE407AF1EE10FA20D1D1ED16
:108CF000027AF5EE407AF1EE10FA14BF3E201E2003
:108D0000BCE7D1ED017A91ED027AFDEEE77ABDEE96
:108D1000C77A17EE900A17EE103A5840BDEC028B56
:108D2000400040F0010008BDBDEC028B084608BDC4
:108D30003E20A3E732F09AFBF0EE407AB0E700BFA6
:108D40009CC9066030B50C46114604221D462046DB
:108D50002DED028B85B0FEF795F82CB3012C30D0A9
:108D60002868354C820702D10368A34253D0FEF72E
:108D700097FDF0EE408A9FED318A6868830702D143
:108D80000368A3423ED0FEF78BFD30EE088A002137
:108D90000C20F3F787FB0460C0ED018A80ED028AA6
:108DA00005B0BDEC028B30BD21460C20F3F77AFBF9
:108DB0000023214A43600260836005B0BDEC028B52
:108DC00030BD28681E4B0340062B29D0810707D1F0
:108DD00003681C4A934223D0174CA34201D1DFE71A
:108DE000154CFEF75DFD0021B0EE408A0C20F3F734
:108DF00059FB0023046080ED018A836005B0BDEC5F
:108E0000028B30BDD0ED027A90ED010A78EEE78A50
:108E100038EE008ABBE7D0ED018A90ED028AACE71C
:108E200003A9002405F02CFA012303991A460094A3
:108E3000FCF706FAB4E700BF9CC90660000000001A
:108E40000F0080FFA0DF0660136803B1704740F297
:108E5000334399420BD0B1F5567FF7D1836823F0A5
:108E6000030343F00203A3F1FF4313607047436819
:108E700023F0030343F00203A3F1FF4313607047A1
:108E800008B500210C202DED028BF0EE408AB0EEEB
:108E9000608AF3F707FB044AC0ED018A026080EDA7
:108EA000028ABDEC028B08BD9CC9066043680B605A
:108EB00083681360704700BF10B52DED048B82B03E
:108EC00004460846B0EE409A01AA6946B0EE608AB0
:108ED000FEF7FEFC00284BD0A01E20284CD8DFE86F
:108EE00000F0824B4B4B4B4B4B4B4B4B4B4B50592E
:108EF000624BA36F4B114B4B4B4B4B5059624BA3E7
:108F00006F4B110068EE087AE9EE097AF5EE407AC7
:108F1000F1EE10FA00F1C380B1EEE70AB5EE400AB7
:108F2000F1EE10FA40F09280DDED017AF5EE407A34
:108F3000F1EE10FA40F0B880DDED007AF5EEC07A7F
:108F4000F1EE10FAC0F2B080F5EE407ADFED597A1A
:108F5000F7EE008AF1EE10FA48FEA78A00210C20F5
:108F6000F3F7A0FA544BC0ED018A036080ED028A4A
:108F700002B0BDEC048B10BD002002B0BDEC048B30
:108F800010BDDDED008ADDED017A79EE288A38EE3C
:108F9000278AE3E7DDED008ADDED017A79EE688A64
:108FA00038EE678ADAE79DED007ADDED017A67EE4B
:108FB000C88A28EE078AE9EE078AA9EE278ACDE754
:108FC000DDED017AF5EE407AF1EE10FA1CD1DDED1F
:108FD000007AF5EE407AF1EE10FA69D0C9EE278AF0
:108FE00088EE278ABAE7DDED007AF4EE497AF1EEF1
:108FF00010FA17D1DDED017AF4EE487AF1EE10FAAD
:1090000014BF1E203E20B3E79DED006AB5EE406A16
:10901000F1EE10FA0BD1B1EE490AC8EE278A80EEC4
:10902000278A9BE71E20A3E72448FCF759FE67EE3A
:10903000A75AF1EE676AE6EE065A86EE257AC6EE84
:10904000A57A8DED007ACDED017AB0E731F0CAFF57
:10905000F0EE490AF0EE408AB0EE480A33F0EAFB3F
:109060009DED007ADDED016A27EE008A20EE660AAA
:10907000A6EEA88AA7EE280A31F0ACFDB0EE409A21
:10908000B0EE480A33F0AEF8F0EE408AB0EE480A8F
:1090900033F05EF820EE098A68EE898A5EE7B0EE6A
:1090A000670A32F0E3F939E705490648FCF76CFD39
:1090B000FDF73CFD000000009CC9066078FB0660DF
:1090C0004807076020D006600B461146D3ED020A20
:1090D00093ED010AFFF7F0BEF8B514460E461D46A3
:1090E000154A214607463046FDF7CCFE134B2A6849
:1090F0009A421DD16868FEF741FB041E18DB00216F
:109100001820F3F7CFF9621C002104460760426083
:109110009000C4E90211F3F7E1F9022E206101D8B1
:109120002046F8BDA868FEF729FB60612046F8BD1F
:109130000020FCF7C1FD00BF0600040048E2066005
:1091400010B5C2684468531C9C4208BF00234469A0
:10915000E40702D584689C4211D0046944F82210C7
:109160008268C3609A4201D00E2010BD013342686C
:1091700093428360F8D1002383600E2010BD024922
:109180000248FCF701FD00BF5CFF06600CCE0660E4
:1091900004280BD0052807D1D1E90230C01A0CD41D
:1091A000400040F00100704700207047D1E9020301
:1091B000984214BF3E201E2070474B681844400060
:1091C00040F00100704700BF10B5D0E9022103460E
:1091D0008A420DD00169002451F8220041F8224052
:1091E000D3E9011201328A4208BF22469A6010BDBB
:1091F00001490248FCF7C8FC14FE06600CCE06606C
:109200000B6830B484689C4211D9C56801E09C4267
:109210000DD055F833204FEAC30C0133002AF6D0A5
:10922000042AF4D00B60C06830BC60447047002052
:1092300030BC704710B4074C034600220C6090F815
:1092400008C008465DF8044B81F804C05B68C1E9BA
:109250000232704704CC066010B40122044C002393
:109260000C600A715DF8044BC1E9020308467047BF
:1092700004CC066008B503799B0700D408BD002024
:10928000FCF72EFD2DE9F047D1F800901746044673
:1092900082B048460D46FFF7EDFF3968344A204654
:1092A0000909FDF7EFFD022C1AD07A68A2B100245B
:1092B00009F10409BD6855F8341005EBC40541B146
:1092C000042906D0012248464DF0C6F86B68436079
:1092D0007A680134A242EDD80E2002B0BDE8F087D2
:1092E000686810F0030104D10368DA68214B9A42E0
:1092F00027D0002109F1040AFDF7C2F8804606E0F4
:10930000E0B90122294650464DF0A6F84460404697
:10931000FDF72AF90028C8D00021FDF7B1F806466C
:10932000FDF722F905463046FDF71EF904463046A2
:10933000FDF71AF9002C18BF002DE1D10E48FCF7FB
:10934000BBFC2B689842B0D009F10406019107E0FC
:109350000122216830464DF07FF8636843606868F9
:1093600001A9FFF74DFF04460028F1D19DE700BF9A
:109370000500020015980160C4FD0660F8B50D46B1
:10938000064614460F6892B92246381D69684DF0AA
:1093900063F8034620B1406810B1022C0FD0F8BD2D
:1093A000022E08D0A868012CF9D15860F8BD3846C3
:1093B000FFF760FFE8E7022C04D00E20F3E700225D
:1093C0005A60F8BD69680148FDF78AFB28CE06603F
:1093D0000122FFF7D3BF00BF0222FFF7CFBF00BFBC
:1093E0000022FFF7CBBF00BF10B500F10C0182B027
:1093F00004468068FFF704FF60B12379012B0ED08B
:10940000022B09D06946D0E900230220CDE90023D0
:1094100006F0ECFC02B010BD406802B010BD006860
:1094200002B010BD032A2DE9F04F164685B005465F
:10943000884664D0394A0B680092934266D0DA8835
:1094400001233749DFF8F0901E46DFF8F0B00193B2
:10945000F4F72AFE33492846F4F702FA00230127DD
:10946000DFF8DCA003930DE032462846FEF79EF8B5
:1094700049462846F4F7F4F9324661682846002741
:10948000FEF794F803A94046FFF7BAFE0446E0B1A0
:10949000B7B1032E2168E7D1234B0B40062BE3D055
:1094A0008B0724D051462846F4F7DAF9216828467C
:1094B0000322FEF77BF851462846F4F7D1F9D7E7A7
:1094C00059462846F4F7CCF9E3E718492846F4F75B
:1094D000C7F9D8F80030009A934205D0019B1BB120
:1094E00013492846F4F7BCF905B0BDE8F08F0868C9
:1094F000FEF7DEFB0F4B8342D4D12168B4E7002393
:109500000193064BD0E902B90093A3E70123DFF8EA
:109510002890DFF828B01E4601939BE78CCB0660AD
:1095200044CA066048CA06600F0080FFF86C0660F7
:1095300050DA0660E9E90160DC190860A8C6066037
:109540004CCA0660F0B5184B06460A7A85B00C4640
:10955000012553F82210F4F783F914493046144FCB
:10956000F4F77EF9237A134962688DF804300023FA
:109570000091CDE9022305E0012221463046002575
:10958000FEF714F86846FFF72FFF044630B1002DB0
:10959000F2D139463046F4F763F9EDE70649304633
:1095A000F4F75EF905B0F0BD80CB066050CA0660E6
:1095B000A8C6066004CC066054CA066010B5002137
:1095C00004460C20F2F76EFF02490222C0E90014A3
:1095D000027210BDC8CB066010B5002104460C20F5
:1095E000F2F760FF02490122C0E90014027210BDC7
:1095F000C8CB066010B5002104460C20F2F752FFDC
:1096000002490022C0E90014027210BDC8CB0660F6
:1096100070B5044684B0FFF72DFE636833F00F0287
:109620001ED0227900215207019103D5C3F31B13E9
:10963000013B019301A92046FFF7E2FD6268034662
:109640000426103A00256260D0E900120220CDE91C
:10965000021202A9C3E9006506F0C8FB04B070BDA0
:109660004B2202490248FCF79FFA00BFD00707606F
:1096700028CE066010B50446FFF7FCFD201DFDF75F
:10968000F5FD0E2010BD00BF04280AD0052806D124
:109690004868C0F31B10400040F0010070470020F4
:1096A00070474B6833F00F0314BF3E201E207047F5
:1096B00002282DE9F0410E4682B014460FD024282E
:1096C00009D100222146301D4CF0C6FE78B13E2063
:1096D00002B0BDE8F081002002B0BDE8F0818A0749
:1096E00028D0A30703D123682E4A934203D01E201B
:1096F00002B0BDE8F08173686268534033F00F0335
:10970000F5D101AF043401930AE029684CF0A4FEBE
:109710000028ECD041686868FEF776FA0028E6D0A9
:1097200039463046FFF76CFD054600222046002DE5
:10973000EBD1CCE71C4B0A689A42D2D114F003015A
:10974000D5D123689342CFD101AF3046CDE9001186
:109750006946FFF755FD394680462046FFF750FD24
:109760000546B8F1000F19D0C5B12968D8F8000036
:10977000FEF74AFA0028BAD06968D8F80400FEF764
:1097800043FA69460028B2D03046FFF739FD394622
:1097900080462046FFF734FD0546E2E758EA050318
:1097A00095D0A4E78CCB066040CC06600B7A012BE9
:1097B00004D1242802D14968FFF77ABF00207047FE
:1097C00010B5002204300C464CF046FE08B140684B
:1097D00010BD21460148FDF783F900BF28CE066081
:1097E000024B40F8043BFDF711BD00BF8CCB066077
:1097F00010B5002104461020F2F754FE044B214618
:10980000044640F8043BFDF701FD204610BD00BFB3
:109810008CCB06602DE9F041054686B000200E464F
:1098200017469846FFF7E4FF1149044605608D424C
:1098300019D056EA070303D1204606B0BDE8F081EF
:10984000D8F80030394608EB860203A8CDE9014379
:10985000FDF7F0FC03AA01A9701CFFF713FD2046D9
:1098600006B0BDE8F081037943F004030371E0E73B
:1098700040CC066038B505468068FFF7B9FF04465E
:109880002B6803606A684368C2F31B1262F31F13FC
:10989000436003F0FC032A79C06802F0010213431D
:1098A00023712B792279C3F3800363F3820222713F
:1098B000D5E90221D20034F035F9204638BD00BF89
:1098C000F8B50D46064600216868FCF7D9FD022E62
:1098D000044668688CBFAE680E26FEF7D3F800B168
:1098E0004010FFF785FF0746051D02E04CF0B4FD70
:1098F00046602046FCF738FE014601222846002932
:10990000F4D13846F8BD00BF40680009704700BF79
:1099100030B5044683B015460191FFF7ABFC012238
:109920000199201D4CF098FD034620465D6003B070
:1099300030BD00BF30B50D4683B072B1042A04D0EB
:10994000FFF7E6FF0E2003B030BD002204304CF0DC
:1099500083FD58B1406803B030BD02226946CDE9AD
:1099600000051046FFF70AFD0E20ECE729460148E6
:10997000FDF7B6F828CE066010B5022282B00B467D
:10998000044669461046CDE90043FFF7F7FC204640
:1099900002B010BD10B5044682B04068FCF7E4FD8B
:1099A000034660B1A2686946019302205300013268
:1099B00043F00103A260009306F018FA034618462C
:1099C00002B010BD30B585B08C4611461A4602ACC7
:1099D0000C4B05466046019400930223FDF7E8FA1C
:1099E00000210C20F2F75EFD05600446002102987C
:1099F000FCF746FD034620466360039BA36005B069
:109A000030BD00BF7CCC0660F0B50D4611068FB0AE
:109A10001446074602F07F0602D4731E012B16D9A6
:109A2000022E2DD0EEB9696819B34B680BB3284AE2
:109A30002868904201D1022B27D9012B12D1002294
:109A4000896838460FB0BDE8F040FDF7AFBD2B6820
:109A5000D888F3F767FD01463846F3F701FF022E79
:109A60000ED06968224638460FB0BDE8F04005F0D8
:109A7000EFBF184938460FB0BDE8F040F3F7F0BE2D
:109A800015493846F3F7ECFECDE78868C207D4D510
:109A9000322201A909F084FA10B969684B68CCE751
:109AA0006A6803460D49384692685210F4F7FCFA8A
:109AB0006B685B68012B09D907493846F3F7D0FE7C
:109AC0006B6800223846D968FDF770FD0FB0F0BD15
:109AD000D0CE066084300860DC190860C8CC06600F
:109AE0002DE9F04114460D46184A064621462846FF
:109AF0001F46FDF7C7F900211820F2F7DFFC144AD2
:109B000000280446134B14BF044614462660A36085
:109B100025B9114E20466660BDE8F08105F10208C6
:109B200000214FEA88084046F2F7C8FC06460028A4
:109B3000EFD00A4BA8F1080245603946336008307F
:109B400033F0F0FF20466660BDE8F081FEFF0100C3
:109B50003C0400201CE2066048E2066050E2066019
:109B6000F8B50E4615460446D0E901139A188A4204
:109B700009D2C0682A461844314633F0D3FFA268A0
:109B80002A44A260F8BD02781AB90139C068CD1A1A
:109B9000F0E705F110070122C0680F443946F2F7DB
:109BA000ABFC18B1A3686760E060E3E7D4E9015358
:109BB0002070013DE068ED1ADCE700BF10B50446F7
:109BC000FDF7B4FC034BC2689A4214BF20692046DB
:109BD00010BD00BFE19A016008B5FFF7EFFF4368D1
:109BE0005A680AB1986808BD0E2008BD70B51368A0
:109BF00090B0154606460C46F3B1E3290ED0B229C3
:109C000037D0B42928D150680E2868D0830703D1F3
:109C1000624B02689A4276D0306109E050680E28A3
:109C200048D0810763D15E4B02689A425FD1B06031
:109C300000232B6010B070BD3D2916D0A22928D07A
:109C4000E32931D0B22941D0B42936D10369002BA0
:109C500008BF0E231360EDE7E229EBD150684CF00A
:109C600017FC002330752B60E4E74368136010B0E5
:109C700070BD50680E282FD0820703D1474B026871
:109C80009A4240D0F0600122002332752B6010B060
:109C900070BD0368434A934225D04349184610B02B
:109CA000BDE8704007F05CB88368002B08BF0E2346
:109CB0001360BFE73D4BB360BAE7E2292ED1037DC5
:109CC000002B14BF3E231E231360B3E7C368002B91
:109CD00008BF0E231360ADE70023F360D3E7002332
:109CE0003361A5E73046FFF777FF2860A2E7FDF76D
:109CF0001DFCC4884FF4D5734FF49F62B4212C48E7
:109D00000094FBF7F5FFFDF711FCC5884FF4D57300
:109D10002122214626480095FBF7EAFF22490068E8
:109D200007F01EF8002885D040F2FD239C42D9D0D0
:109D300040F2CA439C4206D173685A68012A1AD974
:109D4000DB682B6076E740F20E339C4208D17368E3
:109D50005A68022A02D91B692B606BE70E23FBE7C6
:109D600040F20F339C427FF465AF73685A68042A4F
:109D7000F4D99B69F0E7002AF0D0322203A9986851
:109D800009F00EF904460028E8D033F049FF0146F7
:109D9000204603F08FFB28604CE700BF2CCD066007
:109DA00028E206605CCF0660D0CE06601CE206604A
:109DB00024F6066000231A461946FFF791BE00BF3D
:109DC00010B4C46813460022A4465DF8044B6047F3
:109DD0002DE9F0410D4686B0002106461020904640
:109DE000F2F76CFB044628460EF0E4FE002107461D
:109DF000F2F764FB5CB328B301232946039702AD55
:109E000000278DF80830164B4246059068460193AE
:109E100004970095F4F756F9DDE90432D754049914
:109E2000A1600598E0600F4B2360F3F739FA2B46E9
:109E300000220121606030460294FFF751FE06B017
:109E4000BDE8F081014602ADC4E90200EBE723461C
:109E500022462146304606B0BDE8F041FFF740BE3D
:109E6000619B0160A0DF06600EB400B582B003AA5A
:109E700052F8041B0192FFF7ABFF02B05DF804EB50
:109E800003B07047FFF7F0BF830703D1064B0268AA
:109E90009A4202D0054906F063BF054BC2689A4258
:109EA000F8D10120704700BF74E306602CCD066036
:109EB000E19A016008B5FDF739FBBDE80840FFF7FE
:109EC000E3BF00BF10B582B004460191FFF7F2FF77
:109ED000019928B9204602B0BDE8104006F040BF05
:109EE0002046FDF723FB04460199204602B0BDE859
:109EF000104006F035BF00BF08B5FFF75FFE002336
:109F0000024A03618382C0E9022308BD1CE20660A5
:109F1000024AC0E90012FFF7EFBF00BF48E2066047
:109F20002DE9F843894690461F46FFF747FE8468AF
:109F30000546254E94B1B44210D0A668F6B1E0882B
:109F4000A188831C8B422ADA06EB8003C21CE280C4
:109F500046F82090C3E90187BDE8F88300210C2072
:109F6000F2F7ACFA034600282BD0AB6096E8070066
:109F700083E80700AC68A668002EE0D131460C20CB
:109F8000F2F79CFAA060AB689A68002AE4D003223A
:109F90009A80AB68DE80AC68A668E088D4E70331BD
:109FA000304601228900F2F7A7FA0028D4D0AB6826
:109FB0009860AA68938803339380AC68A668E088A9
:109FC000C2E7024BD1E700BF1CE20660300400206C
:109FD00038B50D461446FFF7F1FD83682BB1DB88D9
:109FE0002B6083689B68236038BD2B60236038BD7D
:109FF00030B5054683B009E068680E2802D0FBF74B
:10A0000013FF044620464CF043FA60B9A868FCF7F9
:10A01000ABFA01AB00220121044601900028EBD1EC
:10A02000204603B030BD019C204603B030BD00BFC8
:10A0300070B50C461D46114606464FF004122046E8
:10A04000FCF720FF00210C20F2F72CFA06602B68A9
:10A050000446002143606868FCF712FA0346204674
:10A06000A36070BD01F1FF4323F0030307EE903AB4
:10A07000072805D8DFE800F01308040415041D06BE
:10A0800000207047002B0ADAF1EE677A17EE901A7B
:10A0900021F0030141F00201A1F1FF4070470846A1
:10A0A0007047F5EE407AF1EE10FA14BF3E201E2004
:10A0B0007047FDEEE77A17EE901A490041F0010073
:10A0C000704700BF01F1FF41672230B521F0030363
:10A0D00087B00025044600EE103A1021062302A89E
:10A0E0000095FAF7A1FC02A92046F3F7B9FB2E214F
:10A0F00002A833F0F9FD08B107B030BD652102A810
:10A1000033F0F2FD0028F7D16E2102A833F0ECFD08
:10A110000028F1D102492046F3F7A2FBECE700BF8B
:10A1200078D0066038B590ED000A0546D1ED000AFA
:10A130000C4631F021F9B5EE400AD5ED006A94EDF8
:10A14000007A36EEC06AF1EE10FAC6EE077A1DD13B
:10A1500017EE103A9FED250A9FED256A002B20FE91
:10A16000060AF5EE407AF1EE10FA2AD1C6EE877AA9
:10A170009FED1E7A17EE903ADFED1D7A002B27FE39
:10A18000277A85ED007A84ED000A38BDB5EEC00A65
:10A19000F1EE10FAB5EEC07A4CBF01220022F1EECA
:10A1A00010FA4CBF012300239A42DAD0B7EE006ABE
:10A1B00030EE070A77EEC67AF5EE407AF1EE10FA45
:10A1C000D4D0F6EE006ABBFE677A77EEC77AF4EE7B
:10A1D000E67AF1EE10FAD4DDF7EE007A37EE277A60
:10A1E00085ED007A84ED000A38BD00BF0000000054
:10A1F0000000008030B50C4687B011460222204690
:10A200001D46FCF73FFE14B9124807B030BD0122CD
:10A2100003A92868FDF716FDA0B9286800F003031C
:10A22000022B0AD0FDF73CFB10EE103A23F003009E
:10A2300040F00200A0F1FF40E7E7074B0340062B88
:10A24000E3D1EFE70023DDE903011A460093FAF7B3
:10A25000F7FFDAE702008080070080FF30B50D4687
:10A2600087B0044603A928468DED010AFDF7DCFA04
:10A27000A8B3232C35D8DFE814F0E000EC00F80098
:10A280000401B600340034003400340034003400DB
:10A29000340034003400240097005000340057008C
:10A2A000650071003700340034003400340034009D
:10A2B00024009700500034005700650071003700FB
:10A2C000C2009DED010ADDED037A30EE270A10EEA3
:10A2D000103A23F0030040F00200A0F1FF4007B065
:10A2E00030BD002007B030BD9DED010ADDED030A51
:10A2F000B5EE400AF1EE10FA5DD1F5EEC00AF1EECE
:10A3000010FA58D5F0EEE07A9FED6A7AF4EE477ACB
:10A31000F1EE10FA4FDCFCF709FC9DED010ADDEDD2
:10A32000037A20EE270AD2E7DDED037AF5EE407AD4
:10A33000F1EE10FAEFD003A901A8FFF7F3FE9DEDAF
:10A34000010AC4E7DDED037AF5EE407AF1EE10FA8A
:10A35000E1D09DED017A87EE270AB8E7DDED030A2B
:10A36000F5EE400AF1EE10FAD5D09DED010A31F07C
:10A3700003F8B5EE400AF1EE10FA00F08E80B5EE6B
:10A38000C00ADDED037AF1EE10FAF5EEC07A4CBFAB
:10A3900001220022F1EE10FA4CBF012300239A4261
:10A3A00095D030EE270A92E79DED010ADDED037AA4
:10A3B00030EE670A8BE7B5EEC00AF1EE10FA75D5FC
:10A3C000F4EE600AFBFE607AF1EE10FA6ED6F4EE5F
:10A3D000607AF1EE10FA69D02946DFED370A2220C3
:10A3E000FEF76AFD7BE79DED017ADDED037AB4EEC1
:10A3F000E77AF1EE10FAACBF3E201E206FE7DDEDEC
:10A40000037AF5EE407AF1EE10FA84D003A901A8A0
:10A41000FFF788FE019A039B022022F0030204A9A1
:10A4200023F0030302430343A2F1FF42A3F1FF43DE
:10A43000CDE9042305F0DAFC51E79DED017ADDED6D
:10A44000037AB4EEE77AF1EE10FA4CBF3E201E20FC
:10A4500045E79DED017ADDED037AB4EEE77AF1EEA2
:10A4600010FACCBF3E201E2039E79DED017ADDEDCC
:10A47000037AB4EE677AF1EE10FA14BF1E203E2084
:10A480002DE79DED017ADDED037AB4EEE77AF1EE8A
:10A4900010FA94BF3E201E2021E7039B9FED060A81
:10A4A000DFED067A002B20FE270A10E730F08EF849
:10A4B0000DE700BFFFFF7F7F00000000000000806D
:10A4C00001F1FF439107844623F0030310B403D145
:10A4D0000A4914688C4207D0114600EE103A6046D3
:10A4E0005DF8044BFFF7BABE1146DFED050A00EE3A
:10A4F000103A5DF8044BFEF7DFBC00BF9CC9066054
:10A500000000000007EE901A06EE900A9FED047A14
:10A51000F8EE677AB8EE660AA7EE870A704700BFC2
:10A520000000804FDFED067ABCEEC07A60EE277A3D
:10A5300017EE100AFCEEE77A17EE901A704700BF8C
:10A540000000802F1346002210B504460846194625
:10A55000FCF798FC6368BDE81040184770B51C46CE
:10A560000546084611464FF00212FCF78BFC6B685B
:10A570002068BDE87040184770B51C46054608467F
:10A5800011464FF00412FCF77DFC6B68D4E9000122
:10A59000BDE87040184700BF70B51C460546084628
:10A5A00011464FF00612FCF76DFC6B682068D4E989
:10A5B0000112BDE87040184770B50D4686B01146CF
:10A5C0000446426828461E460191FCF75BFC63681E
:10A5D000019913F0010F06D1A3683146284606B051
:10A5E000BDE87040184706EB850203A8FCF722FE81
:10A5F000A36803AA31462846984706B070BD00BF3D
:10A60000836813F9012B002AFBDB13F9012B002AC5
:10A61000FBDB1888704700BF0B46084910B504469D
:10A6200082B018460193FFF7EBFF019B02462046DC
:10A6300002B0BDE81040F3F737BD00BFB8D00660E8
:10A640002DE9F8430E46914698460546D0B1476835
:10A6500041B3781D00218000F1F724FF224B04460E
:10A6600005F108010360BA00204BDB69C0E90298DC
:10A670004360103033F056FA043744F82760204620
:10A68000BDE8F88321B329461420F1F70BFF164BE0
:10A690002F4604460360154BDB69C0F80C80C0E907
:10A6A0000139E9E7381D8000F1F7FCFE0E4B044646
:10A6B000BA00036005F108010C4BDB69C0E9013900
:10A6C000C4F80C80103033F02DFA2046BDE8F88332
:10A6D0001020F1F7E7FE044A044B04460260DB69F0
:10A6E000C0E902984360CAE7CCD0066000040020AD
:10A6F0002DE9F047D0F8048006460F4682B0D8F81E
:10A70000080010F8014B2506C4F3C309C4F3800107
:10A7100016D54FF0000C10F801EB4FEA4C0A0EF082
:10A7200030050EF002041EF0800F04FA0CF405FA56
:10A730000AF50CF1010C49EA050941EA0401EAD1E4
:10A7400009F1010901EB4100002148440830800073
:10A75000CDE90023F1F7A6FE05460B4839462860EF
:10A76000307AC5F80C8028720E20A5F81890686021
:10A770000020DDE90023286105F10C0008F064FCED
:10A78000284602B0BDE8F087B0D2066008B543683D
:10A7900013B14160184608BD0148FBF78DFA00BFB0
:10A7A0003800076030B50B7A054683B00C46C868A0
:10A7B0005BB1FFF725FF40F2A32203460949284673
:10A7C0000094F3F771FC03B030BDFFF719FF40F2BE
:10A7D00037320346034928460094F3F765FC03B07B
:10A7E00030BD00BF34D2066008B5037A03B108BD9E
:10A7F000AD2340F2373202490248FBF7D5F900BFDA
:10A80000B40A076010CD066038B505460C460C202A
:10A810000021F1F747FE024A0472C0E9002538BD65
:10A82000ECD206602DE9F0410446884616461F46E4
:10A83000FCF718FB2569002D4BD0616800294DD02D
:10A84000626904F11C030E2908BF31469A423AD0CE
:10A85000C2F80080234E4FF000082046C4F8048060
:10A86000F369E36150F80C3F5B68F3614BF008FE5D
:10A87000E36901280546F3614FF00E0363601AD0C7
:10A88000022807D06369C4F810801B683B60284623
:10A89000BDE8F081206AC4F810803860FCF746FEFD
:10A8A000114906F05DFA0028F1D010491048FFF771
:10A8B000E9FA3860EBE76269284612683A60626933
:10A8C0001360BDE8F081B8F10E0FC3D00948FBF763
:10A8D00007FA0E2328463B60BDE8F0810648FBF7E7
:10A8E000EBF900BF000400205CCF06605C0007604D
:10A8F00024CF0660B4FB06603800076010B582B054
:10A900001C4601ABFFF78EFF01280AD002280FD0AA
:10A91000019B0E2B08D074B9084A2046936202B0FE
:10A9200010BD019802B010BD002213460192F2E75B
:10A930000198F1F791FD1846FCF7DEF800040020BD
:10A9400010B5037A2BB91A460E21BDE81040FFF767
:10A95000D5BF0148FBF7C4F95C03076002288C46A9
:10A960004A6803D98B680E2B18BF1A4601230E21A3
:10A97000DCF80000FFF7C2BF01230022FFF7BEBFD3
:10A9800010B5044682B00F490F48FFF7C1FA01AB7A
:10A990000D4A0E212046FFF745FF01280ED0022860
:10A9A00006D10198FCF7C2FD064906F0D9F910B1AD
:10A9B0000E2002B010BD0198F1F74EFD0349044886
:10A9C000FBF7E2F8B8CD06600010202048000760D1
:10A9D00024CF066010B596B0044603A8F1F724FD15
:10A9E00050B104980E4A0368934202D00D4A934234
:10A9F00014D1002016B010BD0146221D0120FBF726
:10AA000087FAE368019023F00103023343F0010366
:10AA1000E360F1F701FD019816B010BDF1F71CFDE0
:10AA20000CCE06605CCF066010B40346054C0122D4
:10AA300008460C601C684C605B685DF8044BC1E91B
:10AA40000232704728D30660C2070DD5401009D0E6
:10AA5000B0F1404F0AD00028B8BF4042B0FA80F0B1
:10AA6000C0F1200000F066BC00F03EBB202000F0EA
:10AA700061BC00BF30B589B0284B0431013802AC4D
:10AA8000CDE900340323FCF727FA9DF81030002BA2
:10AA90003DD1012205A90298FDF7E8F8039D40F297
:10AAA000D663059A9D4225D042F2E6439D422AD1C3
:10AAB0000699944601244B1E19B3013B002004E083
:10AAC000B0F5800F03F1FF330BD29CF800E0B3F137
:10AAD000FF3FA4444EEA0020F2D100F02BFC09B065
:10AAE00030BD40F2D660281A18BF012000F010FBDC
:10AAF00009B030BD06994FF0FF344B1E02EB030C3A
:10AB0000DAE70846E9E740F26D20FCF761FB40F226
:10AB1000012240F29B410248FBF7CAFF64D3066062
:10AB2000B4F90660002808B500DA82B1032905D817
:10AB30002AB9CA0001239340984208DA08BDCB0025
:10AB40000122013B02FA03F35A429042F4DA01482F
:10AB5000FBF7BAFF9C0B076010B510EE104AC4F368
:10AB60000F4303F4FF43B3F5FF4F23D0002C0EDB5C
:10AB7000174B2340B3F19C4F11D900F073FA00EE4C
:10AB8000104A04460430F3F75BFD204610BD34F054
:10AB9000004304D004F1FF43B3F19C4FEDD807EE1E
:10ABA000904AFDEEE77A17EE904A600040F001040B
:10ABB000204610BDC4F316045E2224B940F262316F
:10ABC0000448FBF781FF40F2A9110248FBF77CF82B
:10ABD000000080FF30FB066030B50C4685B01146A2
:10ABE000042220461D46FCF74DF95CB3012C17D119
:10ABF0002868C30724D410F0030226D10268254B2D
:10AC00009A421DD0244B0340062B3AD01046FDF744
:10AC10004FF8224B8342286833D000F0030218E03B
:10AC200003A9286803F02CFB039904466868019186
:10AC3000FCF7A4FD0023024601992046FAF766FAC4
:10AC400005B030BD012005B030BD134B0340062BCD
:10AC500017D0022A06D00146082005B0BDE83040D2
:10AC6000FBF752B80E4B0340062BF4D000F1FF4027
:10AC700020F0030300EE103A05B0BDE83040FFF7C6
:10AC80006BBF03A903F0FCFA002303991A46FAF7F5
:10AC90003DFAD5E7F4D306600F0080FFE9E90160D3
:10ACA000070080FF38B50B4C214411F8014CB0FB74
:10ACB000F4F463B1084D631CA5FB03135D08104653
:10ACC0000AB132F0ADFF03342C44204438BD1D4698
:10ACD000F5E700BFE4D30660ABAAAAAA2DE9F04FBE
:10ACE00085B080468B469DF840409DF84490029484
:10ACF00013F0010401920094DDE90E6700F09E80DC
:10AD00005D1040D44B463A4631462020FFF7CAFF3B
:10AD1000DBF80030824683424FF000030093039338
:10AD2000C0F08380D8F800B000230BEB0A0000F8D5
:10AD3000013C002D40F08B803023841E00F8023C43
:10AD40007FB1384632F06CFF201A584509D93B785C
:10AD500033B1024602F8013B17F8013F002BF9D14D
:10AD600004465C4504D9009B13B1039B013C23704E
:10AD7000D8F800302046019A53441B1B013B136056
:10AD800005B0BDE8F08F4B463A4631462020FFF72C
:10AD900089FFDBF800306D428246984243D8D8F8EC
:10ADA00000B000232D225844039200F8013C0138E2
:10ADB000029BB9F1000CCDF808900146A3F10A03FB
:10ADC00018BF4FF0010C9946B5FBF6F306FB135480
:10ADD0001D46092C04F1300288BF09EB0402003B38
:10ADE00001F1FF3418BF012301F8012C5C4594BF29
:10ADF0000022012213EA0C0F02D0A0EB040E2AB9A4
:10AE0000002B9DD0002A9BD02146DDE7BEF1030F29
:10AE1000FAD18C1E029A5C4501F8022C204694BFA0
:10AE200000220122ECE72D23039300215046F1F785
:10AE300039FBC8F80000CBF800A073E7029CCDF8FE
:10AE40004490109405B0BDE8F04F00F01BB90138F4
:10AE5000AEE700BF70B58CB00B4600250A2210216A
:10AE600008AE04460092069107AA06A905A8019516
:10AE70000596CDE90255FFF731FF01462046F2F76E
:10AE8000EFFC0598B04201D0F1F738FB0CB070BD73
:10AE900070B5054682B00E4614461AB3012000F084
:10AEA000B1F90190F300581E00F0ACF90199024687
:10AEB0000C204BF0F1FA04462946002022464BF0C4
:10AEC000EBFA3E280AD121460120FAF71DFF294658
:10AED000024604204BF0E0FA3E281BD031460E48D3
:10AEE000FBF7F2FD00F02AF90028F7DB012000F063
:10AEF00089F90146F000019100F084F901990246B8
:10AF00000C204BF0C9FA2946024620464BF0C4FA01
:10AF10003E28E3D102B070BD9C0B07602DE9F043E1
:10AF20008DB0304B0D46013805AC0431CDE900340D
:10AF30000323FBF7D1FF059C002C4FDBDDF81880C5
:10AF400040F2D66108A82D68B8EB010721469DF8AC
:10AF50001C9018BF0127F2F751FB0A9E22460021E0
:10AF6000304632F023FEEB072CD56B1014D0184678
:10AF70004A4621460393FFF7D5FD042C039B254643
:10AF800028BF0425002B0BDA22464FF0FF31304654
:10AF900032F00CFE039B03E0042C254628BF042559
:10AFA00040F2D662904501D0641B264432463946B1
:10AFB000284606F0D3FE08A90B4802F045FA0DB06A
:10AFC000BDE8F0834A4621462846FFF761FF334635
:10AFD00022463946284600F0ADF8ECE70020FAF7A3
:10AFE0006BFE00BF7CD306603CDD066008B1FFF756
:10AFF00099BD70471E2A38B514460D4621D03E2A09
:10B0000024D01D2807D1A0F500030E3B1340062BCA
:10B0100010D0930701D0002038BD1068FCF748FE1F
:10B020000D4B834206D023680C4A934202D00C4A4F
:10B030009342F0D12A4621461D20BDE838404BF00E
:10B040002BBA0122BDE838404BF026BA0322BDE8F6
:10B0500038404BF021BA00BFE9E9016050E20660D8
:10B0600024D5066010B500211020F1F71BFA044B1F
:10B07000044640F8043BF3F77FFA204610BD00BFBA
:10B08000F4D306602DE9F04F85B0054698680E466A
:10B09000DDF838801C46DDF83C9017469DF844A04A
:10B0A00000014A46414653469DF840B0FFF7FAFD7D
:10B0B000336883420FD3CDF800A05B462D684A4623
:10B0C0004146201D0195F4F7E3FA034628463B600C
:10B0D00005B0BDE8F08F00210390F1F7E3F9039A82
:10B0E00028603260E7E700BF836873B16FF0004209
:10B0F000C068591C1A4430F81200B0FA80F0C0EB56
:10B100000110400040F0010070470120704700BF6F
:10B1100010B50C4682B001920090FFF7A3FF2246C3
:10B120000446019B04300099F3F74EFB204602B021
:10B1300010BD00BF0430F4F731BA00BFC30706D515
:10B14000401000280FDB14BF0120002070478368E7
:10B150003BB1037913F0010F14BF4FF0FF30012012
:10B160007047184670474FF0FF30704720B50D46C6
:10B17000072805D8DFE800F005121B0424042B077C
:10B180000025284620BD0B79DB07FAD5FFF76AFFBB
:10B19000291D05460430F3F793FBF2E7FFF762FF42
:10B1A000291D05460430F3F797FB284620BDFFF71D
:10B1B00059FF291D05460430F3F7A0FB284620BDA2
:10B1C0008B68002B14BF3E251E25284620BD081D78
:10B1D000F4F7B0F9400040F00105284620BD00BF5B
:10B1E00010B584B003910290FFF73CFF01210446A3
:10B1F000029A0430039B0091F3F7F4F9204604B05F
:10B2000010BD00BF90EA40024FEA400302D443F071
:10B2100001007047C117FFF7E3BF00BF10B584B04E
:10B2200003910290FFF71EFF00210446029A0430AA
:10B23000039B0091F3F7D6F9204604B010BD00BF80
:10B240002DE9F04710F001088AB006460C46154675
:10B2500005D181073CD1334B02689A4238D114F0B2
:10B26000010A2FD015F0010905D1AB0730D12D4BC4
:10B270002A689A422CD100200021FFF7CFFF074611
:10B28000B8F1000F33D10436BAF1000F29D10434DC
:10B29000B9F1000F1FD104356B68002B3ED02B464F
:10B2A00022463146381DF4F7DBF801AB9E422BD025
:10B2B00004AB9C422ED007AB9D421ED038460AB04C
:10B2C000BDE8F087A20703D1164B22689A42C9D085
:10B2D0001548FAF705FD691007A807ADF3F752F90D
:10B2E000DAE7611004A804ACF3F74CF9D0E7711069
:10B2F00001A801AEF3F746F9C6E72846F3F756F979
:10B3000038460AB0BDE8F0873046F3F74FF904AB92
:10B310009C42D0D12046F3F749F9CCE703490448D1
:10B32000FAF732FCF4D30660E8070760D807076035
:10B3300004D0066010F0404F03D1400040F00100FF
:10B3400070470021FFF76ABF70B5044684B01E46FF
:10B350000D460392FFF786FE039B2A46009605469C
:10B3600021680430F3F7DCF92368024628461344C9
:10B37000236004B070BD00BFC30701D54010704703
:10B380000430F4F7D7B800BFC30700B583B003D5C6
:10B39000401003B05DF804FB01A90430F4F7DEF8B7
:10B3A00018B1019803B05DF804FB02490248FAF7AE
:10B3B000EBFB00BF78070760ECCE06602DE9F04399
:10B3C0000D4607461446E9072DED028B89B055D48A
:10B3D00005F10408E2072AD414F0030313D123680B
:10B3E0008F4A934200F086808E4A934277D0294656
:10B3F00022463846FFF7FEFD0546284609B0BDEC5B
:10B40000028BBDE8F083022BF1D1874B2340062B42
:10B41000EDD04046F4F71CF921463846FEF71EFFF2
:10B420000546284609B0BDEC028BBDE8F08302AEAC
:10B430006310022201A902A8F3F7ACF8202F26D04E
:10B44000132F24D0A7F109095FFA89F31A2B3AD8F0
:10B45000FFF708FE0546B9F1190F00F2C380DFE8D7
:10B4600009F0BBB5AF64649DA9A3C18DC17D73BB59
:10B47000B5AF64649DA9A3C18DC17D736B10022219
:10B4800001A902A80DF10808F3F784F8A2E7736890
:10B49000002B00F0BD804046F4F7DAF8B0EE408AA9
:10B4A0003046F4F7D5F8C8EE007A17EE900A20F08F
:10B4B000030040F00200A0F1FF45284609B0BDECB2
:10B4C000028BBDE8F08331464046F3F7D9F9042FEB
:10B4D00000F2A380DFE807F0241F1A151000404691
:10B4E000F4F7B6F82146DFED510A3846FDF7E4FCE3
:10B4F000054682E7261DA1E70028B4BF1E253E258C
:10B500007BE70028CCBF1E253E2576E7002814BF28
:10B510001E253E2571E70028D4BF1E253E256CE779
:10B520000028ACBF1E253E2567E72046FFF72CFF0D
:10B53000021E6FDB192F414605F1040065D00C2F68
:10B5400063D0F3F77FFA58E73378DB073FF561AF55
:10B55000324641460430F3F7DFFD4EE77368002BB7
:10B5600056D005A8F3F708F805A833464246291D2A
:10B57000F3F71CFE05A8F3F719F83EE77368002BF4
:10B5800046D005A8F2F7F8FF281D3346424605A924
:10B59000F3F70CFE05A8F3F709F82EE7324641460B
:10B5A0000430F3F7BBFA28E7324641460430F3F79C
:10B5B0001FFD22E7324641460430F3F7F7FA1CE755
:10B5C000324641460430F3F74BFB16E7324641461C
:10B5D0000430F3F787FC10E7324641460430F3F7B6
:10B5E000E5FB0AE773689BB1FFF73CFD291D334675
:10B5F000044642460430F3F7D9FD05A90220CDE9FF
:10B60000054504F0F3FB0546F7E6F3F7B7F9F4E672
:10B61000FBF78CFA0648FAF74FFB0025EDE600BF72
:10B62000F4D306609CC90660070080FF000000009C
:10B63000040507600430F4F70BB800BF10B4054AE6
:10B640000023054CC1E90203C1E9004208465DF848
:10B65000044B70475DB6016070D80660D0E90212F5
:10B6600003468868824205D2C868511C50F82200FF
:10B67000D96070470020704738B50D46114905F074
:10B68000FFFB0446D0E901138B4206D2E268591C45
:10B690000E20A16042F8235038BDC900C068F0F701
:10B6A0001FFF0021E060D4E9012352006260D21A3A
:10B6B0000133013A00EB8300920032F077FAA3687D
:10B6C000E4E700BF24D5066038B50B4604460021E8
:10B6D0001846FAF7D5FE054601E0FFF7CDFF2846EC
:10B6E000FAF742FF014620460029F6D138BD00BFD7
:10B6F00038B50A49002505F0C3FB04461021C0688F
:10B70000A560F0F7EDFE042203460E206260E360C0
:10B710001D605D609D60DD6038BD00BF24D50660A2
:10B720000B460B4910B50446184605F0A9FB042C3E
:10B7300008D0052C04D18068400040F0010010BD05
:10B74000002010BD8368002B14BF3E201E2010BDBA
:10B7500024D50660104938B505F092FB81680029B0
:10B760008C46B8BF01F1010C01294FEA6C0C11DDC8
:10B770006FF0404200230A449200C1688D5851F88E
:10B78000234041F823500133C16863458C50A2F136
:10B790000402F2DB0E2038BD24D506602DE9F84FF7
:10B7A00083468A4615469846FBF75CFBD34551D243
:10B7B000ABF10409002D58D0DAF800102846FAF74A
:10B7C0008FFB0746544609F10406B44216D9316886
:10B7D0001DB12846FAF784FB01463A4600204AF09C
:10B7E0005BFE80450AD11AE02168FAF779FB3946F9
:10B7F000024600204AF050FE80450CD1043C284609
:10B80000A6420ED2002DEFD12268394600204AF020
:10B8100043FE8045F2D03368226832602360B1462F
:10B82000D1E7AAEB0603A4EB0B0230689B10DAF811
:10B830000010013B3160CAF80000B3EBA20F0BDD32
:10B84000584643462A46214609F1080BFFF7A6FF52
:10B85000DA45ADD8BDE8F88F514643462A4609F18E
:10B860000800A246FFF79AFFF2E7DAF80070A9E7AE
:10B8700030B585B0124B0C46013802AD0431CDE92C
:10B8800000350223FBF728FB0E49206805F0F8FA83
:10B890008368012B11D9029A6FF040419DF80C404A
:10B8A0000E2A1944C06808BF0022002C00EB810159
:10B8B00014BF1E233E23FFF771FF0E2005B030BDDD
:10B8C00048D4066024D5066010B50C4682B00749FE
:10B8D0000190206805F0D4FA2346019AD0E90210BD
:10B8E00002B0BDE8104005F08FBC00BF24D5066053
:10B8F000032A2DE9F041174606460D4621D0DFF810
:10B900005080012710493046F1F7AAFFAB6893B188
:10B910000024EB683A46304653F824100134FBF714
:10B9200045FEAB68A34206D9002CF2D04146304612
:10B93000F1F796FFEDE730460449BDE8F041F1F735
:10B940008FBFD0F80880DDE744D40660A4C6066047
:10B95000A8C6066000B50A4683B00649019205F004
:10B960008FFA019AD0E9021003B05DF804EB05F0FC
:10B970008BBC00BF24D5066070B511F003060C46E1
:10B98000034603D11E4A0D68954205D0214618464C
:10B99000FFF79AFE0E2070BD294605F071FA0346A6
:10B9A000204629461C4605F06BFA82680546A368C6
:10B9B0006068991881420CD8E0689200E96800EB51
:10B9C000830032F0AFF8A368AA680E201344A36086
:10B9D00070BD0431E0688900F0F782FDA368E06083
:10B9E0003146AA681A4404326260AE683344D21AFF
:10B9F00000EB8300920032F0D9F8A368AA68DBE775
:10BA000024D5066070B50C461449154605F038FA81
:10BA10006310826806464FF00E0148BF9B1823EA68
:10BA2000E374944228BF1446FFF726FEB268531E03
:10BA3000A3420DD90A4911444FEA810CF16851F82B
:10BA40000C20ACF1040C41F82320013BA342F5D1BA
:10BA5000F3680E2043F8245070BD00BF24D5066063
:10BA6000FEFFFF3F70B50D4606461E49286805F0EB
:10BA700007FA012E04464FF0000314BF6A684FF026
:10BA8000FF320068A168FBF7BBFFA2682AB3E36836
:10BA9000013A53F8205003EB8001A260121A0846C5
:10BAA0000431920032F06EF80021D4E9022343F809
:10BAB00022106168042903D9A368B1EB430F01D8B0
:10BAC000284670BD4908E0688900F0F709FD636801
:10BAD000E06028465B08636070BD6C210248FAF79D
:10BAE000DFF800BF24D50660D007076000B583B03B
:10BAF00002460B4602206946CDE90023FFF7E4FE2B
:10BB00000346694602200193FFF7ACFF0E2003B005
:10BB10005DF804FB38B5826804462AB3C068013A70
:10BB200050F8215000EB8103A260521A1846191DEB
:10BB3000920032F027F80021D4E9022343F82210C2
:10BB40006168042903D9A368B1EB430F01D82846E3
:10BB500038BD4908E0688900F0F7C2FC6368E0601E
:10BB600028465B08636038BD6C210148FAF798F8F5
:10BB7000D00707602DE9F04107460E460E2190469A
:10BB8000FFF77AFDBA68531EB3420DD9094C14442D
:10BB90004FEA840CFC6854F80C50ACF1040C44F8E7
:10BBA0002350013B9E42F5D1FB6843F82680BDE857
:10BBB000F08100BFFEFFFF3F38B50D4604460C4A3A
:10BBC0000021042D2B46026038BF0423856063608A
:10BBD0009800F0F767FC626803460021521B00EBF7
:10BBE0008500E3609200BDE8384031F0DFBF00BF60
:10BBF00024D5066010B5044600211020F0F752FC51
:10BC000021460446FFF7D8FF204610BDF0B50E468A
:10BC1000044685B03B493046154605F031F90746E4
:10BC20001D2C15D8DFE804F018181818181414146F
:10BC30001414141414143D1414141414141414149B
:10BC400014141420140F03A92846FBF7C3FD80BB6E
:10BC50000024204605B0F0BDAB0742D0022CF7D13E
:10BC60001E24204605B0F0BD15F00304F0D1254B8D
:10BC70002A689A42EDD1AB6880681844FFF7BAFF92
:10BC80000446C068D7E90221920031F04BFFB86842
:10BC9000E368D5E9022103EB8000920031F042FF16
:10BCA000D7E7344629463046FFF766FE204605B002
:10BCB000F0BD0399002902DA002319460393B868FE
:10BCC00005F098F9FFF796FF0446D7E90223E168EB
:10BCD0001846039B0091042105F09AF9204605B00F
:10BCE000F0BD084B2A689A42B8D1D0E9022120461B
:10BCF000D5E90243009405F031FA0028B0D03E2483
:10BD0000A7E700BF24D5066038B50C4611460222CD
:10BD10001D462046FBF7B6F824B92046BDE838405A
:10BD2000FFF768BF0020FFF765FF2968BDE83840CE
:10BD3000FFF7CABC38B50C460546FFF75BFF64B198
:10BD40005DB1231FC4F1040103EB850CCA1853F83D
:10BD5000045FC4686345A550F8D138BD044908B5EF
:10BD600005F08EF8BDE80840D0E90201FFF7E2BF18
:10BD700024D5066038B50D460449144605F080F810
:10BD800083682B60C368236038BD00BF24D506607C
:10BD90008160704730B5154683B00A460749019265
:10BDA00005F06EF8044681680023019A0068FBF7ED
:10BDB00027FEE36843F8205003B030BD24D5066069
:10BDC0002DE9F041164688B00C467149804605F0D1
:10BDD00057F805462EB3042E10D014F0030703D1F4
:10BDE0006C4B22689A4252D03246214640460E277A
:10BDF000FFF7D0FF384608B0BDE8F081A30703D1B4
:10BE0000644B22689A4275D000232246A9682868AC
:10BE1000FBF7F6FDEB6853F82070384608B0BDE834
:10BE2000F08114F0030603D15A4B22689A420AD0DB
:10BE300005A90220CDE90554FFF714FE0E27384668
:10BE400008B0BDE8F08102AA2146806805F0F4F848
:10BE5000002800F09A800399AA68EB680298521AA9
:10BE6000441A920003EB810103EB800031F08AFE5B
:10BE70003146C4EB8472D5E902309200234400EBD2
:10BE8000830031F093FEAB682344AB60D6E701AA90
:10BE900030466946FBF772FD05AA2146A86805F001
:10BEA000CBF8002871D0009ADDE905618C1B141BCA
:10BEB000002C2DDDAB6868682344834249D8E868CC
:10BEC000164400EB81019A1B00EB8600920031F0D2
:10BED00059FE009A0598EB689200019903EB8000E7
:10BEE00031F050FEAB680E2723443846AB6008B0F3
:10BEF000BDE8F0812146806805AA05F09DF800287C
:10BF000033D105AAD5E9020105F0BAF8074671E771
:10BF1000E8689200019900EB860031F033FE069943
:10BF2000059B009ED5E902203344521A00EB8101A3
:10BF300000EB8300920031F025FEA868C4EB847208
:10BF4000EB6820443946920003EB800031F02EFE6E
:10BF5000C8E79900E868F0F7C3FAAB68E8602344E3
:10BF6000009A6B60059E0699AAE7DDE90530C01AC4
:10BF7000FFF740FE0599EB680746D0E9022003EB86
:10BF80008101920031F0CEFD34E70020FAF788FD00
:10BF900024D50660B0DC06602DE9F0478046406895
:10BFA00000218000F0F77EFAD8F804108146C1B174
:10BFB00008F10806071F002505E047F8040FD8F828
:10BFC0000410A9420DD956F8040F0135FAF7CCFA3E
:10BFD00004460028F1D14846F0F790FA2046BDE823
:10BFE000F0874B46D8F808000022BDE8F047F9F783
:10BFF0001BBF00BF2DE9F0410E4604461146104A12
:10C0000030461D46FAF73EFFB01C013E002180007D
:10C01000F0F748FA8046C0E900462B68836066B1B5
:10C0200000F1080700240134002155F8040FFAF745
:10C0300027FAA64247F8040FF5D14046BDE8F08143
:10C04000FEFF0500F0B51646126883B005460C46A3
:10C05000002A3AD0456809012B799B070FD441F09B
:10C0600006017068F0B10191F0F7A6FE0199024651
:10C070002846FDF74DFC0023336003B0F0BD41F0CE
:10C0800006010022281D01914AF0E6F91D4B019995
:10C090009D420BD00028F0D0426873689A42EAD0E3
:10C0A00003B0F0BD2846FDF767FCE4E7164CD4F872
:10C0B000C450002DD5D10120FDF79AFBF0F77CFE8E
:10C0C00001990546C4F8C400CBE70F01406847F06A
:10C0D0000607043039464AF0BFF918B143683360A7
:10C0E00003B0F0BD0E2CC8D06B680246E621181DC7
:10C0F0004AF0B2F90028C0D039464068F9F7F0FE9E
:10C100003060BAE770E606600004002070B50C46A7
:10C11000054600224FF4BB71606804304AF09CF978
:10C12000B0B1406802F090F806466068002240F620
:10C13000A63104304AF090F960B1406802F084F80A
:10C140003246034607492846BDE87040F1F7ACBFC8
:10C15000054EEAE7324628460449BDE87040F1F74B
:10C16000A3BF00BF9CD5066084300860B4D50660CC
:10C1700070B5044601221048240144F0060421460B
:10C180004AF06AF9456806460DB1284670BD01219E
:10C190000820F0F787F9094B054601202B60FDF7D1
:10C1A00027FBF0F709FE22464FF4BB716860FDF7EC
:10C1B000AFFB2846756070BD8804002000D806607B
:10C1C000406870474160704770B5054682B00022F4
:10C1D00014482D0145F0060529464AF03DF904466C
:10C1E00018B16468204602B070BD024629460E4868
:10C1F0004AF032F904460028F4D046686A46112114
:10C200003046F9F7F9FE009B002BEAD000216A4680
:10C210000846F9F77DFE0122294602484AF01CF93A
:10C220004660DEE788040020C4D506600E20704713
:10C230000B461146002210B504461846FAF722FEB6
:10C2400000210420F0F72EF9046010BD820700B52C
:10C2500083B00DD1084A0168914209D1074AC368E9
:10C26000934205D101A904F05DFB03B05DF804FB26
:10C270000348F9F735FD00BF74E306605509026015
:10C280005CF906604368184730B587B08C461146A4
:10C290001A4602AD0A4B04466046009304230195FA
:10C2A000FAF786FE00211020F0F7FCF80460029AED
:10C2B0004260039A8260049AC26007B030BD00BF3A
:10C2C000ACD8066038B504460D4610200021F0F7C2
:10C2D000E9F8844694E80F008CE80F006046CCF83B
:10C2E0000C5038BD38B504460D4610200021F0F73B
:10C2F000D9F8844694E80F008CE80F006046CCF82B
:10C30000085038BD38B504460D4610200021F0F71E
:10C31000C9F8844694E80F008CE80F006046CCF81A
:10C32000045038BD032304300B607047032A02D049
:10C330000249F1F795BA0249F1F792BAD87406604A
:10C3400028D9066038B50C46064905462368DA88C0
:10C35000F1F7AAFE2168224628464031BDE8384060
:10C36000FCF7FABA6CD9066038B513688BB9046863
:10C37000E56B6DB104F13C0C02E00133AB4207D038
:10C380005CF8044FA142F8D1023350F82330136017
:10C3900038BD0148F9F76CFCE0FB066010B4C46BD3
:10C3A0006CB100F13C03002002E00130A04206D055
:10C3B00053F8042F8A42F8D15DF8044B70474FF0D0
:10C3C000FF305DF8044B70472DE9F0470C46C16B18
:10C3D00007469246A51898468D423CD14FEA8409FB
:10C3E00000212846554403F001FD414606464A46D1
:10C3F00040F8087B31F096FB09F108004FEA8A0209
:10C400000021304431F0D2FBAC4217D208F10409CC
:10C4100058F8240001F094F801463846FFF7BEFFB3
:10C42000431C0ED006EB800CDCF8083073B959F8C9
:10C4300024300234AC42CCF80830E9D33046BDE8B1
:10C44000F0870A4606480749F9F7AEFB0A46044852
:10C450000549F9F7A9FB2A460448F9F749FC00BF4A
:10C46000CCCF0660D40A07607CFF06600C00076032
:10C470002DE9F041074610300D4600218000F0F70D
:10C4800011F880463C22002131F090FBC8F83C7046
:10C4900067B1043D08F13C060024013455F8040F4F
:10C4A00001F04EF846F8040FA742F6D14046BDE829
:10C4B000F08100BF30B585B0019101F041F8019BDA
:10C4C0000446184A1A40062A25D09A0703D1164A6C
:10C4D000196891421FD003AA184602A9134DFBF711
:10C4E0004DFADDE90201FFF7C3FF8822104982807F
:10C4F000104A01600261104A10490262104AC48069
:10C500004162104C10494261104AC5608261C0E925
:10C510000A4105B030BD01A9012002F07FFD0346AC
:10C520000190D8E70F0080FFA0DF0660C9C301605B
:10C5300074E3066045C3016015FB0160A5FB016063
:10C5400069C30160B9FC016031FA016050E2066024
:10C55000C368002B06DDD0E901218A4207DB0021F8
:10C5600008467047FBD0D0E901218A42F7DD51002F
:10C57000134441F0010143600846704710B4D1E90B
:10C580000143CA681B1B002A1344CCBF03F1FF33CD
:10C590000133042893FBF2F30DD0052807D123EAD9
:10C5A000E3705DF8044B400040F00100704700204C
:10C5B0005DF8044B7047002B5DF8044BCCBF3E2068
:10C5C0001E20704710B4C368D0E90142CB60084612
:10C5D000034BC1E901420B605DF8044B704700BF9B
:10C5E000CCD9066038B50C460546D1E90123094986
:10C5F000F1F75AFDE268012A05D028460649BDE850
:10C600003840F1F751BD28460449BDE83840F1F7FC
:10C6100027B900BF78D9066088D9066050DA06606D
:10C62000F8B514460D46174A0746214628461E46C9
:10C63000FAF728FC00211020EFF734FF002304460E
:10C64000C0E9007301239D42C36030680AD0FBF744
:10C6500095F860607068FBF791F8032DA06006D034
:10C660002046F8BDFBF78AF8A0602046F8BDB06808
:10C67000FBF784F8E0600028F2D17C210248F9F74A
:10C6800023FB00BF0600020040F80660136810B5E7
:10C69000144603B110BD922908D096290BD09529D4
:10C6A000F8D1C068FEF7AEFD206010BD4068FEF70F
:10C6B000A9FD206010BD8068FEF7A4FD206010BDBC
:10C6C000042A30B5044685B025D1D0E90123C068DD
:10C6D000A3EB020C00288444CCBF0CF1FF3C0CF10E
:10C6E000010C11F003059CFBF0FC2CEAEC7003D16B
:10C6F0001A4B0A689A4211D00A4600230146206864
:10C70000FBF77EF9E268636802FB0030400040F00E
:10C71000010005B030BD002005B030BD01AA04F015
:10C720008BFC29461020EFF7BDFE0D4B0360019AEC
:10C73000E168636801FB02334360029AE168636861
:10C7400001FB023383600399E268002901FB02F2D6
:10C75000C260DEDAE2689B1A8360DAE7B0DC06606A
:10C7600090D90660034610B4806850B1441E04227C
:10C77000586861009C605DF8044B41F00101FBF7D3
:10C78000A9BA5DF8044B704770B50E4682B01D46DD
:10C79000114604464FF002123046FAF773FBD321DC
:10C7A00028686A46F9F728FC0099264641B100211D
:10C7B0006A460846F9F7ACFB0446204602B070BD55
:10C7C0000C20EFF76FFE0446066028686060FBF7F8
:10C7D00081F9FAF7D3FFA060204602B070BD00BF18
:10C7E000830709D10068064B984207D0054BC01A51
:10C7F000B0FA80F040097047002070470120704770
:10C80000F4DA0660B8DA066030B4D0E902536C6836
:10C810009C4217D96FF04042E9681A4401EB82014B
:10C8200001E09C420ED051F8042F4FEA830C0133F3
:10C83000002AF6D0042AF4D0C360EB6830BC53F869
:10C840000C007047002030BC704700BF10B4054A90
:10C850000023054CC1E90203C1E9004208465DF826
:10C86000044B704709C8016070D80660012204308B
:10C8700008B5FAF74BFD0E2008BD00BF02220430B8
:10C8800008B5FAF743FD0E2008BD00BF38B50B46CA
:10C890000446002118460434F9F7F2FD054601E08C
:10C8A000FAF734FD2846F9F75FFE014601222046DB
:10C8B0000029F5D138BD00BF0128F8B506460F465E
:10C8C00009D90D460124013455F8041F3868FFF7D3
:10C8D000DDFFA642F7D10E20F8BD00BF38B50B46EC
:10C8E0000446002118460434F9F7CAFD054601E064
:10C8F000FAF70CFD2846F9F737FE014603222046D9
:10C900000029F5D10E2038BD30B50B4685B0044660
:10C9100069461846F9F7B4FD0434054602E0FAF713
:10C92000F5FC50B92846F9F71FFE014600222046C3
:10C930000029F4D13E2005B030BD1E2005B030BD29
:10C9400038B5044600211020EFF7ACFD23680546FA
:10C9500040F8043B6168FAF7CDFCA368E868AB6077
:10C960006268E168920031F0DDF8284638BD00BF0A
:10C9700010B582B00191FFF7E3FF04460199FFF77C
:10C9800085FF204602B010BD10B582B00191FFF7BF
:10C99000D7FF04460199FFF7A1FF204602B010BD62
:10C9A000043008B5FAF780FD0E2008BD2DE9F843E4
:10C9B00080460F463AB3D1F80090B8F1010F1FD965
:10C9C000012609F1040505E001362846FAF76CFD59
:10C9D000B04515D057F8040F8145F5D00021F9F77F
:10C9E0004FFD044601E0FAF791FC2046F9F7BCFD43
:10C9F0000146022228460029F5D10136B045E9D189
:10CA00004846BDE8F8830868FFF79AFF8146D4E7F7
:10CA10000022FFF7CBBF00BF012208B5FFF7C6FF1A
:10CA20000E2008BD2DE9F8438B070D46064603D1BD
:10CA3000304B0A689A4246D0AB685BB32E49304609
:10CA4000F0F70EFF6A68002A4DD04FF0000800246E
:10CA500001202A4F07E001223046FAF7A7FD6A6855
:10CA60000020A2421CD9EB684FEA840953F8241035
:10CA700001340029F5D00429F3D00028EBD1394640
:10CA80003046F0F7EDFEEB6853F80910E3E71C4978
:10CA9000F0F7E6FE30461B49BDE8F843F0F7E0BE8C
:10CAA00019493046F0F7DCFEB8F1000F05D1BDE8BA
:10CAB000F88315493046F0F7D3FE30461349BDE8F8
:10CAC000F843F0F7CDBE8B68002BE0D01049F0F7AB
:10CAD000C7FE09493046F0F7C3FE6A68002AE8D06D
:10CAE0004FF00108B3E730460749BDE8F843F0F7D7
:10CAF000B7BE00BFB8DA066048CA0660A8C60660BE
:10CB000044DA06604CDA0660F86C066050DA0660BB
:10CB100054DA066010B5022204300C46FAF7F6FB30
:10CB200008B10E2010BD21460148F9F7D9FF00BF1A
:10CB300028CE06600528F8B50D4605D006280ED08B
:10CB4000042806D00020F8BD8868400040F00100AD
:10CB5000F8BD8B68002B14BF3E201E20F8BD11F0DD
:10CB60000300EFD10C4B0E689E42ECD14F6877B1B9
:10CB70000446EB6853F82410013431B1042904D081
:10CB80000620F9F7C1F806EB6006A742F1D1700064
:10CB900040F00100F8BD00BFB8DA066008B5043007
:10CBA000FAF75CFC00B108BD8C2202490248F8F794
:10CBB000FBFF00BFD007076028CE06602DE9F041DB
:10CBC00006460D4610200021EFF76CFC0B4B074684
:10CBD0008046314647F8043B3846FAF78BFB56B19E
:10CBE000043D00240134012255F8041F3846FAF7A9
:10CBF0008DFBA642F6D14046BDE8F081F4DA06602E
:10CC00002DE9F8430C460021804691460846FFF77F
:10CC1000D5FF002107462046F9F732FC08F104064B
:10CC2000054603E02146FAF771FB68B92846F9F793
:10CC30009BFC044600223046002CF3D1B9F1000FD2
:10CC400008D13846BDE8F88301222146381DFAF79D
:10CC50005DFBEBE7D8F80C00EFF750FC7B68C8F8F9
:10CC60000430BB68C8F80830FB680E27C8F80C30E1
:10CC70003846BDE8F88300BF814201D0FFF7C0BF4E
:10CC80000AB10E207047FFF75BBE00BF0022FFF71E
:10CC9000F3BF00BF814202D00122FFF7B1BF0E20D7
:10CCA000704700BFF8B50C460646114602222046E2
:10CCB0001F46FAF7E7F83CB921462046FFF77EFF0A
:10CCC000054606602846F8BD00210846FFF776FFB6
:10CCD000054600213868F9F7D3FB2F1D044601E013
:10CCE000FAF714FB2046F9F73FFC014601223846CB
:10CCF0000029F5D128462E60F8BD00BF2DE9F0418E
:10CD000086B014460546CDE90010FFF769FD0028FE
:10CD100044D00027009E3046FFF762FD002833D044
:10CD20004FF000081CB1AA68B3689A421CD0204B8F
:10CD3000341D049502931F4B03930023059302E0D7
:10CD4000FAF7E4FA80B102A8FFF75EFD014600227F
:10CD500020460029F4D13E244FB9B8F1000F0CD180
:10CD6000204606B0BDE8F0811E24002FF5D0281D16
:10CD7000FAF79AFBB8F1000FF2D0301DFAF794FBE6
:10CD8000204606B0BDE8F08102466B4601210A4804
:10CD9000FFF788FF4FF001080646C3E7024601ABE4
:10CDA00001210548FFF77EFF01270546B2E700BFD6
:10CDB00070D8066009C80160F4DA06600022FFF747
:10CDC0009DBF00BF0B46002201461846FFF796BFE5
:10CDD000F0B511F0030783B00C4616460546CDE9C1
:10CDE00000120FD1464B0A689A422AD0242D3A46A7
:10CDF0000CD100223146201DFAF788FA002857D0BE
:10CE00003E241BE000221746242DF2D03046FFF7C7
:10CE1000E7FC90B11C2D10D8DFE805F03C432A2E2A
:10CE2000350F0F0F0F16204C0F0F0F540F0F0F0F52
:10CE30000F0F18225A0F0F0F61000024204603B075
:10CE4000F0BD01221746DFE7002F54D12046FFF73F
:10CE500077FD31460446FFF719FDEFE7002F45D176
:10CE60002046FFF76DFD31460446FFF737FDE5E745
:10CE7000A268B3689A421BD1204600223146FFF7D0
:10CE80003DFF0446DAE7214600223046FFF736FF31
:10CE90000446D3E7204601223146FFF72FFF044620
:10CEA000CCE7214601223046FFF728FF0446C5E7BC
:10CEB0001E24C3E720463146FFF7DEFE002F08BFE1
:10CEC0000446BBE769460220FFF770FD0446B5E75C
:10CED000204600223146FFF7CFFE0446AEE700228F
:10CEE00069460220FFF762FD0446A7E73146204667
:10CEF000FFF7F4FCA2E769460220FFF7DDFC9DE79F
:10CF0000F4DA066001220430FAF700BA0B4602494F
:10CF10005A68F1F7C9B800BF6CD9066070B504460D
:10CF20000D46104E1049F0F79BFC0122696820461F
:10CF3000FAF73CFB31462046F0F792FC0122A96843
:10CF40002046FAF733FB31462046F0F789FCE968C2
:10CF500020460122FAF72AFB20460449BDE870402A
:10CF6000F0F77EBCA8C60660A8DC066050DA066052
:10CF70002DE9F041114E0C461D461146864219D14D
:10CF80000F4A2046F9F77EFF012C0FD0032CD5E97C
:10CF900000870CBFAC680E2400211020EFF782FA46
:10CFA000C0E90068C0E90274BDE8F0810E242F6872
:10CFB000A046F1E70348F9F773FD00BFB0DC066057
:10CFC00006000200BC0E0760136803B17047922987
:10CFD0000ED0962909D095290DD040F2613399429F
:10CFE000F4D1064BC2E90030F0E783681360704764
:10CFF000436813607047C36813607047CCDC0660F9
:10D0000070B506460D46102000211446EFF74AFA87
:10D01000024AC4600260C0E9016570BDB0DC066010
:10D020002DE9F0410746C0680C4690460E2841D0D5
:10D03000FAF7A4FB061E4CD021DD78680E281CD020
:10D04000FAF79CFB051EB8BF2D1925EAE575A54228
:10D05000A8BF2546B8680E2809D0FAF78FFB031E33
:10D06000B8BF1B1923EAE3739C42A8BF1C46C8F84B
:10D070000860C8E90054BDE8F0810025EAE7786857
:10D080000E2808D0FAF77AFB0028B8BF001940EA4A
:10D09000E075A54200DB651EB8680E280FD0FAF7D0
:10D0A0006DFB0028B8BF001940EAE070A0420EDB1B
:10D0B000013CDCE7786801260E28C1D1DDE74FF09E
:10D0C000FF34C8F80860C8E90054BDE8F0810446A0
:10D0D000CDE740F2A3410148F8F7F6FD40F80660BD
:10D0E00010B5044686B00846FEF74EF96A4601467A
:10D0F0002046FFF795FF029B03205B00DDE900124D
:10D1000043F001034C0003A95200059344F00104CD
:10D1100042F00102CDE9034202F068FE06B010BD04
:10D120003E2818BF1E280CBF0123002302D010F098
:10D13000010301D0184670478207FBD103680348FA
:10D140001B1AB3FA83F35B0918467047F4D30660E1
:10D1500008B50146FFF7E4FF18B901F00303022BFD
:10D1600000D008BD02480840063818BF012008BD9D
:10D17000070080FF10B4054A0023054CC1E90203F3
:10D18000C1E9004208465DF8044B7047D1E00160F8
:10D1900070D8066008B5FAF7C9F903460348D9887C
:10D1A00097290CBF42229722F8F7A2FD3CFB0660AC
:10D1B000884210B503D20378303B092B00D910BD4B
:10D1C0000023864613601EF801CBACF1300C03EB54
:10D1D0008303714570460CEB43031360EFD01EF8D8
:10D1E00001CBACF1300C5FFA8CF4092CEFD910BDF7
:10D1F0002DE9F84F8D188B4606461F46A9426AD284
:10D200000B46002206E0BCF1220418BF01249D4217
:10D2100009D944B113F801CBBCF1270FF3D1012296
:10D220009D421446F5D8002A4ED0002C4CD0222422
:10D2300022222F493046F0F737FFDFF8C480DFF8AD
:10D24000C490DFF8C4A00EE05C2A2ED01F2A1CD99F
:10D250007F2A1AD00FB1130622D425493046F0F7A1
:10D2600023FF5D450AD91BF8012BA242ECD12246CF
:10D2700020493046F0F718FF5D45F4D82246304685
:10D280001B49BDE8F84FF0F70FBF0A2A12D00D2A4C
:10D2900015D0092A04D149463046F0F7E1FAE0E713
:10D2A00041463046F0F700FFDBE713493046F0F720
:10D2B000D7FAD6E711493046F0F7D2FAD1E751460E
:10D2C0003046F0F7CDFACCE727220949304627242B
:10D2D000F0F7EAFEB1E7272205491446F0F7E4FE2D
:10D2E000304603492246BDE8F84FF0F7DDBE00BFE7
:10D2F000DCDC0660D4DC0660D8DC0660E0DC0660BE
:10D30000ECDC0660E8DC0660E4DC06602DE9F8434E
:10D310000C461546214906462544F0F7A1FAAC42D1
:10D3200021D2013C013D1E4FDFF88480DFF884905C
:10D330000BE00A2A27D00D2A2AD0092A1ED04146FE
:10D340003046F0F7B1FEA5420DD014F8012F222A85
:10D350000FD05C2A0DD01F2AEBD912493046F0F7C6
:10D36000A3FEA542F1D130460C49BDE8F843F0F7E1
:10D3700077BA39463046F0F797FEE4E7494630463B
:10D38000F0F76EFADFE708493046F0F769FADAE7B6
:10D3900006493046F0F764FAD5E700BF4CCA06608C
:10D3A000D4DC0660DCDC0660E0DC0660E4DC066001
:10D3B000F4DC0660E8DC066099422DE9F047DDF810
:10D3C00020901F46804692460FD3B9F1000F10DD22
:10D3D000CE1A002408EB04053A465146284630F0A0
:10D3E0000DFC18B1B4424C44F4D100252846BDE8E8
:10D3F000F087CC1A0026EDE7F8B5074615460E462D
:10D4000010200021EFF74EF804460760856086B1D2
:10D4100029463046EFF744FF00216060681CEFF7B3
:10D4200041F831462A46E060064630F07BFB002397
:10D4300073552046F8BD00BF08B5EFF799FF00010E
:10D4400040F0060008BD00BF194B984270B5064673
:10D450000C461CD000211020EFF724F8066061680C
:10D4600005468160A068EFF71BFF6860A068D4E9FB
:10D4700000310131994207D1AA680023E860835442
:10D48000A3602360284670BDEFF72AF8F4E7D1E9DE
:10D490000110EFF725FF05460028DBD020462D01BF
:10D4A000F0F7D2F8002345F006052360EAE700BF55
:10D4B000A0DF066038B504460D46EFF711FF18B13E
:10D4C000000140F0060038BD2A4621460248BDE86A
:10D4D0003840FFF791BF00BFA0DF066010B4074CD3
:10D4E0000B46844204D006485DF8044BFFF784BF26
:10D4F000114618465DF8044BFFF7DCBFA0DF06605D
:10D500003CDD066003460A4601481946FFF774BF32
:10D510003CDD066000B5024687B0114602A80192C4
:10D52000F0F76CF8019A0021049830F03FFB02A953
:10D530000248FFF789FF07B05DF804FB3CDD066099
:10D5400008B50A4B0340062B0BD083070BD1084BC1
:10D5500002689A4207D1D0E90210BDE80840EFF70F
:10D5600007BF000908BDFFF715FE00BF0F0080FFD1
:10D57000A0DF0660054B0340062B03D083680B60D9
:10D58000C06870470009EFF7D5BF00BF0F0080FFEC
:10D59000F0B50C4687B011460646062220461D46C9
:10D5A000F9F770FC8CB1012C12D16A46102102A847
:10D5B000F0F73EF8296868460022F9F7F7FF02A95C
:10D5C0003046FFF741FF07B0F0BD162007B0F0BDB1
:10D5D0002868830703D1224B02689A420ED002A921
:10D5E0000122FAF743FBDDE90201F0F761FE98B38F
:10D5F000DDE90201FFF75EFF07B0F0BD6946FFF706
:10D60000B9FF2A68174B04461340062B1FD05568F4
:10D6100075B100992046F0F74BFEE8B1009920461D
:10D62000EFF75EFE014648B1000140F00600CAE790
:10D6300000992046EFF734FE0546EAE7009F1020E8
:10D64000EEF730FF06604560C0E90274BBE71009E1
:10D6500048F012FF0546DBE700210348F8F794FA8B
:10D660003CDD06600F0080FFE8CF0660012800B5B2
:10D6700083B006D10A6840F6162369460220CDE938
:10D6800000230B46002201460248FFF781FF03B04A
:10D690005DF804FBA0DF06602DE9F04304468BB083
:10D6A0000191F9F743FF02A906462046FFF762FF02
:10D6B000019B07469A075FD0354AD46801AB002228
:10D6C00001213348A0470346019004AA03A9184644
:10D6D000FAF754F9039D2DB30024DFF8C0802546E6
:10D6E00005E00134039B8068A34205441AD9049BDA
:10D6F0004FEA840953F82400F9F718FF864243D112
:10D700000CB1029B1D44049B53F8090000EA080277
:10D71000062AE6D100090134EFF7FAFE039B05441F
:10D72000A342E4D8294606A8EFF768FF039B089DAB
:10D73000DBB10024049B05A953F824000134FFF752
:10D7400019FF059A0146284630F0ECF9039B059A2B
:10D75000A342154409D9002CECD02846029A394638
:10D7600030F0E0F9029B1D44E4E706A93046FFF7DC
:10D770006BFE0BB0BDE8F0831968054A9142A4D056
:10D780000448814299D1A0E70348F8F7A9FA00BFFD
:10D7900024D5066050E20660200307600F0080FF7A
:10D7A000F0B585B0254B0C46013802AD0431CDE90A
:10D7B00000350123F9F790FB2068F9F7B7FE002147
:10D7C00007460846FEF7B6FA03A906462068FFF7A3
:10D7D000D1FE039D01460544A84211D20A461378A2
:10D7E000944601320A2B0ED00D2B1FD09542F6D84D
:10D7F000521A3846FFF772FE01463046FDF73CFFED
:10D80000304605B0F0BD01249DF80830ACEB0102B4
:10D8100003B1224464443846FFF760FE01463046B7
:10D82000FDF72AFFA542EBD92146D7E79CF8013046
:10D830000A2B14BF01240224E6E700BF18DD0660AE
:10D840002DE9F04F87B00C460746086898460392CA
:10D85000F9F76CFE06466068F9F768FE864250D11B
:10D8600004A92068FFF786FE05A905466068FFF752
:10D8700081FE049A022F824605EB020B16D8A946B8
:10D88000CB452CD3039B5246ABEB09014846009392
:10D89000059BFFF791FD10B31D4B9E4229D0401B05
:10D8A000400040F0010007B0BDE8F08FA3680E2BE8
:10D8B0001DD0012130460091294601F0A5FE814688
:10D8C000032FDDD0E3680E2BDAD001222946304643
:10D8D0000092049A01F098FE8346CB45D2D2B8F16B
:10D8E000000F11D14FF0FF3007B0BDE8F08FA9460F
:10D8F000E6E701462846F0F741FC400040F0010011
:10D90000D1E76068FFF746FC0248F8F7D5F900BF99
:10D91000A0DF0660A409076000230122FFF790BF83
:10D9200000234FF0FF32FFF78BBF00BF01231A46E1
:10D93000FFF786BF01234FF0FF32FFF781BF00BF23
:10D940002DE9F04F8BB00C461546029010680592F9
:10D95000F9F7ECFD012C064607905FD06868F9F7EF
:10D96000E5FD864271D1059B09A958680391FFF72F
:10D9700001FEDDF8248007460399059B1868FFF730
:10D98000F9FD029B0646012B099B06934BD04FF0F5
:10D99000010A0024069D35B300234FF001099B4680
:10D9A0000393049302E0013D544419D0012332193A
:10D9B00041463846CDF80090FFF7FEFC0028F2D132
:10D9C000BBF1000F18D1029B002B36D0029B012B1C
:10D9D00037D0013D4FF0010BCDE903445444E5D16C
:10D9E000BBF1000F0AD11B4B079A1B489A4208BF94
:10D9F00016200BB0BDE8F08F0394D4E7039A049B84
:10DA00000132D21A069B9A4212D0049B07983344E3
:10DA10001946FFF763FD0BB0BDE8F08F4FF0060825
:10DA20000E4F09A9A9E74FF0FF3A03EB0A04B1E74B
:10DA3000059B18680BB0BDE8F08F069B04941A1B79
:10DA4000E0E7621CCDF810B0DCE7059B5868FFF7F3
:10DA5000A1FB00BFA0DF06602CDD066098DF06603A
:10DA600003460A4602201946FFF76ABF03460A46E4
:10DA700000201946FFF764BF03460A4601201946F5
:10DA8000FFF75EBF70B586B00C46054601A9FFF7EB
:10DA900071FD06462046F9F771FE019B044683425C
:10DAA00017D2014602A8EFF7A9FD224620210498CB
:10DAB00030F07CF8019A04983146A41A00EB540027
:10DAC00030F030F82846F9F731FD02A9FFF7BCFC29
:10DAD0000546284606B070BD2DE9F04F04282DED0F
:10DAE000028B8FB0059100F0AC804FF0FF330393B1
:10DAF000059C2068F9F71AFD034660681D4608EE8C
:10DB0000903AF9F713FD059BA842044640F0A68021
:10DB10009868F9F70BFD844240F09C80059C07A9AA
:10DB20002068FFF727FD08A904906068FFF722FD31
:10DB300009A98346A068FFF71DFD08EE100ADDE97C
:10DB40000743A34276D84FF00009002B6AD1B9F100
:10DB5000000F05D0099A18EE101A48462FF0E2FF80
:10DB60004FF00108039B099E984561D0002C5FD0BF
:10DB70002346DDF820A04C46049F994601235A46CF
:10DB80004946384600935346FFF716FC054618B33E
:10DB9000BAF1000F00D10135A4B3EA1BA019394630
:10DBA00016442FF0BFFF099A18EE101AA0192FF093
:10DBB000B9FFDDF820A0049B08F10108079905EBE7
:10DBC0000A07099A1944039B16449845A1EB0709D3
:10DBD00002D0B9F1000FD1D14B46A1461C46B9F194
:10DBE000000F12D02246394609EB06002FF09AFFAB
:10DBF0000AA918EE900AFFF727FC0FB0BDEC028BC4
:10DC0000BDE8F08FEF1B3E44D5E73119B8F1000FA6
:10DC100010D00AA8EFF7F2FCDDF83090DDE90743F9
